:020000040000FA
:107800005469616E59696E673130300000000000C4
:1078100054593230302E3038303030306200000071
:10782000424154333247313339474B3634464200B4
:1078300043414E5F5354440000000000000000002C
:1078400043414E5F43485F300000000000000000ED
:1078500043414E5F3530304B6270730000000000D2
:10786000E8070000E0070000DF070000000000005C
:020000040000FA
:10800000802F0020DD800000E5800000E780000078
:108010000000000000000000000000000000000060
:10802000000000000000000000000000EF800000E1
:108030000000000000000000F380000001A9010022
:108040005D0B0100A10B0100D10B0100010C01002F
:10805000310C0100610C0100910C0100C10C010008
:10806000F10C0100210D0100550D0100690D010009
:10807000790D0100AD0D0100BD0D0100CD0D010018
:10808000010E0100450E01008D0E0100D50E01000C
:108090001D0F0100650F0100750F0100A90F010000
:1080A000DD0F01000D1001004110010075100100ED
:1080B0008510010095100100C9100100FD1001009C
:1080C000EF3FE8FF0448854600F02CFA00480047DF
:1080D0003DEB0100C046C046802F00201648804777
:1080E00016480047FEE7FEE7FEE7FEE7FEE7FEE78D
:1080F000FEE7FEE7FEE7FEE7FEE7FEE7FEE7FEE758
:10810000FEE7FEE7FEE7FEE7FEE7FEE7FEE7FEE747
:10811000FEE7FEE7FEE7FEE7FEE7FEE7FEE7FEE737
:10812000FEE7FEE7FEE7FEE7FEE7FEE7FEE7FEE727
:10813000FEE7FEE7FEE700000DAF0100C58000008E
:1081400030B50B46014600202022012409E00D46EF
:10815000D5409D4205D31D469540491B2546954077
:1081600040191546521E002DF1DC30BD70B50024BB
:108170002546002801DA01244042002901DA0125C0
:108180004942FFF7DDFFAC4200D04042002C00D056
:10819000494270BDF0B51FB40646002082B00546C6
:1081A0004024019100901BE0019922460F46304681
:1081B00000F066F9049A059B801A994110D3104685
:1081C0001946224600F04CF9361A8F410197224693
:1081D00001200021009F00F043F938184D41009024
:1081E0002046641E0028DFDC019B009829463246A9
:1081F00007B0F0BDF0B51FB486B00020009001902C
:1082000002900698069980B204900798090C02041F
:108210000014114307900027089D099806913E46D7
:108220003C4603900398A9B20204000C0390049802
:108230002D0C154348430021224600F011F9C719BF
:10824000714110340E46402CECDB3846029A00F0A7
:1082500007F9009A019B80180090594102980191FA
:10826000103002904028CCDB00980BB0F0BD0346E4
:108270000B439B0703D009E008C9121F08C0042A5A
:10828000FAD203E00B780370401C491C521EF9D24D
:108290007047D2B201E00270401C491EFBD2704709
:1082A0000022F6E710B513460A4604461946FFF7C2
:1082B000F0FF204610BD30B504460020034600E024
:1082C0005B1C934203D2E05CCD5C401BF8D030BD18
:1082D0000321001D401E037812021A43491EF9D5DE
:1082E00010467047034603220870000A491C521EBC
:1082F000FAD518467047024670B54A40D30FDB07DF
:1083000040002DD04A002AD0010E140E00021202A5
:108310000919400A520A8418E50104465443000A28
:10832000120A2E045043A4194219200CC543AA185E
:10833000120C0125AD03521C521912047F3924047A
:1083400000D0521C104301D44000491EC2B20C069A
:10835000C0092018401C4008802A02D003E00020F9
:1083600070BD40084000002900DA0020184370BDAD
:1083700070B502464A40D50F40004A00ED0740085C
:108380005208002814D0002A12D0C40DD30D410287
:108390000120C0055202490A520AE41A09181218AB
:1083A0007D34914201D3641C00E04900002C01DAC5
:1083B000002070BD0023914201D3891A0343400875
:1083C00049000028F7D100290AD0914202D10121A9
:1083D000C90705E0914201D2012101E00121C94311
:1083E000E005C018401900F05CF870BD10B500221F
:1083F0009623114600F05DF810BDC20FD207400071
:1084000040080BD0C10D0723DB01C9184002090544
:10841000400A1143C208400711437047002001463B
:108420007047000010B5002904DB0124E407404236
:108430008C412146002B04DB1C460123DB07524202
:10844000A341994200D1904210BD00000122D20701
:10845000002800DB101A002900DB511A88427047FF
:1084600010B5202A04DB0146203A9140002010BDBF
:10847000914020239C1A0346E3401943904010BDCD
:1084800010B5202A04DB0846203AD040002110BD58
:108490000B46D340D0402024A21A914008431946ED
:1084A00010BD002904DA401C490001D140084000F9
:1084B000704770B40024050C05D11024000402D1CB
:1084C000002921D01124050E01D100020834050F26
:1084D00001D10001241D850F01D18000A41C0028BA
:1084E00001DB4000641C002908D020252E1B0D460E
:1084F000F540A14000D001212943084301061B1B80
:10850000000ADB1D02D5002070BC7047DB0518187F
:1085100080180029F8DA401C4900F5D170BC4008E9
:1085200040007047064C0125064E05E0E36807CC85
:108530002B430C3C98471034B442F7D3FFF7C6FDE9
:108540001CFF01003CFF010070B58C180578401C31
:108550006B075B0F01D10378401C2A1106D102780A
:10856000401C03E006780E70401C491C5B1EF9D1CC
:108570002B0705D40023521E0DD40B70491CFAE7BB
:108580000378401CCB1A921C03E01D780D70491C27
:108590005B1C521EF9D5A142D8D3002070BD70B526
:1085A00006F078FE0524204616F082FA00252846BB
:1085B00006F064FE204616F07BFA0126304606F0EF
:1085C00039FE204616F074FA284606F033FE20469F
:1085D00016F06EFA304606F051FE204616F068FAA4
:1085E00070BDB0B506F056FE0524204616F060FAC0
:1085F0000125284606F042FE204616F059FA284684
:1086000006F018FE204616F053FA002006F012FE7F
:10861000204616F04DFAB0BDF0B581B006F026FE4A
:10862000052016F045FA08270026012006F002FE74
:108630000524204616F03CFA204616F039FA06F0DA
:108640000BFE0546204616F033FA002006F0F2FD38
:10865000204616F02DFA76002E437F1E3806E4D110
:10866000F0B201B0F0BD70B50446002006F0E2FDA6
:1086700006F010FE052016F01BFA0826E0B2C0092D
:1086800006F0FCFD0525284616F012FA012006F03A
:10869000D1FD284616F00CFA002006F0CBFD284646
:1086A00016F006FA284616F003FA6400761E300625
:1086B000E4D1052016F0FCF9012070BDF0B583B0BF
:1086C000019314460E4607460120384302900325C5
:1086D00004E000F08EF86D1E280631D000F067F837
:1086E0003846FFF7C0FF00F0A7F80028F1D1304668
:1086F000FFF7B9FF00F0A0F80028EAD100F057F822
:108700000298FFF7B0FF00F097F80028E1D1019838
:1087100002280BD3451E0026FFF77EFF2070FFF7CF
:108720003EFF641C761CF0B28542F5DCFFF774FF57
:108730002070FFF756FF00F05CF8202003B0F0BD7A
:10874000102003B0F0BDF0B583B01C46009201913B
:108750000290032504E000F04CF86D1E280623D09B
:1087600000F025F80298FFF77EFF00F065F800287A
:10877000F1D10198FFF777FF00F05EF80028EAD109
:10878000002C0CD00026009F3878FFF76CFF00F01B
:1087900053F80028DFD1761C7F1CA642F4D300F0EA
:1087A00028F8082003B0F0BD102003B0F0BDB0B52C
:1087B00006F070FD0524204616F07AF901252846BA
:1087C00006F038FD204616F073F9284606F056FDEF
:1087D000204616F06DF90025284606F04FFD20468C
:1087E00016F066F9284606F025FD642016F060F9BB
:1087F000B0BDB0B506F04EFD0524204616F058F980
:108800000025284606F016FD204616F051F92846A8
:1088100006F034FD204616F04BF90125284606F0F7
:1088200009FD204616F044F9284606F027FD64208D
:1088300016F03EF9B0BD0000B0B506F017FD0524F6
:10884000204616F035F9012006F0F4FC204616F01B
:108850002FF90B4D06F000FD044606F0E5FC002C58
:1088600002D06D1E2804F5D10525284616F020F902
:10887000002006F0DFFC284616F01AF92046B0BDAD
:1088800033210000034801780B2901D8491C0170ED
:108890007047C0466F2B002070B584B0002503954B
:1088A00002950195009506F0BFFC0F20C6430E4CC3
:1088B0001036F1B2A0206A461023FFF744FF20468D
:1088C00016F0F6F8204616F0F3F8912EF0D3A0201B
:1088D000B0216A461023FFF736FF204616F0E8F86D
:1088E0000248058004B070BD581B0000622B0020B8
:1088F00070B5022902D2EB24E0B270BD891EEB25CF
:108900000022134605E0401C5B1CDDB2A94225464F
:108910000EDB04786C40154604E034466E1C072DCF
:108920003546F0D26608E407F7D09A246640F4E7AB
:10893000E0B270BDF0B591B00C91417810AA117001
:1089400083781B025918C37804792402E3181B04A6
:1089500059180B0ED3700C0C94700D0A55700B91B6
:1089600008956918099409190A93C9180278D2431D
:108970008918427983791B029A18C379047A2402F0
:10898000E3181B049A188918130A0693C918130CC4
:108990000593C9180792120E04928918827AC37A35
:1089A0001B029A18037B0F90447B2402E3181B04DC
:1089B00098180918020A02928918020C0192891863
:1089C0000D910390000E0E9000200346014606E034
:1089D00032409A40D2B211435B1C082B0ED00126C4
:1089E00035469D400746024602E07F1C042FEFD02B
:1089F00010ACE45D2542F8D0521CF6E70E9C0D98B1
:108A00000019C3B20F98827B934205D0427A9142FB
:108A100002D1002011B0F0BD1021FFF769FF0C99C1
:108A2000CC72019A8A72029A4A72039A0A72049A62
:108A3000CA71059A8A71069A4A71079A0A710A9A46
:108A4000CA70099A8A70089A4A700B9A0A7011B013
:108A5000F0BDF0B58DB055220270002747720B783B
:108A60004370CA79059202728A790492C2714A7976
:108A7000039282710A7902924271CA7A0892427311
:108A80008A7A019202734E7AC6720C7A84720CAAA8
:108A900013704D782D02EB188D78C97809024919A9
:108AA0000904CB18190E01711D0CC57009931B0A1E
:108AB0000B90837038460A91D17007959570069394
:108AC000537031020919089A1202019BD21812043C
:108AD0005118089103990902029A8918059A1202FD
:108AE000049BD2181204511805913D463A4605E000
:108AF0002640AE4032436D1C082D0ED00124214685
:108B0000A9400346064602E05B1C042BF0D00CAFE4
:108B1000FF5C3942F8D0761CF6E70B9B5A72099835
:108B200006994018079940180A994018059A801824
:108B3000110A4018110C4018110E4018089A80189C
:108B4000110A4018110C4018110E4018563898732D
:108B500010211846FFF7CCFE0DB0F0BDF0B58FB078
:108B60000446FF20E070A07060700F20C0430290A8
:108B70000F302070704815F09BFF7049086863281B
:108B800001D8642008606E4F002038806D4E01903F
:108B9000308008E00B99814222D338881030388029
:108BA00080B2A1286DD206F03FFB3978A02003AA3D
:108BB0001023FFF783FD30802028EED103AD0BA9F1
:108BC0002846FFF7B7FEE97B8842E6D1287855288A
:108BD000E3D15D48017800290298DBD10846D9E746
:108BE0003888A0284DD8C0B20021019105E006F0D8
:108BF0001BFB3988C8B2A12943D2C1B2A02003AA65
:108C00001023FFF75BFD3080398810313980202830
:108C100037D103AD07A92846FFF78CFEE97B8842D0
:108C2000E5D128785528E2D14748007800280299F4
:108C300000D1014607988842D9D240490A68962156
:108C400051430B9A824208D90818904219D30BA9B4
:108C50000E222046FFF70BFBC9E78918814210D38B
:108C600007A90E222046FFF702FB0BA80A99818173
:108C700007980B9008980C9009980D9038880190EF
:108C8000B5E72078617809020818A178E278120225
:108C9000511809040818401C24D100200190388084
:108CA000A020B02103AA1023FFF708FD3080202860
:108CB00018D103AD0BA92846FFF73CFEE97B88429B
:108CC00010D1287855280DD11F480078002800D1F0
:108CD00002900B980299884204D20BA90E222046DA
:108CE000FFF7C5FA2078617809020818A178E278C0
:108CF0001202511809040818401C0CD10020E0721F
:108D0000A07260722072E071A07160712071E070D9
:108D1000A070607020700198388020786178090216
:108D20000818A178E27812025118090408180749B6
:108D3000086030880FB0F0BD701101005C2B00207E
:108D4000622B0020582B00205B2B0020682B00207A
:108D5000F0B581B000910646214800250570002A33
:108D60002ED01446C036631B71190F200840102204
:108D7000101A834200D303461A480278102A01D001
:108D8000042A1AD1C809FE2707405F2F13D80127EC
:108D9000B8436038C0B29E3282420CD3009A521956
:108DA000C9B2DFB23B46FFF789FC0F490880ED19D5
:108DB000A542D8D304E0082000E004200A49088036
:108DC000094801880020042902D0082900D0012088
:108DD00003490870411E8841400001B0F0BDC04603
:108DE0006E2B00205A2B00206C2B00200A4A0123F6
:108DF00013700A4A10700A4A11600A4A0021116071
:108E0000042801D105218901102801D11D208101EB
:108E1000054801807047C0465B2B00205A2B00207C
:108E20005C2B0020682B0020602B0020F0B587B061
:108E3000994D00262E80994B1B688B4224D1994C6A
:108E40002188202925D1029000920196964C002776
:108E50002760964D964E2878062809D806F0E4F942
:108E60002068401C2060B042F5D38D480421018069
:108E70002F70904C20880107029B31D08848202118
:108E80000180854D019E0BE001204002844908804D
:108E900006E003A8FFF762FE208081488021018060
:108EA0007F4800883F2807DD874988420BDC40283F
:108EB00012D0802810D010E004280DD008280AD045
:108EC000202809D009E001214A02904204D0C902B9
:108ED000884201D001E002262E80288807B0F0BD2C
:108EE000A128019E00D32780009A012A6A4D1ED135
:108EF000187B012856D1DF719F715F711F711F733D
:108F0000587B012804D1DF729F725F721F725F73FA
:108F100003AF38461946FFF79CFDF87320880028F8
:108F200046D01038C1B2A02003AA102344E0002A82
:108F3000B6D1614801780029B2D00270187859780A
:108F4000090208189978DA781202511809040818E9
:108F50005A490978002901D00F21C943884233D2E8
:108F6000274603AC20461946FFF773FDE0733978B6
:108F7000A02010232246FFF7E6FB029A484908800A
:108F800008288DD13888103038801078517809023F
:108F900008189178D2781202511809040818484923
:108FA00008607DE7597B012911D10128A3D0A7E7EB
:108FB000A02003AA10230146FFF7C5FB384908800B
:108FC0003D48009901706BE70120C0025EE73D4813
:108FD0000078012812D103AC20461946FFF739FD6D
:108FE000E073A020B02110232246FFF7ACFB2C49F0
:108FF00008800828E4D133480770E1E718785978E9
:10900000090208189978DA78120251180904081828
:109010002B490968214A12685118884203D2204816
:1090200040210180CCE725490978002901D00F2192
:10903000C94388422DD203AF384619461C46FFF774
:1090400008FDF8731B480178A02010233A46FFF76B
:109050007AFB134908800828B2D1164908881030D5
:1090600008802078617809020818A178E278120255
:109070005118090408181249086008490A6815219E
:109080005143FFF75DF800299AD101200D4908707E
:1090900096E70120C00291E7742B00205C2B002092
:1090A000722B0020582B0020782B00206F2B0020E3
:1090B000818D5B00622B0020642B00205B2B002045
:1090C000682B0020702B0020FF010000F0B585B058
:1090D0000646434C0027278004921018414A128804
:1090E000904241D201910397404F00200290386096
:1090F0003F4C404D2078052809D806F095F838688F
:10910000401C3860A842F5D33748042101800298FA
:1091100020703948018839480278102A01D0042A81
:1091200032D188190346C033049C651A0F240440C9
:109130001020001B854200DB0546DC09603C01264F
:109140003002E7B27F09052F12D3B443E6B29E3254
:10915000B242234C039F0DD301984218D9B2EBB20F
:109160003046FFF7F0FA05E01F482021018011E0AA
:109170001B4C039F1C49088008280BD1E8B21E4AEB
:1091800011880818108005E0012080021649088027
:10919000134C039F144800881F2809DD202813D092
:1091A00001210A0290420FD0890288420CD00CE0C3
:1091B000042809D0082808D10F480088049988425B
:1091C00001D3022700E001272780208802210143E4
:1091D000022902D1084900220A8005B0F0BDC0462C
:1091E000742B0020602B0020722B0020782B002095
:1091F0006F2B0020818D5B007C2B00205A2B0020E0
:10920000F0B585B0044600200190042C6FD20BF01D
:1092100075FB002801D10BF0F1FB0020009000BF8E
:109220000098401C00900BF069FB03900398002805
:1092300003D0484900988842F2D30398002856D1B9
:10924000042145480BF03CFB444845490880210176
:10925000444A515C4900404A505A41490A88012118
:10926000090300F055F902900120049020013D49C6
:1092700040184078002801D100264BE020013949F0
:1092800040184078012802D13548068842E0200184
:1092900034494018407802282AD120014018057925
:1092A0002901304A515C49002B4A505A2C490A88FE
:1092B0000121090300F02CF9064628012A49431828
:1092C0002801284940180289280140180021C76850
:1092D0003046B84706462801224BC018C2882801EC
:1092E000C0188178304600F087F8064612E02DE07D
:1092F00020011C4940184078032804D02001401860
:109300004078132804D1200116494018868801E0CE
:10931000002004900498002818D020011249431816
:109320002001104940180289200140183146C768C1
:109330000298B847019020010A4BC018C28820014A
:10934000C0188178019800F057F80190019805B095
:10935000F0BD000050C300000C0100208813000085
:1093600006010020C0F5010000F60100F8B5054631
:109370000E4614460020009001211C4801751C482F
:10938000007888431A490870084680780821084305
:109390001749887000208871084600780121084329
:1093A0001349087008460572002717E01048007836
:1093B000802108430E49087000BF0E48007D002838
:1093C000FBD000200B4908750948C0892080A41CE7
:1093D0000748C1890098081800907F1CB742E5D360
:1093E00031460098FEF7ACFE80B2F8BD4061004007
:1093F000005004404060004010B50346012908D1E8
:10940000094CA41A9C4202D99C18A0B20BE0064851
:1094100009E0022906D1934202DD9C1AA0B202E0C3
:10942000002000E0184610BDFFFF000010B5044604
:109430000121202001F0D0FF0020324908700121D5
:1094400031480175002031490875152015F018F8CC
:109450002C488078E17808432A498870084680784B
:1094600021780843274988702078802806D108464B
:109470000079E17949000843224908712148807840
:10948000E17A08431F498870A078002803D1084674
:10949000007908710FE0A078012806D119480079F9
:1094A000602108431749087105E0164800798021BA
:1094B00008431449087113488079217908431149F8
:1094C000887108468079617908430E498871207A4D
:1094D000C872607A88720846007838218843094942
:1094E0000870084600786178C9000843054908708B
:1094F000A07A0873084600780121084301490870E2
:1095000010BD000000500440406100404060004039
:10951000F8B504460E461746002E01D100250FE08F
:10952000A64201DC3D460BE00094009C20467843B7
:10953000009031460098FEF703FE0090009885B237
:109540002846F8BD0146042904D28A00024BD218ED
:10955000508800E000207047AC2400200146042918
:1095600003D28A00024B985C00E0002070470000A4
:10957000AC240020FFB587B004460898844203DA83
:109580000A988068002802D12448019042E0089897
:10959000001B82B20292002625460A9880680021AC
:1095A0002F463A463346049605910690FEF722FE72
:1095B00005460E46002328463146029AFEF7EAFD8C
:1095C00005460E46304600210A46494050400143B8
:1095D00002D0124801901DE003950A98C068039DCF
:1095E000A84202D30020019014E00A98C1680398B1
:1095F000401A039009990398FEF7A2FD039003987F
:10960000000C0004002802D00448019002E00398F6
:1096100080B2019001980BB0F0BD0000FFFF000088
:1096200010B5084800788021884306490870012158
:1096300005480175002005490875152014F020FF24
:1096400010BD0000005004404061004040600040F8
:10965000F8B505460E4614461F4621462846FEF735
:1096600085FD80B2F8BD0000FFB587B006460A98B8
:109670004068002801D1029035E00A9801684068EE
:1096800008180390002534460021274603980695C4
:109690000491059038462946049B059AFEF7AAFDD9
:1096A00004460D460A984068024600230190204671
:1096B0002946FEF76FFD04460D4600232046294645
:1096C000099AFEF767FD04460D46284607492140E2
:1096D000002359405840014303D00448C04302903E
:1096E00001E0A0B2029002980BB0F0BD0000FFFFB5
:1096F00010B5FE4800688079030014F0A7FE070546
:109700009ED8F5F4F3F2F100F848006840790300C0
:1097100014F09CFE0805138A2A8A468A638A11F08F
:1097200027F80020F1490968C873F04800684079BB
:10973000401CEE49096848717DE0ED494969EB4AF2
:109740001268D27A885C11F08BF8E848006840799A
:10975000401CE64909684871E44800684079401CAB
:10976000E2490968487166E009F008FC002810D158
:1097700011F076F8DD4800684079401CDB49096843
:109780004871DA4800684079401CD8490968487136
:1097900005E011F017F80020D449096848714AE043
:1097A00009F0ECFB002811D1112011F059F8CF4835
:1097B00000684079401CCD4909684871CB48006871
:1097C0004079401CC9490968487105E010F0FAFF6A
:1097D0000020C649096848712DE009F0CFFB002838
:1097E0001BD1C2480068C07A401CC0490968C872D1
:1097F000BE480068C07ABE49097888420DDB002067
:10980000BA490968C872B94909684862B748006826
:109810008079401CB5490968887110F0D3FF002099
:10982000B2490968487106E010F0CCFF0020AF494A
:109830000968487100BF00BF32E3AC480068407C53
:10984000002817D0AA48C068002803D0A848C168DB
:10985000192088470020A54909684862A348006884
:109860008079401CA1490968887100209F490968D6
:1098700048711BE09D480068406A282807D29B4831
:109880000068406A401C9949096848620EE000205F
:10989000964909684862954800688079401C934958
:1098A000096888710020914909684871F8E28F4879
:1098B00000684079030014F0C9FD080518A42FA41E
:1098C0004CA480A410F054FF002088490968C87394
:1098D000864800684079401C84490968487197E0CF
:1098E000D4E2C7E230E25DE194E0814949697F4A10
:1098F0001268D27A885C10F0B3FF7C480068407927
:10990000401C7A4909684871784800684079401CD1
:109910007649096848717BE009F030FB002811D1D5
:10992000012010F09DFF714800684079401C6F498C
:10993000096848716D4800684079401C6B490968A6
:10994000487105E010F03EFF002068490968487141
:109950005EE009F013FB002828D164490968C97A40
:1099600024225143634A12688918604A1268D27BE4
:10997000885C10F075FF5D480068C07B401C5B4947
:109980000968C87359480068C07B242814D3574815
:1099900000684079401C554909684871534800687F
:1099A0004079401C51490968487105E010F00AFFF0
:1099B00000204E49096848712AE009F0DFFA0028C2
:1099C00018D14A480068C07A401C48490968C872E2
:1099D00046480068C07A4649097888420ADB002078
:1099E00042490968C872414800688079401C3F4973
:1099F0000968887110F0E6FE00203C49096848714A
:109A000006E010F0DFFE002038490968487100BF09
:109A100000BF45E2354800684079030014F016FDA8
:109A20000A0614B92BB948B978B995B910F0A0FE57
:109A300000202E490968C8732C4800684079401CF2
:109A40002A4909684871ABE029494969274A1268DF
:109A5000D27A885C10F004FF244800684079401CEA
:109A6000224909684871214800684079401C1F4913
:109A70000968487194E009F081FA002811D14A2060
:109A800010F0EEFE194800684079401C174909683B
:109A90004871164800684079401C144909684871AB
:109AA00005E010F08FFE002010490968487177E04A
:109AB00009F064FA002824D1FF2010F0D1FE0B48F1
:109AC0000068C07B401C09490968C87307480068E2
:109AD000C07B24281BD3054800684079401C0349FB
:109AE0000968487101480068407905E0D007002006
:109AF000402B0020CC070020401CEA49096848712F
:109B000005E010F05FFE0020E6490968487147E073
:109B100009F034FA002811D1FF2010F0A1FEE1482D
:109B200000684079401CDF4909684871DD480068D9
:109B30004079401CDB490968487105E010F042FE9D
:109B40000020D849096848712AE009F017FA00286E
:109B500018D1D4480068C07A401CD2490968C8723C
:109B6000D0480068C07AD049097888420ADB0020D2
:109B7000CC490968C872CB4800688079401CC94943
:109B80000968887110F01EFE0020C64909684871F6
:109B900006E010F017FE0020C2490968487100BFB6
:109BA00000BF7DE1BF4800684079030014F04EFC1F
:109BB0000C0715C32CC349C366C382C39FC310F0EF
:109BC000D7FD0020B7490968C873B64800684079D6
:109BD000401CB44909684871B4E0B3494969B14AC5
:109BE0001268D27A885C10F03BFEAE48006840797B
:109BF000401CAC4909684871AA4800684079401C7B
:109C0000A849096848719DE009F0B8F9002811D108
:109C1000772010F025FEA34800684079401CA14938
:109C2000096848719F4800684079401C9D4909684F
:109C3000487105E010F0C6FD00209A490968487196
:109C400080E009F09BF9002811D10C2010F008FEEB
:109C5000944800684079401C9249096848719148CD
:109C600000684079401C8F490968487105E010F090
:109C7000A9FD00208B490968487163E009F07EF96D
:109C8000002810D110F0ECFD864800684079401C97
:109C9000844909684871834800684079401C8149BB
:109CA0000968487105E010F08DFD00207D490968C4
:109CB000487147E009F062F9002811D1132010F033
:109CC000CFFD784800684079401C764909684871A2
:109CD000744800684079401C72490968487105E081
:109CE00010F070FD00206F49096848712AE009F002
:109CF00045F9002818D16B480068C07A401C6949B2
:109D00000968C87267480068C07A6749097888425C
:109D10000ADB002063490968C872624800688079DC
:109D2000401C60490968887110F04CFD00205D49B5
:109D30000968487106E010F045FD0020594909689E
:109D4000487100BF00BFABE056480068407903008F
:109D500014F07CFB080513872A874787638710F078
:109D600007FD00204F490968C8734E4800684079D4
:109D7000401C4C49096848717AE04B494969494A95
:109D80001268D27A885C10F06BFD46480068407912
:109D9000401C444909684871424800684079401CA9
:109DA00040490968487163E009F0E8F8002811D1DA
:109DB000492010F055FD3B4800684079401C394966
:109DC00009684871374800684079401C354909687E
:109DD000487105E010F0F6FC00203249096848712E
:109DE00046E009F0CBF8002810D110F039FD2D48DD
:109DF00000684079401C2B4909684871294800686F
:109E00004079401C27490968487105E010F0DAFCE8
:109E100000202449096848712AE009F0AFF80028B9
:109E200018D120480068C07A401C1E490968C872D1
:109E30001C480068C07A1C49097888420ADB002067
:109E400018490968C872174800688079401C15498C
:109E50000968887110F0B6FC002012490968487141
:109E600006E010F0AFFC00200E490968487100BF01
:109E700000BF15E000200B4909688871094909688D
:109E80004871062007490968C87009E010F09AFC7B
:109E9000002004490968487102490968887100BFB7
:109EA00000BF10BDD0070020402B002010B56A482D
:109EB00000684079030014F0C9FA090610C627C6E5
:109EC00044C6608EC60010F053FC634800684079B9
:109ED000401C614909684871BCE0604949695E4AB3
:109EE0001268D27A885C10F0BBFC5B48006840794D
:109EF000401C594909684871574800684079401C1E
:109F0000554909684871A5E009F038F8002811D1D1
:109F10007F2010F0A5FC504800684079401C4E4955
:109F2000096848714C4800684079401C4A490968F2
:109F3000487105E010F046FC002047490968487167
:109F400088E009F01BF8002810D110F089FC424885
:109F500000684079401C4049096848713E480068E3
:109F60004079401C3C490968487105E010F02AFC22
:109F700000203949096848716CE008F0FFFF0028AB
:109F800022D135480068C07A401C33490968C8723C
:109F900031480068C07A3149097888420FDB0020D7
:109FA0002D490968C8722C4800684079401C2A492C
:109FB00009684871002028490968486208E00020C3
:109FC00025490968487103E0002023490968487160
:109FD00010F0F8FB3EE020480068407C002816D0D6
:109FE0001E48C068002803D01C48C1681920884753
:109FF00000201949096848621749096848711649DB
:10A0000009688871052014490968C8701AE0124867
:10A010000068406A282807D20F480068406A401C40
:10A020000D49096848620DE000200B490968486243
:10A030000949096848710849096888710520064975
:10A040000968C87006E010F0BDFB002002490968ED
:10A05000487100BF00BF10BDD0070020402B00207A
:10A0600010B50024F7480068807A01287ED1F548B1
:10A070000068C07900287AD0F2480068807900280A
:10A0800004D0012874D0022873D191E1ED48006812
:10A09000007B24286ED2EB480068C07901287AD171
:10A0A000002475E0E7480068C07A24214843E64967
:10A0B00009684018E3490968097B415CE148006888
:10A0C000C07A24225043E14A12688018DD4A12689F
:10A0D000127B805C814229D0DA480068C07A242152
:10A0E0004843DA4909684018D6490968097B415C48
:10A0F000D4480068C07A24225043D34A126880189A
:10A10000D04A1268127B8154CE480068407B2428D4
:10A1100005D3CC480068007BCA4909684873C94820
:10A120000068007BC7490968887308E0C548006873
:10A13000407B242803D20120C24909688871C148A4
:10A140000068007B401CBF4909680873BD4800686F
:10A15000007B242808D3BB480068407B242803D216
:10A160000120B84909688871B64805E0D3E1CDE11E
:10A1700069E0BAE138E00EE00068007B242804D2F0
:10A18000B04800688079012800D103E0601CC4B2A7
:10A19000242C87D356E0002413E0AA480068C07A34
:10A1A00024214843A94909684018015DA548006871
:10A1B000C07A24225043A44A126880180155601CBA
:10A1C000C4B2242CE9D300209E4909684873232097
:10A1D0009C490968887301209A490968887124207C
:10A1E0009849096808732DE00020964909680873AA
:10A1F00094480068C07A401C92490968C872914826
:10A200000068C07A92490978884217DB8D48006857
:10A21000007C012804D102208A490968887106E07F
:10A22000002088490968887186490968C87100203A
:10A2300084490968C8728349096808740020814903
:10A240000968487161E17F4800684079030014F0B3
:10A25000FDF8080513A62AA651A68EA60120794965
:10A260000968087410F084FA764800684079401C48
:10A2700074490968487199E075494969714A1268D9
:10A28000D27A885C10F0ECFA6E4800684079401C85
:10A290006C49096848716B4800684079401C6949FD
:10A2A0000968487182E008F069FE00281BD1654901
:10A2B0000968497B491CC8B210F0D2FA61480068AD
:10A2C000407B60490968C8735E4800684079401C5B
:10A2D0005C49096848715B4800684079401C5949ED
:10A2E0000968487105E010F06DFA002055490968C9
:10A2F00048715BE008F042FE00282BD15149096803
:10A30000C97A24225143504A126889184D4A12686A
:10A31000D27B885C10F0A4FA4A480068C07B401CDD
:10A3200048490968C87347480068C07B45490968BF
:10A33000897B88421ADD434800684079401C4149C6
:10A34000096848713F4800684079401C3D490968E8
:10A3500048710BE010F036FA3A480068407B394902
:10A360000968C87300203749096848711EE008F081
:10A3700005FE00280CD13349096888712420314931
:10A380000968C8732F49096848732E49096888739A
:10A3900010F018FA00202B490968487106E010F007
:10A3A00011FA002027490968487100BF00BFACE0DE
:10A3B000244800684079030014F048F808050F8E1F
:10A3C000268E4C8E688E10F0D3F91E4800684079B6
:10A3D000401C1C490968487185E01D494969194AB2
:10A3E0001268D27A885C10F03BFA1648006840790F
:10A3F000401C144909684871124800684079401CA3
:10A400001049096848716EE008F0B8FD002811D1C4
:10A41000492010F025FA0B4800684079401C094992
:10A4200009684871074800684079401C0549096877
:10A43000487105E010F0C6F900200249096848712A
:10A4400051E00000D0070020CC070020C807002002
:10A45000402B002008F092FD002810D110F000FAE7
:10A460009C4800684079401C9A490968487199489D
:10A4700000684079401C97490968487105E010F070
:10A48000A1F900209349096848712CE008F076FD95
:10A4900000281AD18F480068C07A401C8D4909688D
:10A4A000C8728C480068C07A8B49097888420CDBF6
:10A4B000002088490968C8728649096888718549F9
:10A4C0000968487183490968C87110F07BF9002058
:10A4D00080490968487106E010F074F900207D4950
:10A4E0000968487100BF00BF0FE010F06BF9002051
:10A4F0007849096848717749096888717549096818
:10A50000087374490968C87200BFE2E0002071490D
:10A5100009688872DDE06F480068807A0228F4D10B
:10A520006C480068007A002879D06A480068407951
:10A53000030013F08BFF0B0711BB25BB41545EBB1F
:10A540007590BB0010F014F9624800684079401C17
:10A55000604909684871B7E05F494969087810F0B7
:10A560007FF95C4800684079401C5A490968487185
:10A57000584800684079401C564909684871A3E072
:10A5800008F0FCFC002810D110F06AF9514800686E
:10A590004079401C4F49096848714E48006840792D
:10A5A000401C4C490968487105E010F00BF9002087
:10A5B00048490968487187E008F0E0FC002807D1A5
:10A5C000444800684079401C42490968487103E0EA
:10A5D000002040490968487110F0F4F874E010F068
:10A5E000C7F83C4800684079401C3A4909684871FE
:10A5F0006AE0394949690978491CC8B210F030F954
:10A60000344800684079401C324909684871314833
:10A6100000684079401C2F490968487154E054E0B3
:10A6200008F0ACFC00280FD110F074F82949096833
:10A630008870012010F0E8F8264800684079401C36
:10A6400024490968487105E010F0BCF80020214950
:10A650000968487138E01F480068807811280CD1DB
:10A6600000201C4909680872AA201A4909688870E4
:10A67000002018490968487011E0164800684078C1
:10A68000401C144909684870124800684078032843
:10A6900005D308F013FD00200E490968487010F03A
:10A6A00091F800200B49096848710DE010F08AF814
:10A6B0000020084909684871064909684870AA20BD
:10A6C00004490968887000BF03E000200149096857
:10A6D000887210BDD0070020402B002010B5024624
:10A6E0009000074BC018405C002802D00320C043F4
:10A6F00010BD01209300024C1B1958540020F7E7AD
:10A70000E826002070B5002508E06D1C1B48854236
:10A7100002D20AF09FF901E0002503E00AF0EEF80A
:10A720000028F2D100BF022100200AF0F5F8032131
:10A7300000200AF0F1F8052100200AF0EDF80721C9
:10A7400000200AF0E9F8002408E00020A1000C4AEB
:10A750005054A10089184880601CC4B2042CF4D362
:10A7600001200849087000204870052088700020EA
:10A77000C87005480549088070BD000050C300003E
:10A78000AC240020080100208813000006010020EE
:10A79000F8B58D480078030013F058FE060405163E
:10A7A0003D5EFDFC0EE10AF029F900208649C870E3
:10A7B000487008468078002802D10320087002E023
:10A7C000022081490870FDE07F488078002804D08D
:10A7D0007D488078401E7C4988700AF08FF80028F8
:10A7E0000BD10AF00BF900207749C8700846807831
:10A7F00000280FD1032008700CE07348C078401C7B
:10A800007149C8700846C078052803D30520087030
:10A810000AF020F9D6E00AF071F800280ED10421E0
:10A820006A480AF04DF800206749C87048706848C7
:10A83000684908800420644908700CE06248C078C8
:10A84000401C6149C8700846C078052803D305201C
:10A8500008700AF0FFF8B5E05B49497809015E4AE3
:10A86000515C4900594A505A5A490A880121090342
:10A87000FEF74EFE009001255348407800015649EE
:10A8800040184078002801D100243CE04E48407830
:10A890000001514940184078012802D14D480488F0
:10A8A00031E04948407800014B494018407802287F
:10A8B00012D1454949780901474A89180879FEF7B4
:10A8C00041FE0446404949780901434A89180879FC
:10A8D000FEF744FE054616E03B48407800013E493D
:10A8E00040184078032806D03748407800014018C7
:10A8F0004078132806D13448407800013649401882
:10A90000848800E00025002D2FD02F4840780001DA
:10A91000324943182C48407800012F4940180289D9
:10A9200029484078000140182146C7680098B84778
:10A930000646254840780001274BC018C2882248A7
:10A9400040780001C01881783046FEF755FD064674
:10A950001D484078800022494018468001201A494D
:10A96000497889001E4A50540AE000201649497867
:10A9700089001B4A89184880134949788900505436
:10A9800011484078401C1049487008464078042817
:10A9900009D301E013E007E00AF030F800200A498B
:10A9A0004870032008700DE009F0A8FF002803D1CB
:10A9B00001200549087001E00AF04CF802E0FFF7B9
:10A9C000A1FE00BF00BFF8BD080100200C0100205F
:10A9D0008813000006010020C0F5010000F6010008
:10A9E000AC24002010B509F053FF002405E000203E
:10A9F000A100074A5054601CC4B2042CF7D30020B5
:10AA0000044908700520887003480449088010BD77
:10AA1000AC2400200801002088130000060100205B
:10AA200070B50446002000F0AFF8002000F0DAF81E
:10AA3000002000F09BF8002000F0C4F8002000F097
:10AA400087F8002000F0AEF800BF012000F08EF87B
:10AA5000012000F0B7F8002521E0002000F086F882
:10AA6000002000F0AFF880202040002806D0012010
:10AA700000F08AF8012000F0B5F805E0002000F0B1
:10AA800083F8002000F0AEF800BF012000F06EF85F
:10AA9000012000F097F86006040E681CC5B2082D6E
:10AAA000DBDB012000F054F8012000F07BF870BDE2
:10AAB00070B504460D46012000F066F8012000F054
:10AAC00091F8002000F052F8002000F07BF8002000
:10AAD00000F03EF8002000F065F800BF012000F013
:10AAE00045F8012000F06EF8002628E0002000F074
:10AAF0003DF8002000F066F880202040002803D0B8
:10AB0000012000F041F802E0002000F03DF8802034
:10AB10002840002803D0012000F064F802E0002063
:10AB200000F060F800BF012000F020F8012000F0E4
:10AB300049F86006040E6806050E701CC6B2082EA1
:10AB4000D4DB012000F004F8012000F02BF870BDE8
:10AB500010B50446002C04D0812103200AF008F827
:10AB600003E0802103200AF003F810BD10B504466D
:10AB7000002C04D08121042009F0FAFF03E0802199
:10AB8000042009F0F5FF10BD10B50446002C04D0D8
:10AB90008121022009F0ECFF03E08021022009F06E
:10ABA000E7FF10BD10B50446002C04D081210448F5
:10ABB00009F0DEFF03E08021014809F0D9FF10BD54
:10ABC0000107000010B50446002C05D081210720A4
:10ABD000000209F0CDFF04E080210720000209F007
:10ABE000C7FF10BD10B50446002C04D081210448D5
:10ABF00009F0BEFF03E08021014809F0B9FF10BD54
:10AC00000207000010B5F920FFF70AFF8820FFF7C0
:10AC100007FF9020FFF704FF9820FFF701FF0821AE
:10AC20000846FFF745FFE820FFF7FAFE1221084625
:10AC3000FFF73EFFA020FFF7F3FE70210846FFF765
:10AC400037FFA820FFF7ECFE70210846FFF730FF22
:10AC5000B020FFF7E5FE70210846FFF729FFB82076
:10AC6000FFF7DEFE00210846FFF722FFC020FFF7B6
:10AC7000D7FE00210846FFF71BFFC820FFF7D0FED4
:10AC800000210846FFF714FFD020FFF7C9FE2F214F
:10AC90000846FFF70DFFD820FFF7C2FE2F21084618
:10ACA000FFF706FFE020FFF7BBFE2F210846FFF766
:10ACB000FFFE4020FFF7B4FE00210846FFF7F8FE34
:10ACC0000A20FFF7ADFE002405E000210846FFF74B
:10ACD000EFFE601CC4B25A2CF7DB00240AE000200F
:10ACE0000B4908550B4908550B4908550B490855A0
:10ACF000601CC4B25A2CF2DB8120FFF791FE0020C9
:10AD0000074908708870C8700871487010BD00004D
:10AD1000EC21002046220020A0220020FA22002060
:10AD2000D000002010B58020FFF77AFE10BD000093
:10AD30000020044908700120034908700020487071
:10AD400070470000D5000020D000002010B5484812
:10AD5000007800287AD046488078030013F076FB0C
:10AD60000604434A535A687E414800794149085CC9
:10AD70003F490979404A515C884209D13C480079F1
:10AD80003E49085C3A4909793D4A515C88421BD0EA
:10AD9000374800793749085C35490979364A5054B3
:10ADA000334800793549085C31490979344A5054AF
:10ADB0002F48C078002803D004202D49887011E066
:10ADC00001202B4988700DE000202949C8700846F1
:10ADD0000079401C0871084600795A2802DB0020DF
:10ADE0000871087041E04020FFF71AFE0220204958
:10ADF00088703AE01E4A11791079FFF759FE032056
:10AE00001B49887031E00A20FFF70AFE0420184928
:10AE100088702AE0164A1279194B995C144A127903
:10AE2000154B985CFFF744FE0520114988701CE023
:10AE30000F480079401C0E490871084600795A28CD
:10AE400005DB002008710870C87003E00EE00120E7
:10AE50000749C87000200649887006E000200449B0
:10AE600008708870C870087100BF00BF10BD000076
:10AE7000D0000020EC21002046220020A02200204B
:10AE8000FA22002010B510F0AFF8012811D10E48B9
:10AE900000780A2806D1FF22A5320021012011F0F6
:10AEA0008DFD0FE04B22D2000021012011F086FD24
:10AEB00008E00020054988804880002211460120D2
:10AEC00011F07CFD10BD0000200100201C000020BE
:10AED000002003490872487088704860704700007D
:10AEE000D00C002058221152704710B504460121A1
:10AEF000022000F071FA0021022000F06DFA10BD6E
:10AF0000014600205322525C10231A40002A08D028
:10AF10005322525C0C231A409210032A18D10320AA
:10AF200016E05422525A0123DB031A40002A0ED0A5
:10AF30005322525C0C231A409210032A05D053224C
:10AF4000525C9207920F032A01D1022000E00120F7
:10AF500070470246002058239B5A0B40002B01D01B
:10AF6000012000E000207047014600226020405A86
:10AF7000FF231B0218400005020F1001014BC018EF
:10AF8000704700000055044010B5002A0AD056232F
:10AF90001B5A0C0223435624235256231B5A8B431D
:10AFA000235209E056231B5A0C02A3435624235272
:10AFB00056231B5A0B43235210BD0000F8B504461C
:10AFC0000D46012700263448844203D10121022086
:10AFD00000F002FA2878401EA0702088FF2101317D
:10AFE000084320802088400840002080A878401E28
:10AFF000C1B25A20015568790007000CE9790902AD
:10B000000843A97908435C210853288981B240206C
:10B010000153A868C000C10C42200153A88981B225
:10B0200044200153E868C000C10C46200153288A1F
:10B0300081B2482001532869C000C10C4A20015345
:10B04000A88A81B24C2001536869C000C10C4E200F
:10B0500001535020005B297909020843502108530D
:10B060005020005B297988435021085300E0761C6A
:10B070005020005B4007400F2979884202D00748E2
:10B080008642F4D15020005B4007400F2979884266
:10B0900000D000273846F8BD00540440FFFF0000F0
:10B0A00030B5034600201C898C4209DD082A05D2F0
:10B0B00018244C431D682C19A05C02E0002000E01D
:10B0C000002030BD10B5024613898B4205DD1823E0
:10B0D0004B431468E318987C00E0002010BD014643
:10B0E000FF22C889C007C00F00280AD00120C881EC
:10B0F00000E0521EC889C007C00F002801D0002AF6
:10B10000F7D1C889C007C00F00280FD10220C8811D
:10B110000420C881487A400840004872487A3823A1
:10B120009843487200204872012070470020FCE7D5
:10B130000246507A012318435072507A0B78DB0094
:10B1400018435072087A012808D1888850814868CD
:10B15000000C0123DB031843908108E0087A0028E3
:10B1600005D15081486880001A4B18409081487A78
:10B17000012804D1507A40231843507206E0487ADF
:10B18000002803D1507A4023984350720878002851
:10B1900011D1C87A1072087B1070487B5070887B80
:10B1A0009070CB7BD370087C10714B7C5371887C82
:10B1B0009071CB7CD371887A002803D00120C00223
:10B1C000D08101E00820D081FF200130D081012012
:10B1D00070470000FC1F0000002904D0427A802341
:10B1E0001A43427203E0427A80239A4342727047C4
:10B1F00030B5024600200F4B5024A45A0D022C43B8
:10B200005025AC525024A45A8C43AC5200E05B1E33
:10B210005024A45A6407640F8C4201D0002BF6D14D
:10B220005024A45A6407640F002C01D0002000E0D1
:10B23000012030BDFFFF0000827A80231A40802A5F
:10B2400000D081727047000070B5044600250023CD
:10B25000002D02D00126602006530420C881888971
:10B260000126F6033040002808D00120107288899A
:10B27000C004C0084E893043506006E000201072C0
:10B2800088890F4E304080105060087AD0720023B9
:10B2900004E0CE5C10460C30C6545B1CD07A984259
:10B2A000F7DCC88904263040002804D1C889F6029A
:10B2B0003040002801D0002070BDD07AFCE70000AB
:10B2C000FC1F0000027C80231A40802A00D00174F9
:10B2D000704710B50246FF23D089C007C00F002871
:10B2E0000AD00120D08100E05B1ED089C007C00FCA
:10B2F000002801D0002BF7D1D089C007C00F00284B
:10B3000001D0002010BD507A012420435072507AA1
:10B310003824A0435072C87A1072487A00280FD19E
:10B32000087B1070487B5070887B9070CC7BD47009
:10B33000087C10714C7C5471887C9071CC7CD471E9
:10B34000FF200130D0814000D081107ADAE7000080
:10B35000F8B504460D460020002C00D100BF002A9D
:10B3600000D100BF012C01D141263043012A01D177
:10B3700012263043022C01D1C0263043022A01D1CB
:10B3800030263043134E307076788027BE43114FFD
:10B390007E70012C08D1FF2100BF0E4EB3781E46EF
:10B3A0000E4033468B42F8D10A4E76784027BE4392
:10B3B000084F7E70012A0BD10026009603E000BFE3
:10B3C000009E761C0096FF276937009EBE42F6D984
:10B3D000F8BD000000040240002905D0054A12789B
:10B3E0000243044B1A7004E0024A12788243014B74
:10B3F0001A70704720040240002905D0054A927E49
:10B400000243044B9A7604E0024A927E8243014B47
:10B410009A7670470008024001200649087000BF74
:10B4200004480078802108400028F9D00120024912
:10B4300008707047000C0240A401002070B503465C
:10B4400014460020002B01D1C0B202E00546803531
:10B45000E8B2012902D1051DE8B206E0022903D1B4
:10B4600005460835E8B200E0C0B2012C02D1851CC7
:10B47000E8B200E0C0B2084DA870AD7801263543AF
:10B48000054EB570002201E000BF521C7D252D0144
:10B49000AA42F9D970BD0000000C024070B500242A
:10B4A0002448007920210840002801D0224D3FE0A7
:10B4B00000F046F805462148007880210840002821
:10B4C00036D01E4880780840002801D01A4D02E08E
:10B4D00000F036F80546194880780007840F022CE2
:10B4E00001DBAD0804E0012C01D16D0800E000BFD4
:10B4F000124880788007C00F002801D02D0101E09C
:10B500000C2045430D4800784007840F002C02D1E1
:10B51000601CC4B207E0032C03D1601C4006040E7B
:10B5200001E06006040E21462846FCF709FE0546A8
:10B53000284670BD0004024000127A00000C024050
:10B5400000B5C0229178F82211401C4A12781143AC
:10B55000EA2923D00ADC0A46E03A130012F076FF0B
:10B560000A181C20242A2A2A2A161A2AED291FD052
:10B5700004DCEB2916D0EC291CD117E0F02903D00C
:10B58000F82917D10E4817E00E4815E00E4813E0D1
:10B590000E4811E00E480FE00E480DE00E480BE09B
:10B5A0000E4809E00E4807E00E4805E00E4803E0AB
:10B5B0000E4801E00D4800BF00BF00BD201C024046
:10B5C0000090D003006CDC020048E80100366E01F8
:10B5D0000024F400001BB70000127A00808D5B008D
:10B5E00000093D00C0C62D0080841E0040420F00AF
:10B5F00010B50446204600F05FFD002010BD00009D
:10B6000010B590211348FCF74BFE12481249086010
:10B6100012484860062008810020887206220F49DF
:10B620000D4800F04BFA00210B48FFF705FE802182
:10B630000B48FCF735FE0A480A4948600A4B0422C9
:10B640000A49084800F0CBFB55210648FFF73AFEAF
:10B6500010BD0000480800202808002030F201003A
:10B66000D808002034080020F1B50000C0F1010026
:10B670000C4A127812060B4B5B781B041A43094BD9
:10B680009B781B021A43074BDB781A43104642088B
:10B690004240D20083085A401146034A5140034AAF
:10B6A000116070471B0700200102000020070020E6
:10B6B000F8B504460F46A07A4006400E002874D123
:10B6C0000025ACE01820684321680818407C012858
:10B6D0003CD101211820684322681018017400260B
:10B6E0000CE018206843216808180830815D182094
:10B6F0006843226810188155701CC6B2082EF0D31A
:10B70000002118206843226810180174182068432B
:10B71000226810184174182068432268101841618B
:10B72000182068432268101881742C2068436168CF
:10B730000818406A002809D018236B432268D018E3
:10B740002C236B436268D218516A884718206843DB
:10B75000216808184069FF21C94388425DD8182034
:10B760006843216808184069C11918206843226895
:10B7700010184161182068432168081841692C207D
:10B780006843626810188069814246D31820684374
:10B7900021680818807C55283FD05521182068431F
:10B7A000226810188174002624E03CE018206843C9
:10B7B00021680818805D2C21694362685118103196
:10B7C000895D08401821694322685118885518205E
:10B7D000684321680818805D2C216943626851180C
:10B7E0000831895D0843182169432268511888553A
:10B7F000701CC6B2082ED9D32C2068436168081883
:10B80000806A002809D018236B432268D0182C23A3
:10B810006B436268D218916A8847681C85B2208998
:10B82000A84200DD4EE7F8BD10B50446002013F035
:10B8300071F9022841D121480078002802D1012065
:10B840001E4908701D48007801281FD11B48407808
:10B85000401C1A49487021465A20FCF771FC1749D0
:10B860004978884229D800201449487008468078D1
:10B87000401C8870084680780A2803D3002088700E
:10B8800002200870002013F075F916E00B480078CC
:10B89000022812D109484078401C084948702146C6
:10B8A0007D20C000FCF74CFC04494978884204D84C
:10B8B00000200249487013F05DF910BD78000020A7
:10B8C00000B587B0002168460171042141710C4820
:10B8D0000290411003910B49049105910A4806908A
:10B8E000FFF78EFE01A813F0A9F900F02FFB00F07E
:10B8F0000FF80021054809F0A7F907B000BD0000C6
:10B90000FFFF1F00FFFFFF1F45BB000002050000F7
:10B9100010B5FF2002306549486000200872012000
:10B92000087000204872012088726148FFF7D7FB39
:10B930005E495F48FFF7FCFB01215D48FFF74CFCC7
:10B940005C485A49486000200872012008700020B5
:10B9500048720120887256481030FFF7C0FB5349E7
:10B9600053481030FFF7E4FB012151481030FFF736
:10B9700033FC5048401E4D494860002008720120A9
:10B980000870002048720120887249485030FFF743
:10B99000A6FB464946485030FFF7CAFB0121444800
:10B9A0005030FFF719FC4348C13840494860002037
:10B9B00008720120087000204872012088723C48FB
:10B9C0004030FFF78CFB394939484030FFF7B0FB76
:10B9D000012137484030FFF7FFFBFF201230334989
:10B9E0004860002008720120087000204872012081
:10B9F00088722F486030FFF772FB2C492C4860306A
:10BA0000FFF796FB01212A486030FFF7E5FBFF2096
:10BA1000213026494860002008720120087000206B
:10BA20004872012088722248A030FFF758FB1F4956
:10BA30001F48A030FFF77CFB01211D48A030FFF715
:10BA4000CBFB3F20400119494860002008720120CB
:10BA50000870002048720120887215482030FFF7D6
:10BA60003EFB124912482030FFF762FB01211048CB
:10BA70002030FFF7B1FB10480C49486000200872E5
:10BA80000120087000204872012088720848303078
:10BA9000FFF725FB054906483030FFF749FB012138
:10BAA00003483030FFF798FB10BD0000E42500206C
:10BAB0001055044002040000DF070000F0B50B46FB
:10BAC000144643600481002136E0002216E02C2554
:10BAD0004D4346687519AD5C18274F430668F61943
:10BAE000B5542C254D4346687519AD5C18274F4356
:10BAF0000668F6190836B554551CEAB2082AE6D38A
:10BB0000002518274F430668F619357418274F4348
:10BB10000668F619757418274F430668F619B57448
:10BB200018274F430668F619F57418274F4306681F
:10BB3000F61975614D1CA9B205898D42C5DC002539
:10BB40008572F0BD70B50446606800F01FFE0546C2
:10BB5000E27A23460C332946094800F0DFFD094903
:10BB60006068884203D0491C6068884206D1E17A47
:10BB7000A28890B222460C3202F070FD70BD000027
:10BB800028080020DF070000F8B5054600262C46EF
:10BB9000002C07D000BF03E0FF20A055701CC6B2E8
:10BBA000082EF9D304F08CFCC00008210840074699
:10BBB0002068884338432060F8BDF8B50546002664
:10BBC0002C46002C07D000BF03E0FF20A055701CBE
:10BBD000C6B2082EF9D304F0EBFC07122088000A45
:10BBE00000023843208004F0E3FC0002FF21090238
:10BBF00008400746208888433843208004F0CEFD63
:10BC000007126088000A00023843608004F0C6FD15
:10BC10000002FF2109020840074660888843384334
:10BC20006080F8BDFEB5054600260020019001F0B9
:10BC30001FFD0A210090FCF783FA074604F074FC0C
:10BC40000A210090FCF792FA80B201902C46002C59
:10BC500007D000BF03E0FF20A055701CC6B2082E1D
:10BC6000F9D30721090620688843019909120906BA
:10BC7000072212061140084320606068000A000293
:10BC80000199C9B208436060FF21090260688843D6
:10BC9000390C0902FF2212021140084360601102B0
:10BCA00060688843390A0904120211400843606041
:10BCB00060680002000A3906090E09060843606040
:10BCC00004F0F2FBC007C00FC007009020684000DE
:10BCD000400800990843206003F096FE0007000F1B
:10BCE000009020680009000100990843206003F0DB
:10BCF00085FE022806D101210907206888434018E3
:10BD0000206004E00121090720688843206004F0D6
:10BD100091FB0001F02108400090206888430099C1
:10BD20000843206004F05AFCFF2806DDFF210904C7
:10BD300020688843401820600BE004F04FFC0004AA
:10BD4000FF210904084000902068884300990843B7
:10BD50002060FEBDFEB505460026002001900027AC
:10BD600004F00EFA64210090FCF700FA80B2019012
:10BD7000002001F08FFC87B22C46002C07D000BFBA
:10BD800003E0FF20A055701CC6B2082EF9D320682E
:10BD9000000A00020199C9B208432060FF2109048A
:10BDA0002068884339120904FF2212041140084315
:10BDB000206020680002000A3906090E09060843BF
:10BDC000206003F027FE28300002FF21090208400E
:10BDD000009020688843009908432060FEBDFFB5AD
:10BDE00081B004460F460025002600200090276001
:10BDF000039820810498E0600020207400BF9DE03B
:10BE00001C206843216808586A01616888501C201A
:10BE100068432168081880686A0161688918486069
:10BE20001C2068432168081840686A016168891805
:10BE300088601C20684321680818C0686A0161682E
:10BE40008918C8601C20684321680818007C6A01B2
:10BE50006168891808741C20684321680818407CB0
:10BE60006A016168891848741C20684321680818B1
:10BE7000807C6A016168891888831C206843216876
:10BE80000818C07C6A0161688918887400206A01FA
:10BE900061688918C8741C206843216808184068C4
:10BEA000002813D01C20684321680818C07C002893
:10BEB00005D1401E6A0161688918C8831AE0002014
:10BEC000C0436A0161688918C88313E01C20684375
:10BED00021680818C07C002805D000206A0161682C
:10BEE0008918C88306E000206A0161688918C88340
:10BEF00001200090002607E000216A016068801898
:10BF000014308155701CC6B2690160684018808B7E
:10BF1000B042F1DC1C206843216808184069002801
:10BF20000AD06B016268D218104614301C236B4390
:10BF30002268D21851698847681CC5B22089A84276
:10BF400000DD5DE7009805B0F0BD000000B58BB0E6
:10BF500056480790002108A801706846017608A895
:10BF60004170002052498872082108A8C170002041
:10BF700004E0002209A90A54411CC8B208A9C978E2
:10BF80008142F6DC4B48FFF7AAF806A94948FFF7BB
:10BF9000CFF84648401C0790002108A80170684669
:10BFA000017608A84170002041498872082108A83C
:10BFB000C170002004E0002209A90A54411CC8B243
:10BFC00008A9C9788142F6DC3A484030FFF787F883
:10BFD00006A938484030FFF7ABF84520000107902C
:10BFE000002108A801706846017608A84170002069
:10BFF0002F498872082108A8C170002004E000229F
:10C0000009A90A54411CC8B208A9C9788142F6DCC2
:10C0100028485030FFF763F806A926485030FFF74C
:10C0200087F8112040010790002108A80170684698
:10C03000017608A8417000201D498872082108A8CF
:10C04000C170002004E0002209A90A54411CC8B2B2
:10C0500008A9C9788142F6DC16482030FFF73FF87E
:10C0600006A914482030FFF763F8FD20C0000290B5
:10C070000021684601730171417381730821C17306
:10C08000002004E0002204A90A54411CC8B26946F9
:10C09000C97B8142F6DC07481030FFF720F801A980
:10C0A00004481030FFF744F80BB000BDEE06000066
:10C0B000E42500208055044030B585B004460025B5
:10C0C00020680190A1796846C172617941720021AE
:10C0D0000172017000BF05E020460830415D03A8F1
:10C0E00041556D1C6846C07AA842F5D81121490116
:10C0F0000198401A1BD023210901401A11D011497F
:10C100004018002802D0012817D104E069460E48E3
:10C11000FFF7DFF812E069460B484030FFF7D9F827
:10C120000CE0694608485030FFF7D3F806E069464E
:10C1300005482030FFF7CDF800E000BF00BF05B094
:10C1400030BD000062FDFFFF80550440F0B585B0B2
:10C1500004460F4600250026207C4006400E552848
:10C160007ED100BF76E1690160684018807C0028BC
:10C1700077D169016068401840686A016168891870
:10C180008968884209D26901606840184068C0190E
:10C190006A016168891848605AE16901606840185D
:10C1A000C068AF49884208D8690160684018C06813
:10C1B000401C6A0161688918C8606901606840189C
:10C1C000C07C002821D1002607E000216A016068B8
:10C1D000801814308155701CC6B26901606840181F
:10C1E000808BB042F1DC1C2068432168081840694C
:10C1F00000280AD06B016268D218104614301C2344
:10C200006B432268D21851698847690160684058B9
:10C210000090690160684018017C68460171002146
:10C220004171690160684018017F68468171690148
:10C2300060684018417C6846C171002608E06901C9
:10C24000606840181430815D02A88155701CC6B228
:10C25000690160684018808BB042F0DCE06801E062
:10C26000FCE01DE0002806D06846E16888476A01C6
:10C2700061688918C874690160684018C07C00282A
:10C2800004D16A01616889184860E1E06901606869
:10C2900040184068C01B6A01616889184860D7E08F
:10C2A00069016068401880680028EED06901606804
:10C2B0004018C08B0028E8D0690160684018C08B26
:10C2C0006A0161688918C968884207D16901606894
:10C2D0004018C08B6249C94388427DD169016068BA
:10C2E000401840686A01616889188968884209D2E3
:10C2F0006901606840184068C0196A01616889185E
:10C300004860A5E000206A016168891848606901F9
:10C3100060684018C0685249884208D8690160685E
:10C320004018C068401C6A0161688918C86000260E
:10C3300007E000216A016068801814308155701C84
:10C34000C6B2690160684018808BB042F1DC1C20E5
:10C35000684321680818406900280AD06B016268A8
:10C36000D218104614301C236B432268D21851692E
:10C37000884769016068405800906901606840180A
:10C38000017C6846017100214171690160684018B3
:10C39000017F68468171690160684018417C684688
:10C3A000C171002608E06901606840181430815DA1
:10C3B00002A88155701CC6B2690160684018808B64
:10C3C000B042F0DCE068002808D06846E1688847A1
:10C3D0006A016168891800E015E0C8746901606845
:10C3E0004018C07C002804D16A016168891848603F
:10C3F0002EE06901606840184068C01B6A016168EE
:10C400008918486024E01C206843216808184068A7
:10C4100000280FD00020C0436A0161688918C883D2
:10C420001C2068432168081840686A0161688918FF
:10C43000886008E000206A0161688918C8836A0181
:10C4400061688918886000206A0161688918C8607D
:10C45000681CC5B22089A84200DD84E605B0F0BDA5
:10C460000000FFFF7CB500BF19212C480078FBF7C6
:10C4700067FE04462A4860432A4A811800220120A8
:10C480000BF0A2FD20460A2250436430001981B20D
:10C49000002201200DF064FB01200A2262431219E0
:10C4A000D1B20A22624312190090D0B201231A4677
:10C4B00008F0D2FEBA220721002006F0F7FB012087
:10C4C000009001900B20604382B20B20604381B248
:10C4D000002301200CF07CFE6F20604381B201201C
:10C4E0000DF0E4FD104860430246032101200AF0EC
:10C4F0006DFC002505E0012128460AF0A1FB681C1F
:10C50000C5B20F2DF7DB21460B2251436431C8B26F
:10C510000EF030F80EF018F87CBD0000730000201B
:10C52000672B0000A0860100FCB101000020054936
:10C5300008700549087005490870054908700549E3
:10C540000870704774000020750000207300002000
:10C550007200002071000020F0B589B000BF00BF5C
:10C5600000BF00BF00BF00BF00BF00BF00BF00BFD3
:10C5700003215C480078FBF7F9FD5B4948430290D2
:10C5800003210120029A0AF021FC05215548007878
:10C59000FBF7D6FD0446E1B201200AF0DFF90321E2
:10C5A00050480078FBF7E2FD0B214843643080B22D
:10C5B0000690E1B201231846069A09F027F9494985
:10C5C00009788A0088180621FBF7D0FDFF21F53194
:10C5D000484380B207900798FBF7C8FDC7B23946B9
:10C5E000012009F0F7FD03213E480078FBF7BEFD6E
:10C5F0000B214843643080B2089000220120089942
:10C600000DF0AEFA032137480078FBF7AFFD37494C
:10C6100048433749401803900022012003990BF04A
:10C62000D3FC03212F480078FBF7A0FD0B214843E2
:10C6300080B2049003212B480078FBF797FD0B2173
:10C64000484386B20120F1B20090049AD0B201238F
:10C650001A4608F001FEBA220721002006F026FB48
:10C66000032120480078FBF781FD0B21484385B268
:10C670000120009000232A46294601900CF0A8FDD5
:10C68000032118480078FBF771FD6F21484380B201
:10C690000590012005990DF009FD164800783C2809
:10C6A00005DA14480078401C1249087002E03C206A
:10C6B000104908700F4800781D2805DC09480078EB
:10C6C000401C084908700BE006480078002802D199
:10C6D0000449087004E003480078401E01490870CE
:10C6E00009B0F0BD74000020FCB10100672B000010
:10C6F000A086010075000020002000BF06E0002198
:10C70000044A1154044A1154411CC8B25A28F6DB99
:10C7100070470000EC210020A0220020FFB581B06E
:10C7200004460F463D462089A8422DDD1820684367
:10C7300021680818007C002826D1002609E004980A
:10C74000815D182068432268101808308155701CDC
:10C75000C6B2082EF3D301211820684322681018AE
:10C7600041742C20684361680818006A00280BD0C7
:10C7700018236B432268D218104608302C236B43D1
:10C780006268D218116A884705B0F0BD01460620DC
:10C79000104BCA1A99420FD008DCCA1FFA3A002A75
:10C7A00012D0102A0AD01F2A10D10BE0C02A07D0BD
:10C7B000C12A0BD100200BE0012009E0022007E094
:10C7C000032005E0042003E0052001E0062000BF6F
:10C7D00000BF70474103000010B504467D21C90029
:10C7E00061430846322103F06DFC10BD014800682A
:10C7F00070470000500000200148006870470000AA
:10C800004C00002010B505490988652251430846AF
:10C810006421FBF7ABFC80B210BD00005A00002081
:10C8200001480078704700005F0000200148007850
:10C83000704700005800002010B50EF0D5FB01280D
:10C840002CD100F063F8012000F066F803F09EFCA4
:10C85000044600F043F803F045FE044600F04AF8B1
:10C8600003F0CEFF012805D100F03EF8012000F0D2
:10C8700047F805E0002000F037F8002000F040F80D
:10C8800000201349086013480068134988421ED2EB
:10C8900010480068801C0F49086018E000200D490E
:10C8A00008600B4800680C49884204D208480068B8
:10C8B000801C07490860002000F028F8012000F0E3
:10C8C0002BF8002000F00AF8002000F013F810BD4B
:10C8D000500000204C000020FFFFFF7F014908802E
:10C8E000704700005A00002001490870704700009E
:10C8F0005F00002001490880704700005C000020B4
:10C90000014908707047000060000020014908706C
:10C91000704700005800002001490870704700006F
:10C920005E0000200021014A117170470060004044
:10C93000002201494A757047006000400022014909
:10C940004A767047006000400021014A117270472A
:10C95000006000400021014A1173704700600040F0
:10C960000021014A11747047006000400021014A13
:10C9700011757047006000400021014A1176704730
:10C9800000600040002201494A7370470060004087
:10C99000002201494A7470470060004010B51C4CE9
:10C9A0001C49206888421ED106221B49201DFBF726
:10C9B00082FC002817D10D22184920460A30FBF7C7
:10C9C0007AFC00280FD10622154920461730FBF7C4
:10C9D00072FC002807D10622124920461D30FBF7C1
:10C9E0006AFC00280DD000F079FE0A480E49086064
:10C9F000074812F0F0F90C4A2421054812F016FA03
:10CA000004E0242221460848FBF731FC10BD000059
:10CA1000000250007AA7A55A3107002037070020EE
:10CA20002B07002025070020B82A002000200849F5
:10CA3000087008490870012007490870002007495C
:10CA400008700748074908600020074908707047C8
:10CA50001307002012070020150700201A070020E6
:10CA600025060000440700202407002070B5054675
:10CA700000BF9120684304460A212046FBF760FB73
:10CA80000446641D204670BD70B5A8B0054600245C
:10CA90000026A0216846FBF703FC00F09FFC1E491E
:10CAA0000A6814216943505000211B480268142071
:10CAB0006843101841601848026814206843101831
:10CAC000816015484068002824D000BF17E0600648
:10CAD000060E282E00D316E00F480168142060438C
:10CAE0000858B1006A4650500B4801681420604352
:10CAF00008184168701C80001150601CC4B20648C0
:10CB0000007AA042E3DC00BF620003486946436844
:10CB10000220984728B070BD082B002030B5A9B07E
:10CB200000240025A02101A8FBF7BAFB00BF25E0E7
:10CB30006006050E00F052FC1F490A68142161438B
:10CB4000505000211C4802681420604310184160B6
:10CB5000194802681420604310188160282D0BD2F8
:10CB600015480168142060430858A90001AA5050D4
:10CB70000021681C80001150601CC4B20E48007A6D
:10CB8000A042D5DC0C484068002813D00A48007A3F
:10CB90004000282806D30848282201A9436802201B
:10CBA000984707E00448007A4200034801A9436817
:10CBB0000220984729B030BD082B002010B50EF098
:10CBC00013FA01287ED1FFF717FE5549884216D285
:10CBD0000F2054494871887108468078002801D197
:10CBE000052048704F488078052802D100204D4923
:10CBF000487000204B4908724872087035E0FA20EE
:10CC00004849487188714849088803F095FB4648AF
:10CC1000807800280CD14349087008464079C870D4
:10CC200008468079087100208870487048721CE0BE
:10CC300001203C4908700846407A022805D10120AD
:10CC400048720020C87008710FE03648407A00280A
:10CC50000BD1022033494872084640788870084654
:10CC60004079C8700846807908712E4880782D492F
:10CC70004978884213DD00202A49C87008460079A7
:10CC8000401C0871084600798979884222DB00201F
:10CC90002449087108468078401E88701AE02148AF
:10CCA000807820494978884214DA00201D490871AB
:10CCB0000846C078401CC8700846C0784979884248
:10CCC00008DB00E01EE000201649C87008468078A6
:10CCD000401C887014488078002803D10120114935
:10CCE00008721BE010480088732803DB02200D49FE
:10CCF000087213E00C48008870280FDC00200949F6
:10CD000008720BE000200749087008464079C87097
:10CD100008468079087100200872487210BD000032
:10CD2000B80B0000580900207C00002000200449B6
:10CD300088704870C87008710872487270470000A7
:10CD4000580900200020064908808870054988702D
:10CD50004870FA20C8700871002008724872704745
:10CD60007C0000205809002070B503F03FFA04460B
:10CD700003F04EFA05460EF037F901282ED10521B1
:10CD80001A48FEF79FF9552804D1002018498870E9
:10CD9000088027E0012D04D1002015498870088003
:10CDA00020E00120124988701248844202DB201AD8
:10CDB00084B200E000240A212046FBF7D7F90529B8
:10CDC00001DB601D84B20C48844200DD04460A2168
:10CDD0002046FBF7CBF90649088003E00020044910
:10CDE00088700880FFF7EAFE70BD00002808002068
:10CDF0007C000020AA0A0000C60700001CB5002025
:10CE00000090019000F0EAFA0B49086000200B49FD
:10CE1000096808600A48006800280CD007490968BA
:10CE200008680A21FBF78CF9009001226946052069
:10CE3000034B1B6898471CBDE0070020D407002067
:10CE4000DC0700200020084948800849088008497C
:10CE50000880084908700849887208490880488095
:10CE600001200871704700003400002024000020D9
:10CE700026000020280000200C0800202C000020A4
:10CE8000F8B503F095F9074603F0A4F90090FFF711
:10CE9000CDFC012860D10521C548FEF713F95528BE
:10CEA00002D00098012807D10020C2490870C24969
:10CEB0000880C249887256E0BE480078002810D128
:10CEC0000120BC4908703D462846E917890F09181A
:10CED00089030D0CBA48854200DD0546B648058039
:10CEE00041E0B648807A4000B4490F520846867A3D
:10CEF0000EE07000B1490D5A701E4000085A7100D2
:10CF0000AE4A5052701E400011460D52701EC6B2FD
:10CF1000002E08DD7000A949095A701E4000A74A7A
:10CF2000105A8142E5DBA548807A401CA3498872EB
:10CF30000846807A052816DB002088720846C588D6
:10CF40002846E917890F09188D109D48854200DD94
:10CF500005469948058006E00020964908709649E4
:10CF60000880964988729448058896480088A842A7
:10CF700057DA94480088281A84B292480079012828
:10CF800027D190484088A0420BDA8E4840880A306A
:10CF90008C49488008464088A04204DD0846448009
:10CFA00001E088484480874844882046E117890F7B
:10CFB00009188C100A2C00DA0A248248008800190B
:10CFC0008049088008460088A84201DD084605809F
:10CFD000CDE07C484088142805DD7A484088143824
:10CFE0007849488002E000207649488075484488A6
:10CFF0002046E117890F09188C100A2C03DA01204A
:10D0000070490871B3E06F480088A04205DD6D48A3
:10D010000088001B6B490880A9E00020694908804E
:10D02000A5E068480088A84259DD66480088401B92
:10D0300084B264480079012827D1624840881428C6
:10D0400005DD6048408814385E49488002E00020D1
:10D050005C4948805B4844882046E117890F0918DD
:10D060008C100A2C03DA0220564908717FE05548DB
:10D0700000880019534908800846008850498842B2
:10D0800075DD08464F49088071E04E484088A0424F
:10D090000BDA4C4840880A304A49488008464088A4
:10D0A000A04204DD0846448001E0464844804548EB
:10D0B00044882046E117890F09188C100A2C00DAE1
:10D0C0000A24404800882919884202DA3D48058030
:10D0D0004DE03C480088001B3A49088047E0394849
:10D0E00044882046E117890F09188C100A2C3EDD70
:10D0F00034484088142805DD3248408814383149C6
:10D10000488002E000202F4948802E48448820466D
:10D11000E117890F09188C102A480079012813D1CA
:10D120000A2C03DA02202749087120E025480088EC
:10D13000001924490880084600882149884216DDE4
:10D1400008462049088012E00A2C03DA01201D4914
:10D1500008710CE01B480088A04205DD19480088D2
:10D16000001B1849088002E0002016490880164874
:10D170000088502804DC134800881349088016E012
:10D180001048008810490988884204DD0D4800884D
:10D190000D4908800BE00B4800880B490988081AE4
:10D1A00084B2502C03DB0748008807490880F8BD8B
:10D1B0002808002028000020240000200C0800205F
:10D1C000E02E00002C0000202600002010B50446B0
:10D1D00064204443A1212046FAF7B2FF04462046CA
:10D1E00010BD00007CB5002400200190009000F0EC
:10D1F0003FFA05460A21FAF7A3FF044601226946D1
:10D20000042000F06DFC0098401C002814D17D2003
:10D21000C0002018114908600846006801900122EA
:10D2200001A9032000F09AFC012000900122694628
:10D23000042000F093FC0FE0009801280CD17D2021
:10D240000001201805490860084600680190012285
:10D2500001A9032000F082FC7CBD00002801002011
:10D2600010B501200F49087000200F4909680860B7
:10D270000D49096848600C490968886000F07EF92A
:10D28000FFF7BCFDFFF74AFC08480068002807D0FC
:10D2900001220548016808310020044B1B689847AB
:10D2A00010BD0000AD070020A8070020A407002043
:10D2B00010B5184800681849884229D117480068F5
:10D2C000002804D0154800688047154908701548A3
:10D2D0000068002804D0134800688047124908708D
:10D2E00012480068002804D01048006880471049A0
:10D2F000088010480068002805D00E480068804764
:10D300000D49088002E00D480B49088000F078F8CC
:10D3100010BD0000B8070020785634129407002092
:10D32000AC07002098070020AE0700209C070020D3
:10D33000B0070020A0070020B2070020102700003F
:10D3400010B50023174C2360174C2370174C237023
:10D35000174C2370174C2380174C2380174C2370D5
:10D36000174C13682360174C53682360164C93685E
:10D370002360164CD3682360154C13692360002882
:10D380000CD0144B1860134C0B682468A360002366
:10D39000104C246823600F4C246863600E4B014CD2
:10D3A000236010BDB8070020B4070020AC070020A0
:10D3B000AE070020B0070020B2070020AD07002014
:10D3C00094070020980700209C070020A007002059
:10D3D000A4070020A80700207856341205480068EA
:10D3E0000549884203D105480068806870470020DD
:10D3F000C043FBE7B807002078563412A807002086
:10D4000070B50024002500263048007801285CD142
:10D410002F480078002858D12E480078012854D190
:10D420002D4805882D490988694308462C49FAF793
:10D4300087FE85B2E1200001854207D819216943A2
:10D4400008460921FAF77CFE044600E0244C2548F2
:10D4500000680068001923490968086021480068CD
:10D460000068204909684968884207D31D48006858
:10D4700000681C4909684968461A0AE019480068AA
:10D4800040680021C943081A16490968096840180C
:10D49000461C1548864218D3344601462046FAF702
:10D4A0004FFE04460F48006841680F486043081863
:10D4B0000C490968486001200C4908700948006857
:10D4C0008068001907490968886070BDAC070020B2
:10D4D000AD070020AE070020B0070020B2070020F3
:10D4E00010270000A8070020A0860100B407002034
:10D4F00000220C4B1A600C4B0A681A600B4B4A68EE
:10D500001A600B4B8A681A600A4BCA681A600A4B89
:10D510000A691A60002801D0084A1060084A014BC5
:10D520001A607047B8070020940700209807002071
:10D530009C070020A0070020A4070020A8070020C7
:10D540007856341210B50A48006800280ED00948F1
:10D55000007801280AD100200649087001220648F7
:10D56000016808310020024B1B68984710BD00007D
:10D57000A4070020B4070020A80700201CB5002045
:10D58000009001900024FFF729FF04460E48006830
:10D59000046000200C49096848600B4909688860EC
:10D5A0000A48006800280DD007480068006800900D
:10D5B0000548006840680190022269460120034B3B
:10D5C0001B6898471CBD0000BC070020C007002056
:10D5D000F8B505460C4616460027002D17D00E4814
:10D5E0000560FFF7FBFE07462068B84203D90A48EA
:10D5F0000068076003E00849206809680860064978
:10D600006068096848600449A0680968C860034800
:10D61000066000F005F8F8BDBC070020C007002038
:10D6200070B500240025FFF7D9FE04460F480068B6
:10D630000068A04200D903E00C4800680068251A81
:10D640000A48006840684019084909688860074826
:10D650000068806805490968C968884205D9034897
:10D660000068C06801490968886070BDBC07002077
:10D670000148006880687047BC070020002801D07E
:10D68000024A1060024A116070470000BC07002087
:10D69000C0070020014610480268142048431018B3
:10D6A00082680D480368142048431818C0688242F5
:10D6B0000BD909480268142048431018C26806486C
:10D6C0000368142048431818826003480268142035
:10D6D0004843101880687047082B0020002005E0A0
:10D6E00019490A5C19490A54411CC8B20628F7DBDB
:10D6F000002006E016490A5C1449891D0A54411CA1
:10D70000C8B20D28F6DB002006E012490A5C0F497A
:10D7100013310A54411CC8B20628F6DB002006E08B
:10D720000D490A5C094919310A54411CC8B206283E
:10D73000F6DB002005E0002204491F310A54411C99
:10D74000C8B20128F7DB704731070020BC2A00204F
:10D75000370700202B0700202507002010B50020E8
:10D7600005490860486008724872887202F0AEFE8F
:10D770000149C87210BD00006409002070B5002482
:10D78000002502F0A3FE6549C87202F085FD04463B
:10D7900002F08CFD0546FFF749F8012874D10121FC
:10D7A0005F48FDF78FFC552807D100205B490872C0
:10D7B0004872086048608872AFE0FF2C01D0FF2DEE
:10D7C00063D1FF2C2AD1FF2D28D0002053490872A5
:10D7D0000120487253480860FF20143068434860B5
:10D7E00048686621FAF7ACFC4C4948600846406836
:10D7F0004C49884202D90846484948604748406831
:10D80000AA2803D345484068FA2803D90120434990
:10D81000887282E00020414988727EE0FF2C2AD085
:10D82000FF2D28D101203D490872002048723D4853
:10D830004860FF2014306043086008686621FAF7EA
:10D840007FFC36490860084600683649884202D99C
:10D8500008463249086031480068AA2803D32F4897
:10D860000068E62803D901202C49887255E0002081
:10D870002A49887251E02B482849086048600020F6
:10D8800088720872487248E040E00120234908721B
:10D890004872FF2014306043086008686621FAF778
:10D8A0004FFC1E490860084600681E49884202D99C
:10D8B00008461A490860FF20143068431749486039
:10D8C00048686621FAF73CFC1449486008464068FD
:10D8D0001449884202D90846104948600F48006838
:10D8E000AA280BD30D480068E62807D80B484068E3
:10D8F000AA2803D309484068FA2803D90120074918
:10D9000088720AE000200549887206E00020034979
:10D910000872487208604860887270BD640900200F
:10D9200028080020DE030000FFB583B006460D4640
:10D93000174600240020029000BF1420784380196D
:10D940000190002E57D00198002854D02B48066033
:10D950002A49069848600846077200BF45E0FFF76D
:10D960003DFD0290200129580298814204D82001EF
:10D970002858401C002806D1204902980A68142122
:10D980006143505006E0200129581C4802681420C9
:10D9900060431150200140194068401C002807D105
:10D9A000002116480268142060431018416008E006
:10D9B0002001401941681148026814206043101882
:10D9C00041602001401981680C48026814206043BE
:10D9D0001018C16020014019017B0848026814201A
:10D9E000604310180161601CC4B20448007AA04270
:10D9F000B5DC00F005F807B0F0BD0000082B0020F2
:10DA000070B5002400250026FFF7E8FC054600BF9E
:10DA10004EE02A480168142060430858A84239D8CB
:10DA2000264801681420604308582E1A23480168CC
:10DA300014206043081840688119204802681420A7
:10DA40006043101881601D48016814206043081865
:10DA500081681A480268142060431018C068814227
:10DA600024D916480168142060430818006900286A
:10DA700003D02046FFF708F818E01048016814208A
:10DA800060430818C1680D480268142060431018EC
:10DA900081600BE009480168142060430818406861
:10DAA00006490A681421614351188860601CC4B299
:10DAB0000248007AA042ACDC70BD0000082B0020B8
:10DAC00010B500BF14244C432318002805D0002BA8
:10DAD00003D0024C20606260217210BD082B002030
:10DAE000F8B505460E4614462B0010F0AFFC0504B1
:10DAF000121920272E001748FBF730F81649087036
:10DB00001448FAF7E5FB07466421FAF719FB306081
:10DB10001CE0A004020C31461020FBF719F915E0B7
:10DB2000A004020C31463020FBF712F90EE0A004ED
:10DB3000020C31465020FBF70BF907E0A004020C61
:10DB400031467020FBF704F900E000BF00BF002061
:10DB5000F8BD0000CE230020D900002070B5054696
:10DB60000E4614462B0010F071FC05041C232A31CC
:10DB700038003068002802D1FAF78EFE10E06422E7
:10DB80003168514308461649FAF7ACFB00201549A5
:10DB90000870012264211248FBF748F91149087006
:10DBA0001CE0A004020C31461020FBF78FFA15E0B0
:10DBB000A004020C31463020FBF788FA0EE0A004E6
:10DBC000020C31465020FBF781FA07E0A004020C5A
:10DBD00031467020FBF77AFA00E000BF00BF70BD4D
:10DBE000C0230020D800002000B5AFB050211BA8F2
:10DBF000FAF756FB00201A90142115A8FAF750FBEB
:10DC000000201290139014901190402101A8FAF76F
:10DC100047FB00203F49086001221BA9FFF760FF76
:10DC20001B98401C002801D11A9001E01B981A9003
:10DC300039481590394816903948179000201890A7
:10DC40003848199015AA1AA93748FFF779FB02221C
:10DC50001CA90120FFF744FF1C98401C002801D19B
:10DC6000129001E01C9812901C98401C002801D1D1
:10DC7000139001E01D9813902C48149012A92C4881
:10DC8000199AFFF7A5FC08221EA90220FFF728FF1A
:10DC90001E98401C002801D1019001E01E980190BF
:10DCA0001F98029023480390012069460874801E43
:10DCB000059021490791012101A80177881E09904B
:10DCC0001D490B91012109A80173881E0D901A4965
:10DCD0000F9101210DA80173042201A91748199B76
:10DCE000FFF722FE01221BA90320FFF7F9FE1449CA
:10DCF0001B9808601B98401C002806D1FF20F530B7
:10DD0000086001220320FFF729FF0E48014908603F
:10DD10002FB000BDDC0000202DC8000021C800008D
:10DD200005C800005DDB00005423002076841E003F
:10DD3000602300200F2700009F8601007023002031
:10DD400028010020A33AA55A00B585B014216846E1
:10DD5000FAF7A6FA00200F4908600F4800900F4814
:10DD600001900F480290002003900E4804906946ED
:10DD70000D48FFF7BDFB0D480499FFF77FFC042118
:10DD80000B48049AFFF79CFE0A480249086005B058
:10DD900000BD0000DC0000202DC8000021C80000EC
:10DDA00005C800005DDB0000542300206023002034
:10DDB00070230020A33AA55A00200B4908800B4984
:10DDC00008800B49088001200A49087000200A4990
:10DDD00008730A490880488001200871002006491C
:10DDE00048800880704700003C0000203E00002072
:10DDF00040000020420000201808002044000020BD
:10DE0000FEB502F00FFA009002F016FA0190FEF74C
:10DE10000DFD01286BD10521D448FDF753F9552894
:10DE200007D10020D2490870D2490880D2498880A1
:10DE300067E00198012807D10020CD490870CD493D
:10DE40000880CD4988805CE0C9480078002808D166
:10DE50000120C7490870009D0A206843C549088011
:10DE60004FE0009881B2C448007B4200C248801D48
:10DE70008152801F067B11E07100BF48801D455A0A
:10DE8000701E4100BC48801D415A72008152701EB4
:10DE90004100B948801D4552701EC6B2002E0ADDF1
:10DEA0007100B548801D415A701E4200B248801D65
:10DEB000805A8142E0DBB048007B401CAE490873C9
:10DEC0000846007B032807DB002008730846058905
:10DED0000A206843A74908800020A7490880488095
:10DEE000A448008888800120A149087009E000202A
:10DEF0009F4908709F4908809F490880488008739F
:10DF000088809C4805889D480088A84256D29B4836
:10DF10000088281A84B299480079012826D19748A8
:10DF20004088A0420BDA95484088801C934948807D
:10DF300008464088A04204DD0846448001E08F483E
:10DF400044808E48448803212046FAF70FF984B2B2
:10DF5000022C00DA022489480088001987490880C9
:10DF600008460088A84200D90D80CDE0834840884B
:10DF7000062805DD81484088801F8049488002E0EE
:10DF800000207E4948807D48448803212046FAF7D6
:10DF9000EDF884B2022C03DA012078490871B3E06D
:10DFA00076480088A04205DD74480088001B73494C
:10DFB0000880A9E0002071490880A5E06F4800882A
:10DFC000A84259D96D480088401B84B26B4800793B
:10DFD000012827D169484088062805DD6748408820
:10DFE000801F6649488002E00020644948806348F9
:10DFF000448803212046FAF7B9F884B2022C03DAE8
:10E0000002205E4908717FE05C48008800195B4986
:10E010000880084600885A49884275DD08465749F5
:10E02000088071E055484088A0420BDA5348408888
:10E03000801C5249488008464088A04204DD0846BA
:10E04000448001E04D4844804C48448803212046E8
:10E05000FAF78CF884B2022C00DA022447480088D0
:10E060002919884202D245490D804DE04348008875
:10E07000001B4249088047E040484488032120466D
:10E08000FAF774F884B2022C3EDD3C48408806283A
:10E0900005DD3A484088801F3849488002E000206A
:10E0A000364948803548448803212046FAF75EF80F
:10E0B00084B232480079012813D1022C03DA0220FD
:10E0C0002E49087120E02D48008800192B4908804E
:10E0D000084600882A49884216DD084627490880F4
:10E0E00012E0022C03DA0120244908710CE02348D5
:10E0F0000088A04205DD21480088001B1F490880D8
:10E1000002E000201D4908801C4800881D4909883C
:10E11000884203DA194800880F2804DA1748008873
:10E12000184908800AE01548008816490988081A25
:10E130000F2803DB1148008812490880114807881E
:10E140000B48007800280DD06C20474364213846E6
:10E15000F9F7F6FF07460A48874200D907460A49F9
:10E160000F8002E0002008490880FEBD280800203A
:10E17000420000203C00002018080020440000203D
:10E18000C6070000400000203E0000200020074994
:10E1900008800749088007490880488001200871E5
:10E1A0000020054948800880704700003E0000209C
:10E1B00040000020440000201808002000200249F0
:10E1C000087002490870704788000020890000200C
:10E1D00010B5FEF72BFB012813D103210C48FCF7E7
:10E1E00071FF552805D100200A4908700A490870B6
:10E1F0000CE002F065F80749087001200649087034
:10E2000004E00020034908700349087010BD0000B5
:10E21000280800208800002089000020F0B5A9B05F
:10E2200004460E460025002700202890A0216846BD
:10E23000FAF736F8FFF7D2F826490A681421614345
:10E24000505024480168142060430818C068B04248
:10E250000CD220480168142060430818C1681D488A
:10E260000268142060431018416005E019480168F5
:10E27000142060430818466016484068002826D0DD
:10E28000002517E06806070E282F00D316E0114876
:10E290000168142068430858B9006A4650500D4878
:10E2A00001681420684308184168781C80001150E8
:10E2B000681CC5B20748007AA842E3DC00BF6A00C8
:10E2C000044869464368022098470120289028980E
:10E2D00029B0F0BD082B002010B500F0EDFD00F0D6
:10E2E000D7F80FF0C1F800F00DFB00F001F810BDF9
:10E2F00070B541480078912800D070BD00F0BEF89C
:10E30000012876D13D4800883D490880084680783C
:10E31000F021884320303A49887008468078000907
:10E3200000013549097A0907090F08433449887003
:10E330003148807A401E3049887208460089401C66
:10E34000088108460089C988884216DA08202C49C5
:10E35000887200240EE0284841882848001D415C4E
:10E360002748C01C015524484088401C2249488049
:10E37000601CC4B2072CEEDB2DE01F4800891E494B
:10E38000C98888421CD11C4800791B498978401AE9
:10E39000C5B2681C1A49887200240EE016484188EC
:10E3A0001648001D415C1648C01C015512484088A3
:10E3B000401C11494880601CC4B2AC42EEDB0AE04C
:10E3C00000F006FD00200C4908700C49088809215E
:10E3D00000F0B8F991E7012000F0BCFC084A917AFE
:10E3E0001088921C00F070F905490888002100F09F
:10E3F000C1F800BF81E700006C2800200828002039
:10E40000982700201B49097E002932D01949897EAE
:10E410000C225143174A515A174A118000200CE030
:10E420001449897E0C225143124A8918891C0A5CBE
:10E430001149891C0A54411CC8B20828F0DB0D4957
:10E44000897E0C2251430B4A8918897A0A4A9172B3
:10E450000121D1720749097E491E064A11761146EB
:10E46000897E491C91761146897E022901DB0021B3
:10E4700091767047642700208C2700200349487B51
:10E48000012802D10021014A517370477C280020E5
:10E4900010B533484068002861D13148007B030043
:10E4A0000FF0D4FF07590512212E3D4A59002D487F
:10E4B0000078002807D000202A4908702A490888D7
:10E4C000012100F03FF947E026480078002809D0F4
:10E4D00000202449087025494A8808880123091D1D
:10E4E00000F040F938E01F480078002807D00020ED
:10E4F0001C4908701C490888022100F023F92BE010
:10E5000018480078002809D00020164908701749DB
:10E510004A8808880923091D00F024F91CE01148E5
:10E520000078002807D000200E4908700E4908889E
:10E53000092100F007F90FE00A480078002809D007
:10E5400000200849087009494A8808880323091DE2
:10E5500000F008F900E000BF00BF00F039FC10BD7A
:10E560007C2800206C28002008280020A4270020F8
:10E570007047000070B504460D4634480088A0423C
:10E5800063D1002D61D13248007822284ED004DCBE
:10E5900020283DD0212856D141E0902802D0912852
:10E5A00051D115E02A48C08801280AD10020284905
:10E5B000087000F00DFC27490888002100F0C2F81F
:10E5C00005E0032000F0C6FBA020214908703BE0D5
:10E5D0001F4800891E49C98888420AD100201C4969
:10E5E000087000F0F5FB1B490888002100F0AAF82C
:10E5F0000DE01748807A002806D000F0E9FB1449A6
:10E60000087B00F089FB02E0032000F0A3FB1BE085
:10E61000062000F09FFB11200D49087014E0062031
:10E6200000F098FB11200A4908700DE0002008490D
:10E63000087000F0CDFB08494A8808880923091DA5
:10E6400000F090F800E000BF00BF70BD8027002000
:10E650006C28002008280020A427002070B503465D
:10E66000184C247E022C00DB70BD164C647E0C25F9
:10E670006C43144D2B5300200AE0155C114C647E52
:10E680000C2674430F4EA419A41C2554441CE0B25C
:10E690008842F2D30B4C647E0C267443094EA419B5
:10E6A000A1723446247E641C35462C762C46647E4A
:10E6B000641C6C762C46647E022C01DB00246C7694
:10E6C00000BFD1E764270020F0B585B007460D46AE
:10E6D00016461A480780002406E031781748801C47
:10E6E0000155761C601CC4B2AC42F6DB2C4605E03A
:10E6F000AA211248801C0155601CC4B2082CF7DB0B
:10E700000E480088019008216846C17200214172BC
:10E7100001720170002406E00848801C015D03A816
:10E720000155601CC4B2082CF6DB69460448FCF7AE
:10E73000D0FD01200149887205B0F0BD802700207E
:10E740009055044070B504460D46294620460EF00B
:10E75000B7FD70BD70B504460D46294620460EF043
:10E76000BDFD70BDF8B504460D4616461F463B4636
:10E770003246294620460EF0B2FDF8BDF8B50746F0
:10E780000E4615465C480078002804D0092138461A
:10E79000FFF7D8FFF8BD002D01D0602D04DD092161
:10E7A0003846FFF7CFFFF5E754480780458000243F
:10E7B00006E031785148001D0155761C601CC4B23A
:10E7C000AC42F6DB00204C49487008468580FF20AB
:10E7D00088727F2008730846808808282EDA012076
:10E7E000C880084680884880012008814348008806
:10E7F0004349088008468078F02188434049887062
:10E8000008468078000900013B4909790907090F8A
:10E8100008433B49887038480079401C88720024BE
:10E8200007E03648001D015D3548C01C0155601CDD
:10E83000C4B231488088A042F3DC4AE00721681C5A
:10E84000F9F794FC002907D0072128460830F9F78A
:10E850008DFC2949C88005E00721681CF9F786FC72
:10E860002549C88006202449488001200881234882
:10E8700000882349088008468078F02188431030BA
:10E880001F49887008468078000900011A49898864
:10E890000905090F08431A49887008464088FF2176
:10E8A00009028843144989880902FF221202114093
:10E8B00008431349488008208872002407E00F4865
:10E8C000001D015D0E48001D0155601CC4B2062CE0
:10E8D000F5DB012000F03EFA094A917A1088921C7B
:10E8E000FFF7F2FE902004490870054908880021CE
:10E8F000FFF740FE00BF4DE76C28002008280020ED
:10E900009827002010B5FFF77DFD1448C07A002835
:10E9100022D0124880780009002806D0012807D0AC
:10E9200002280AD0032810D10CE000F09DF90FE076
:10E9300000F09EF800F05AFA0AE000F011F800F03A
:10E9400055FA05E000F000F902E0FFF711FE00BF04
:10E9500000BF00200149C87210BD00008C270020B4
:10E9600010B540480078112800D010BD3E480088FE
:10E970003F214901884200D0F7E73B4880780007F3
:10E98000000F3849097A0907090F88420CD0002086
:10E990003449087000F01CFA34494A880888042376
:10E9A000091DFFF7DFFEE0E72E480089401C2D49D6
:10E9B00008810846807A401E887208460089C98806
:10E9C00088421BDA2848807A082800D0CDE7002446
:10E9D0000EE02548C01C015D224842882348001DE6
:10E9E000815420484088401C1E494880601CC4B2A5
:10E9F000072CEEDB062000F0ADF930E019488088E6
:10EA000018494988401A1849897A884203DA164811
:10EA1000807A082800D0A8E700240EE01248C01C25
:10EA2000015D104842881148001D8154601CC4B229
:10EA30000C484088401C0B4948800A4840880949D6
:10EA400089888842EADB00200649087000F0C0F996
:10EA500006494A8808880023091DFFF783FE00BF86
:10EA600083E700006C2800208C270020A4270020CA
:10EA700070B53248007880210840802800D170BDF0
:10EA80002F4800883F214901884200D0F7E72C48F1
:10EA9000807A082800D0F2E72948807805072D0FF2
:10EAA0002D0227484088000A0543082D00DAE6E7D2
:10EAB00000202249487006204880084685800120B1
:10EAC0000881082088720020C8728988481C0721A4
:10EAD000F9F74CFB002909D0184989880846083005
:10EAE0000721F9F743FB1549C88007E013498988D6
:10EAF000481C0721F9F73AFB1049C88010480088E4
:10EB00001049088008464580002407E00C48001D95
:10EB1000015D0C48001D0155601CC4B2062CF5DBDC
:10EB2000042000F017F9102004490870054A5188A4
:10EB30001088FFF70FFE00BFA1E700006C2800203F
:10EB40008C270020A427002010B544480078A02876
:10EB500008D042480078912804D040480078A12885
:10EB600000D010BD3E4800883F21490188420AD0AC
:10EB70003C4908880921FFF7E5FD00F029F900204C
:10EB800036490870EDE73648807A08280AD03549BA
:10EB900008880921FFF7D6FD00F01AF900202F4957
:10EBA0000870DEE72E4880780007000F002804D0A8
:10EBB000012825D0022843D12EE02848407800289B
:10EBC00000D048E02648C078002803D1012023491E
:10EBD000487003E02248C078204988721F480078B6
:10EBE000912803D01E4800791C49087391201B49C5
:10EBF000087000F0EDF81949087B00F08DF82AE064
:10EC000016484078002800D025E0A120134908705C
:10EC1000032000F09FF81EE010484078002800D044
:10EC200019E00E480078A02809D10E49088808216B
:10EC3000FFF788FD00F0CCF80020084908700AE0D2
:10EC4000084908880521FFF77DFD00F0C1F8002084
:10EC50000249087000BF00BF00BF82E76C28002097
:10EC60008C2700200828002010B528480078802133
:10EC70000840802800D110BD24480078002806D024
:10EC8000234800883F214901884200D0F3E720480B
:10EC9000807A1F4989780907090F884203DD1C48DB
:10ECA000807A082800D0E6E7194880780007000F2E
:10ECB000002805D0164880780007000F072800DDDF
:10ECC000D9E7134800881349088011488078000765
:10ECD000000F4880002407E00D48C01C015D0D486E
:10ECE000001D0155601CC4B20A484088A042F3DCF4
:10ECF00000200649087000F06BF806494A88088829
:10ED00000023091DFFF72EFD00BFB4E76C2800208B
:10ED10008C270020A42700207F2805DC7D21C90046
:10ED200041430A4A91600DE0F12808DBF92806DC2E
:10ED30000107090F64225143044A916002E004492B
:10ED4000024A91600221014A517370477C280020D9
:10ED500018F0010000B503000FF078FB0729050B40
:10ED600011171D2329000121144A11731449516000
:10ED700022E00221114A1173114951601CE0032164
:10ED80000E4A11730F49516016E004210B4A1173AA
:10ED90000D49516010E00521084A117300215160AE
:10EDA0000AE00621054A11730849516004E0002178
:10EDB000024A1173516000BF00BF00BD7C280020D3
:10EDC000A8610000F824010028230000F049020097
:10EDD00000200149087370477C28002002490988F7
:10EDE0000918014A118070477C28002010B52F486F
:10EDF0000078102818D12E48408860280ADD2D4858
:10EE0000807800090001801C2A4988702220274947
:10EE1000087025E02748807800090001254988709E
:10EE20002020224908701BE020480078112816D1C4
:10EE30001E48807A002800D010BD1C484078002869
:10EE400000D0F9E70820194988721A48807800092B
:10EE500000011849887020201449087000E0EBE791
:10EE6000FD20C0001349088008468078F0218843BF
:10EE70003030104988700846C0780020C8700846B5
:10EE8000007914200871032088720220FFF762FFC6
:10EE9000084A917A1088921CFFF716FC05490888E9
:10EEA0000021FFF767FB00BFC6E700006C280020C9
:10EEB000A427002098270020244A118852888A42DB
:10EEC00042D0224A52888A4204DA204A52888A1A58
:10EED00090B207E01D4A52880023DB439A1A521C65
:10EEE000521890B2194A5180127B002A10D0174A4A
:10EEF0005268002A0CD0154A5268824205D9134A3A
:10EF00005268121A114B5A6002E000220F4B5A60ED
:10EF10000E4A527B022A17D10C4A9268002A0CD062
:10EF20000A4A9268824205D9084A9268121A074B27
:10EF30009A6002E00022054B9A60044A9268002A17
:10EF400002D10122014B5A73704700007C28002037
:10EF5000FEB50027002002900190009000250026B9
:10EF60000024FDF763FC012879D10021A748FCF7B4
:10EF7000A9F8552808D1A6480178A648F9F790F9CC
:10EF80000020A349087040E101F0AEF9074601F006
:10EF9000BFF9029001F0B2F9019001F0C3F90090BD
:10EFA00001F098F99C490870F020384000110A28B7
:10EFB00005DBF02038400011C01C054303E0F020C1
:10EFC0003840001105432D023807000F0A2804DBE2
:10EFD0003807000FC01C054302E03807000F054347
:10EFE0002D02F0210298084000110A2805DB029842
:10EFF00008400011C01C054304E0F02102980840BD
:10F00000001105432D0202980007000F0A2805DBB6
:10F0100002980007000FC01C054303E00298000798
:10F02000000F0543F0210198084000110A2805DB74
:10F03000019808400011C01C064304E0F02101982B
:10F04000084000110643360201980007000F0A2805
:10F0500006DB01980007000FC01C064304E0CCE06B
:10F0600001980007000F06433602F021009808407F
:10F0700000110A2805DB009808400011C01C064357
:10F0800004E0F02100980840001106433602009881
:10F090000007000F0A2805DB00980007000FC01CBE
:10F0A000064303E000980007000F06435A48007823
:10F0B000002811D100240AE00020A100554A505038
:10F0C000A100564A5050A100554A5050641C482C8B
:10F0D000F2D3002053490870524800784E4909780D
:10F0E000884218DA002D16D04E4802784B4928463F
:10F0F00000F0D8F800280ED14A480078800047492F
:10F100000D5048480078401C464908700846017870
:10F11000424800F0D8F8434800783F4909788842CF
:10F1200018DA002E16D03F4802783C49304600F0ED
:10F13000B9F800280ED13B480078800037490E50BE
:10F1400038480078401C3749087008460178334831
:10F1500000F0B9F8334800782F49097888420EDD6D
:10F16000002407E00020A1002C4A5050A1002C4AA6
:10F170005050641C482CF5D300202A4908702948B7
:10F1800000782549097888423FD100240FE0A0008B
:10F1900022490858A100224A50500020A1001F4ACD
:10F1A00050501B4801781E4800F08DF8641C1D4823
:10F1B00000788442EBD31848007815490870002085
:10F1C00018490870002413E0A00012490858A10053
:10F1D000134A515888420AD0A00011460858A1008D
:10F1E0000C4A50500A480178104600F06CF8641C34
:10F1F000074800788442E7D307E0054801780548CE
:10F20000F9F74EF8002002490870FEBD28080020DA
:10F2100082000020B00B002080000020900A002017
:10F22000700900208100002010B505F0E7FD10BD39
:10F2300000BF704710B504468020204301460320DC
:10F24000400205F095FC10BD10B5102103204002CE
:10F2500005F08EFC10BD000010B50224024805F038
:10F26000D7FC0446204610BD0106000010B5002161
:10F27000014805F07DFC10BD0106000010B50446F4
:10F28000802020430146024805F072FC10BD0000BA
:10F290000106000010B51021014805F069FC10BD01
:10F2A0000106000030B503460C460021002000BFD7
:10F2B00006E08D0065599D4200D101204D1CE9B248
:10F2C0009142F6DB30BDF8B505460E4600240EE04F
:10F2D000601CC7B207E0BA005119A200501900F033
:10F2E0000AF8781CC7B2B742F5DB601CC4B2701EC6
:10F2F000A042EDDCF8BD10B503680C68A34203D949
:10F300000A6803680B60026010BD70B505460024F2
:10F31000FFF71EFE70BD00002E480078401C2D49EE
:10F3200008702D480078401C2B4908702B48007845
:10F33000401C2A4908702A480068401C2849086077
:10F3400008460068FF219131884202D900202449F3
:10F35000086020480078C82802D900201D4908709C
:10F360001D480078842802D900201B4908701B48DA
:10F370000078502802D90020184908701948184907
:10F380000968405C18490870184812490978405CBF
:10F3900017490870174810490978405C16490870E9
:10F3A00016480E490978405C154908701548094906
:10F3B0000978405C14490870144806490978405C93
:10F3C00013490870134803490978405C12490870D2
:10F3D0007047000053070020540700205507002005
:10F3E0005807002053F901004C070020E3FA010000
:10F3F0004D070020ABFB01004E070020F7FC010089
:10F40000500700202FFC01004F07002047FD01009E
:10F41000510700200FFE01005207002010B58200A6
:10F42000054BD218525C012A04D100228300024C01
:10F430001B195A5410BD0000E826002010B50446E0
:10F44000204600F049FA204600F002F810BD000006
:10F4500010B50446B248007800287DD1B148008834
:10F46000B149884278DAB148007800284FD0B048D6
:10F470000078002803D0AB480088AE490880AE4829
:10F480000078002818D1A7480188AA4800881930B8
:10F49000814206D30120A8490870A2480088A549E6
:10F4A0000880A0480088A349098888421CDA9D4842
:10F4B0000088A049088017E09E4801889948008884
:10F4C0001930814206D300209B4908709548008876
:10F4D000984908809348008896490988884203DD46
:10F4E000904800889349088093480078002857D1B5
:10F4F00092480078042803D08D480078002807D06F
:10F5000088480088822803DA05208C490870A1E029
:10F510008A480078032803D085480078002809D05D
:10F5200080480088FF211931884203DA042083498A
:10F5300008708FE081480078022803D07C4800786A
:10F5400000280AD077480088FF21AF31884204DACA
:10F5500003207A4908707DE0E0E0784800780128CF
:10F5600003D073480078002808D06E48008874499A
:10F57000884203DA0220714908706BE06F48007816
:10F58000002803D06A480078002863D065480088C6
:10F590003721090188425DDA01206849087059E085
:10F5A00065480078012855D164480078012803D0C7
:10F5B0005F480078002809D05A480088372109019F
:10F5C000884203DB00205D49087043E05B48007817
:10F5D000022803D056480078002808D051480088F7
:10F5E0005749884203DB01205449087032E05348F0
:10F5F0000078032803D04E480078002809D04948F5
:10F600000088FF21AF31884203DB02204B4908709C
:10F6100020E04A480078042803D0454800780028B4
:10F6200009D040480088FF211931884203DB0320BC
:10F63000424908700EE041480078052803D03C4854
:10F640000078002806D037480088822802DB042092
:10F650003A490870FDF7D0F83349643988425DD3E0
:10F660003848006800193749086031480078002898
:10F6700008D000202E490870324908602F480078D1
:10F680003149087000F082FD00281FD12D48006824
:10F690002E49884239D300202A4908602A48007838
:10F6A00026490978884205DA27480078401C26490F
:10F6B00008702AE02448007820490978884224DD2F
:10F6C00021480078401E204908701EE01D4800684F
:10F6D0001F49884219D300201A4908601A48007847
:10F6E00016490978884205DA17480078401C1649FF
:10F6F00008700AE01448007810490978884204DD4F
:10F7000011480078401E104908700F4800780B49D6
:10F710000978884202D100200A49086010BD000023
:10F720000B000020020000201C0C00001200002032
:10F7300008000020040000200A000020060000202D
:10F74000760200001800002007000020C05D0000C5
:10F75000407E050000200B4908700B49087001200D
:10F760000A4908700A49087000200A4908700A49C5
:10F7700008700A4908800A4908800A4908800A492D
:10F7800008707047060000200700002008000020D5
:10F79000090000200A0000200B0000200C000020BF
:10F7A0000E000020100000201200002000200B4955
:10F7B00008700B49087001200A4908700A4908704E
:10F7C00000200A4908700A4908700A4908800A4955
:10F7D00008800A4908800A4908707047060000201E
:10F7E0000700002008000020090000200A00002077
:10F7F0000B0000200C0000200E0000201000002054
:10F8000012000020F1B500272D480078002804D010
:10F810000320F9F797FE2B4908802B480088192808
:10F8200047D300202849088028480078142829D286
:10F830000320F9F787FE0746002407E0600024490B
:10F84000085AB84200DD05E0601CC4B21F480078C9
:10F850008442F3DB00BF1D48057808E0681E4000C5
:10F860001B49085A69001A4A5052681EC5B2A5427F
:10F87000F4DC600016490F5214480078401C13490C
:10F88000087016E00026052405E060001049085ABB
:10F890008619601CC4B20F2CF7D30A213046F8F742
:10F8A0004FFC0849088000200849087001200949D8
:10F8B0000870054801880098081803490880F8BDB9
:10F8C0000900002002000020160000200000002097
:10F8D000E4070020120000203A4909881E2928DA8E
:10F8E0000021394A1180394A118039490988394A39
:10F8F000914207DC38490978002914D03449098835
:10F90000914210DD0121354A11700021344A1170F5
:10F91000344A1170304A11700121334A11700021AC
:10F92000324A11704CE02A4909880918284A118086
:10F9300046E024490988274A643291422BDB0021A2
:10F94000234A1180214A11801F490988AF221201E0
:10F95000914207DC20490978002916D01A49098804
:10F96000914212DD02211D4A117000211C4A1170C2
:10F9700005211C4A11700021174A117001211A4AF1
:10F9800011700021194A11701AE00F4909880918ED
:10F990000D4A118014E000210D4A11800A4A11809D
:10F9A0000A4909880B4A914205DD00210B4A117072
:10F9B000094A117004E0054909880918034A1180B1
:10F9C0007047000002000020100000200C00002002
:10F9D0000E000020B80B0000090000200B000020E2
:10F9E0000600002007000020080000200A00002078
:10F9F0000148007870470000580900200148007A4B
:10FA000070470000580900200148807870470000C6
:10FA10005809002001480088704700007C00002041
:10FA2000F8B50023002500950024002200BF94E0D3
:10FA300001259D40ACB20D8825400095009DA54252
:10FA40006FD11A468D79012D0DD1464D0326360210
:10FA5000AD192D5C012696403543424E03273F02E7
:10FA6000F61935540CE03F4D03263602AD192D5CD6
:10FA700001269640B5433B4E03273F02F619355405
:10FA8000CD78002D4ED1374D60352D5CCE78002ECF
:10FA900001D1012600E000269640B543314E603684
:10FAA00035548D78002D2ED12E4D19267601AD19A5
:10FAB0002D5C8E78002E01D1012600E000269640B4
:10FAC000B543284E19277F01F61935540D79002DBD
:10FAD0000ED1244D50352D5C0E79002E01D101261A
:10FAE00000E000269640B5431E4E5036355423E0C4
:10FAF0001C4D50352D5C0E7996403543EEB2194DB4
:10FB000050352E5418E0174D19267601AD192D5C8D
:10FB10008E7896403543134E19277F01F6193554D8
:10FB20000AE018E00F4D60352D5CCE7896403543E5
:10FB3000EEB20C4D60352E544D79012D0AD1094D90
:10FB400030352D5C012696403543EEB2054D3035FB
:10FB50002E5400E000BF5D1CABB2082B00DA67E753
:10FB6000F8BD000000000440FFB5074615461E46DC
:10FB700000243846019900F01FF8002802D0012027
:10FB800004B0F0BD00240CE00A2060430949085C81
:10FB9000B04204D12946204600F05EF807E0601C20
:10FBA00084B20A2060430349085C0028ECD100BFFE
:10FBB0000020E5E7B00100200246002A03D14029D9
:10FBC00001DD01207047032A03D1022901DD012054
:10FBD000F8E7042A03D1202901DD0120F2E7052AF4
:10FBE00003D1202901DD0120ECE70C2A03D11029E3
:10FBF00001DD0120E6E70D2A05D1012903DD4029B9
:10FC000001DA0120DEE70E2A03D1202901D10120EB
:10FC1000D8E70020D6E7000010B5064A03231B02F0
:10FC2000D218125C8A43034B032424021B191A5472
:10FC300010BD00000000044010B5064A03231B025B
:10FC4000D218125C0A43034B032424021B191A54D2
:10FC500010BD00000000044070B502460020B1E075
:10FC60000A2353435A4C1B195B1C440004191B19EB
:10FC70009B788B427DD10A235343554C1B195B1C47
:10FC8000440004191B195B78082B33D10A23534312
:10FC90004F4C1B195B1C440004191B574D4C4E4D17
:10FCA0006419E35C012423430A245443484D641936
:10FCB000641C450045196457464D474EAD192B55F8
:10FCC0000A235343424C1B195B1C440004191B5765
:10FCD000404C35466419E35C022423430A24544310
:10FCE0003B4D6419641C450045196457394DAD19E5
:10FCF0002B5564E00A235343354C1B195B1C44000D
:10FD000004191B195B78092B34D10A235343304C57
:10FD10001B195B1C440004191B572E4C2E4D6419F3
:10FD2000E35C402423430A245443294D6419641C92
:10FD3000450045196457274D274EAD192B550A2309
:10FD40005343234C1B195B1C440004191B57214CC3
:10FD500035466419E35C8024A3430A2454431C4DB4
:10FD60006419641C4500451964571A4DAD192B558B
:10FD700025E025E00A235343154C1B195B1C440066
:10FD800004191B57134C144D6419E35C0A245443A3
:10FD90000F4D6419641C45004519641965780124E8
:10FDA000AC402343DCB20A235343094D5B195B1C6F
:10FDB000450045195B57074D074EAD19EC5404E05B
:10FDC000431CD8B2032800DA4AE700BF70BD000028
:10FDD000B00100200000044075080000F8B50024C0
:10FDE000FCF724FD012861D100F030FB0446BA2263
:10FDF0000721002002F05AFF012C21D100F0A4FBC2
:10FE000000280ED000F056FB054600F047FB0646E2
:10FE100001200346024629460090304605F01CFAB0
:10FE200050E000F047FB054600F038FB0646012095
:10FE30000023024629460090304605F00DFA41E0C5
:10FE4000022C21D100F080FB00280ED000F032FB04
:10FE5000054600F023FB06460120034602462946DC
:10FE60000090304605F0F8F92CE000F023FB054641
:10FE700000F014FB0646002001231A462946009094
:10FE8000304605F0E9F91DE000F05EFB054600F0A4
:10FE900011FB064600F002FB0746012003462A46F6
:10FEA00031460090384605F0D7F90BE000200346B4
:10FEB00002460146009005F0CFF9002207211046C6
:10FEC00002F0F4FEF8BD0000F0B585B000247348E0
:10FED0000078012824D1FCF7A9FC012812D1FCF7F5
:10FEE000C1FA00BF0BE0182C02D1601CC4B204E0C0
:10FEF000BA222146002002F0D9FE601CC4B2242C94
:10FF0000F1DBC8E0FCF7F8FB002406E00022214604
:10FF1000104602F0CBFE601CC4B2242CF6DBBAE023
:10FF2000FCF784FC01287DD1FCF766FC5C49884223
:10FF30007FD35C480088032805DA5A480088401CB3
:10FF40005849088011E000205649088000F0ACFABA
:10FF5000064600F0C7FA07460A21F8F7F1F8054609
:10FF600032462946012009F0FBFD00F02DFC064633
:10FF700000F0D2FB0A210390F8F7E2F8054600F002
:10FF800093FA07463246294608F01EF8FFF726FF87
:10FF900000F050FA05462946012006F0DFFC00F08B
:10FFA0009BFA0646FF21F531F8F7E0F8C5B229467D
:10FFB000012006F00FF9FFF71BFD0546FFF72AFDAC
:10FFC0000646FFF721FD07462B46324639460120FB
:10FFD00005F01CFC00F0E0F80546294601200AF077
:10FFE00065F800F0B3FB054600F0BAFA064600F0EB
:10FFF0006DFA074600F0B0FB039000F0B7FA3B46FD
:020000040001F9
:1000000000960195029001460120039A09F0E0F85C
:1000100000F076FB054600F06DFB064600F076FB2F
:10002000074601E008E004E02A46314606F0CEFE2D
:1000300031E0FCF791FA2EE0FCF75EFB0022232171
:10004000104602F033FE00222221104602F02EFE5E
:1000500000220721104602F029FE00220821104646
:1000600002F024FE00220921104602F01FFE0022A9
:100070000A21104602F01AFE00221321104602F057
:1000800015FE00221121104602F010FE002212215E
:10009000104602F00BFE05B0F0BD00000301002089
:1000A000B80B00007600002001490860704700008E
:1000B0008007002002480068401C01490860704722
:1000C0007C070020F3B581B0064600200E49086089
:1000D00000F01EF8044600F01BF805462F1B3046C2
:1000E000029903F087FD00900AE000F011F8054640
:1000F0002F1B06480068002802D00448006880478B
:1001000000988742F1D3FEBD7C07002080070020C5
:1001100001480068704700007C0700200B490978FF
:10012000012901D101200FE008490978022901D1F4
:10013000022009E005490978032901D1042003E0E0
:100140000121024A117001207047000015070020AC
:1001500010B5094B1B8899B20A12C8B2D343313388
:10016000064C2370C3432333637013465633A37086
:1001700003467133E37010BD440700201B070020C5
:1001800001480088704700002400002001480088D2
:10019000704700003C0000200148007870470000D4
:1001A0008800002001480078704700008900002086
:1001B00010B5002205210648FAF772FF0402012259
:1001C00005210348FAF76CFF201880B210BD00002B
:1001D0002808002010B5062205210348FAF760FF21
:1001E000C006C00F10BD00002808002010B5042272
:1001F00005210648FAF754FF040205221146034878
:10020000FAF74EFF201880B210BD00002808002029
:1002100010B5062205210248FAF742FFC01110BDB1
:100220002808002010B5022205210248FAF738FFFD
:1002300010BD00002808002010B506220521034843
:10024000FAF72EFF8006C00F10BD0000280800201E
:1002500010B5042202210348FAF722FFC007C00F9D
:1002600010BD00002808002010B505220221034817
:10027000FAF716FFC007C00F10BD000028080020C5
:1002800010B5002204210348FAF70AFF4006400F88
:1002900010BD00002808002010B5002201210248EE
:1002A000FAF7FEFE10BD00002808002010B501225C
:1002B00011460248FAF7F4FE10BD0000280800209D
:1002C00010B5022203210248FAF7EAFE10BD000031
:1002D0002808002010B5032200210248FAF7E0FEAA
:1002E00010BD00002808002010B500221146024869
:1002F000FAF7D6FE10BD00002808002010B5042231
:1003000000210248FAF7CCFE10BD000028080020AA
:1003100010B5012200210248FAF7C2FE10BD00000C
:100320002808002010B5052200210248FAF7B8FE7F
:1003300010BD000028080020322815DA3C498978D1
:10034000012903DD01213A4A517070E0384989786A
:10035000002905DD2F286ADC0021354A517066E04E
:100360000021334A517062E03E2817DA322815DB4B
:100370002F498978022903DD02212D4A517056E068
:100380002B498978012905DD3B2850DC0121284AC9
:1003900051704CE00121264A517048E0502817DA8C
:1003A0003E2815DB22498978032903DD0321204AF1
:1003B00051703CE01E498978022905DD4D2836DC64
:1003C00002211B4A517032E00221194A51702EE07D
:1003D000622817DA502815DB15498978042903DDCE
:1003E0000421134A517022E011498978032905DD5F
:1003F0005F281CDC03210E4A517018E003210C4ACF
:10040000517014E073280FDA62280DDB08498978EF
:10041000042905DD70280ADC0421054A517006E034
:100420000421034A517002E00521014A51707047CE
:10043000580900200148007870470000070000209C
:100440000148007870470000F00000200148007863
:1004500070470000EF000020F8B5002600240025BA
:10046000FDF706F907460A21F7F76AFE054609482F
:100470000068854200D303E006480068461B344606
:100480007D200001844200D30446034804600068D4
:10049000F8BD000028010020240100200148007858
:1004A00070470000FB000020014800797047000001
:1004B000E80000200148407870470000FB00002061
:1004C0000148807970470000E80000200148407929
:1004D00070470000E80000200148008870470000D5
:1004E0002600002010B50024FFF7DEFF00280AD107
:1004F0000A4800880A49884202DB08460749088002
:100500000648048808E005480088FCF75FFE84B2CE
:100510000448844200DB0446204610BD3E00002013
:10052000C6070000CE040000002005490988054ADE
:10053000914202DB1146024A118001490888704746
:100540003E000020C6070000014800787047000008
:100550004D07002001480078704700004F07002039
:100560000148007A704700006409002070B500243B
:100570000E48C07A01280ED10C490868FCF776FABB
:100580000546323564212846F7F7DAFD84B2632C3C
:100590000ADD632408E005480088401D84B20A2172
:1005A0002046F7F7E3FD84B2204670BD64090020C1
:1005B00070B5002407490868FCF758FA05460A2177
:1005C000F7F7BEFD84B20448844200DD04462046AD
:1005D00070BD000064090020DE03000010B5002497
:1005E00000F016F8012801D103240CE000F010F807
:1005F000022802D1FF24373405E00A21034800888D
:10060000F7F7B4FD84B2204610BD000002000020C0
:1006100001480078704700000B00002010B500244E
:10062000044804F0F5FA002801D0012400E0002479
:10063000204610BD0307000010B50024054804F053
:10064000E7FA002802D00120044601E00020044619
:1006500010BD00000507000010B50024054804F097
:10066000D7FA002802D00120044601E00020044609
:1006700010BD00000707000010B50024062004F09C
:10068000C7FA002801D0012400E00024204610BD54
:1006900010B50024054804F0BBFA002802D0012060
:1006A000044601E00020044610BD000006070000DB
:1006B00010B50024044804F0ABFA002801D001244E
:1006C00000E00024204610BD0305000010B5002402
:1006D000044804F09DFA002801D0012400E0002421
:1006E000204610BD040500000148807A70470000D4
:1006F000640900200148807870470000D00C002079
:100700000148406870470000D00C00200148407844
:1007100070470000D00C002070B50024FFF7C4FE25
:10072000002803D1FCF7A4FF04460DE0FFF7BCFE50
:10073000012806D1FCF79CFF0546FCF747FD04465F
:1007400002E0FCF795FF0446204670BD0148407A60
:10075000704700006409002070B500240E48C07A7C
:1007600001280ED10C494868FCF780F9054632355E
:1007700064212846F7F7E4FC84B2632C0ADD632485
:1007800008E005488088401D84B20A212046F7F71A
:10079000EDFC84B2204670BD6409002070B50024D1
:1007A00007494868FCF762F905460A21F7F7C8FCD3
:1007B00084B20448844200DD0446204670BD000037
:1007C00064090020DE03000070B50024FFF76CFE12
:1007D000002803D1FCF75EFF04460FE0FFF764FE3C
:1007E000012807D10020FCF755FF0546FCF7EEFC79
:1007F000044603E00020FCF74DFF0446204670BD90
:1008000001480078704700004200002070B505469E
:100810000024032D00D170BD002D01D0012D1BD16E
:1008200081210320800204F0A3F98021134804F001
:100830009FF932211248FFF745FC002409E0A2008D
:10084000104BD2189178A200985A04F091F9601CCC
:10085000C4B23B2CF3DB0FE0022D0DD1002409E0E4
:10086000A200094BD2189178A200985A04F080F99E
:10087000601CC4B23B2CF3DB00BFCCE702060000D7
:10088000A0860100E8EF0100D4F00100F8B50021D6
:1008900000240023002200BF0AE001258D40ABB2F6
:1008A00005881D402C469C4200D10A464D1CA9B229
:1008B0001029F2DB0588FF2D1FDC284D6D7E068890
:1008C000B543264E757635462D7E0688B543234EB4
:1008D000357635466D7E8678F607F60F96403543B9
:1008E0001E4E757635462D7E867802273E40760868
:1008F00096403543194E357622E0184DED7E068838
:10090000B543164EF5763546AD7E0688B543134E93
:10091000B5768578ED07ED0F1646083EB5400F4ECB
:10092000F67E35430D4EF5768578022635406D0806
:100930001646083EB540094EB67E3543074EB5769D
:100940000025009505E000BF6D462D786D1CEEB2C8
:1009500000966D462D78012DF5D9F8BD206B044029
:10096000C107C90F002905D00021394A11710022A1
:1009700038490A7102210140002905D00021344A7A
:100980001172002233490A7204210140002905D066
:1009900000212F4A117300222E490A7308210140B9
:1009A000002905D000212A4A1174002229490A741D
:1009B00010210140002905D00021254A117500228F
:1009C00024490A7520210140002905D00021204A30
:1009D000117600221F490A7640210140002904D0E7
:1009E00000221B494A711B494A718021014000299C
:1009F00004D0002216494A7216494A72FF21013179
:100A00000140002904D0002211494A7311494A7358
:100A1000012149020140002904D000220C494A74F6
:100A20000C494A74012189020140002904D00022A6
:100A300007494A7507494A750121C9020140002941
:100A400004D0002202494A7602494A7670470000E3
:100A50000060004000610040C107C90F002905D0B7
:100A600001223C490A7100213B4A117102210140D7
:100A7000002905D0012237490A720021364A117235
:100A800004210140002905D0012232490A730021C6
:100A9000314A117308210140002905D001222D4956
:100AA0000A7400212C4A117410210140002905D03C
:100AB000012228490A750021274A11752021014089
:100AC000002905D0012223490A760021224A117605
:100AD00040210140002905D001221E494A7100220F
:100AE0001D494A7180210140002905D00122194980
:100AF0004A72002218494A72FF210131014000293F
:100B000005D0012213494A73002213494A73012177
:100B100049020140002905D001220E494A740022F1
:100B20000D494A74012189020140002905D00122A2
:100B300008494A75002208494A750121C902014045
:100B4000002905D0012203494A76002202494A764B
:100B500070470000006100400060004010B50C4884
:100B60000078002803D00B4A5068916888470848ED
:100B70004078002803D0084A5068916888470448A4
:100B80008078002803D0054A50689168884710BDD6
:100B900000600040000300208004002000060020C8
:100BA00010B508480079002803D0074A1069516938
:100BB000884704484079002803D0044A5068916867
:100BC000884710BD00600040000300208C04002016
:100BD00010B50848007A002803D0074AD069116A86
:100BE00088470448407A002803D0044A5068916836
:100BF000884710BD006000400003002098040020DA
:100C000010B50848007B002803D0074A906AD16AD3
:100C100088470448407B002803D0044A5068916804
:100C2000884710BD0060004000030020A40400209D
:100C300010B50848007C002803D0074A506B916B20
:100C400088470448407C002803D0044A50689168D3
:100C5000884710BD0060004000030020B004002061
:100C600010B50848007D002803D0074A106C516C6D
:100C700088470448407D002803D0044A50689168A2
:100C8000884710BD0060004000030020BC04002025
:100C900010B50848007E002803D0074AD06C116DBB
:100CA00088470448407E002803D0044A5068916871
:100CB000884710BD0060004000030020C8040020E9
:100CC00010B50848407F002803D0074A5068916853
:100CD00088470448007F002803D0044A906DD16DF6
:100CE000884710BD00600040D404002000030020AD
:100CF00010B508484078002803D0074A506891682A
:100D0000884704480078002803D0044A506E916E4A
:100D1000884710BD20600040E00400200003002050
:100D200010B509480079002803D0084A106F516FA8
:100D300088470548001D4078002803D0044A5068C1
:100D40009168884710BD000020600040000300202B
:100D5000EC04002010B5034AD06F783291688847C0
:100D600010BD00000003002010B5024A50689168D1
:100D7000884710BD8403002010B50948007C002876
:100D800003D0084A50689168884705481030407879
:100D9000002803D0044A50689168884710BD0000BD
:100DA00020600040900300201005002010B5024A8A
:100DB00050689168884710BD9C03002010B5024A16
:100DC00050689168884710BDA803002010B50948F5
:100DD000007F002803D0084A50689168884705487A
:100DE0001C304078002803D0044A50689168884736
:100DF00010BD000020600040B40300203405002036
:100E000010B50C480078002803D00B4A5068916850
:100E1000884708484078002803D0084A50689168FD
:100E2000884704488078002803D0054A50689168B4
:100E3000884710BD40600040C003002040050020EE
:100E4000C006002010B50D480079002803D00C4AD8
:100E50005068916888470948001D4078002803D0F1
:100E6000084A5068916888470448001D8078002827
:100E700003D0054A50689168884710BD4060004023
:100E8000CC0300204C050020CC06002010B50D48F6
:100E9000007A002803D00C4A5068916888470948B6
:100EA00008304078002803D0084A50689168884785
:100EB000044808308078002803D0054A50689168BB
:100EC000884710BD40600040D8030020580500202E
:100ED000D806002010B50D48007B002803D00C4A2E
:100EE00050689168884709480C304078002803D042
:100EF000084A50689168884704480C308078002878
:100F000003D0054A50689168884710BD4060004092
:100F1000E403002064050020E406002010B50D481D
:100F2000007C002803D00C4A506891688847094823
:100F300010304078002803D0084A506891688847EC
:100F4000044810308078002803D0054A5068916822
:100F5000884710BD40600040F0030020700500206D
:100F6000F006002010B5024A50689168884710BD0D
:100F7000FC03002010B50948007E002803D0084A71
:100F8000506891688847054818304078002803D099
:100F9000044A50689168884710BD000040600040D6
:100FA000080400208805002010B50948007F0028AB
:100FB00003D0084A50689168884705481C3040783B
:100FC000002803D0044A50689168884710BD00008B
:100FD00040600040140400209405002010B508482B
:100FE0000078002803D0074A506891688847044871
:100FF0004078002803D0044A50689168884710BDA3
:101000006060004020040020A005002010B50948C1
:101010000079002803D0084A50689168884705483D
:10102000001D4078002803D0044A50689168884722
:1010300010BD0000606000402C040020AC050020C2
:1010400010B50948007A002803D0084A5068916812
:101050008847054808304078002803D0044A506883
:101060009168884710BD000060600040380400208F
:10107000B805002010B5024A50689168884710BD35
:101080004404002010B5024A50689168884710BD9A
:101090005004002010B50948007D002803D0084AFC
:1010A000506891688847054814304078002803D07C
:1010B000044A50689168884710BD00006060004095
:1010C0005C040020DC05002010B50948007E0028E3
:1010D00003D0084A5068916888470548183040781E
:1010E000002803D0044A50689168884710BD00006A
:1010F0006060004068040020E805002010B5094841
:10110000007F002803D0084A506891688847054846
:101110001C304078002803D0044A50689168884702
:1011200010BD00006060004074040020F405002041
:1011300010B5FE4800688079002806D001286ED0DE
:1011400002286DD003286CD104E2F8480068407989
:1011500003000DF07BF90A0614BC2BBC47BC67BC2E
:101160009BBC09F005FB0020F0490968C873EF48F3
:1011700000684079401CED4909684871AEE0EC49CF
:101180000969EA4A1268D27A885C09F069FBE74883
:1011900000684079401CE54909684871E3480068E7
:1011A0004079401CE1490968487197E001F0E6FE8A
:1011B000002810D109F054FBDC4800684079401C3D
:1011C000DA4909684871D94800684079401CD74914
:1011D0000968487105E009F0F5FA0020D34909686B
:1011E00048717BE001F0CAFE002811D1012009F00E
:1011F00037FBCE4800684079401CCC4909684871EB
:10120000CA4800684079401CC8490968487105E02F
:1012100009F0D8FA0020C549096848715EE05FE02E
:10122000FEE0A3E101F0AAFE002828D1BF49096829
:10123000C97A24225143BF4A12688918BB4A1268EE
:10124000D27B885C09F00CFBB8480068C07B401C6E
:10125000B6490968C873B5480068C07B242814D310
:10126000B24800684079401CB04909684871AF48ED
:1012700000684079401CAD490968487105E009F0F3
:10128000A1FA0020A9490968487127E001F076FE1B
:10129000002815D1A5480068C07A401CA3490968F8
:1012A000C872A2480068C07AA1490978884207DB61
:1012B00000209E490968C87201209C49096888710C
:1012C00009F080FA002099490968487106E009F0A0
:1012D00079FA002095490968487100BF00BF4FE1C5
:1012E00092480068407903000DF0B0F808051391AA
:1012F0002A914791709109F03BFA00208B490968C7
:10130000C8738A4800684079401C88490968487158
:1013100084E087490969854A1268D27A885C09F0B5
:101320009FFA824800684079401C804909684871EA
:101330007E4800684079401C7C49096848716DE02E
:1013400001F01CFE002811D1262009F089FA774807
:1013500000684079401C7549096848717348006805
:101360004079401C71490968487105E009F02AFA82
:1013700000206E490968487150E001F0FFFD002827
:101380001DD1012009F06CFA68480068C07B401C40
:1013900066490968C87365480068C07B242814D36F
:1013A000624800684079401C6049096848715F489C
:1013B00000684079401C5D490968487105E009F002
:1013C00001FA002059490968487127E001F0D6FD6B
:1013D000002815D155480068C07A401C5349096857
:1013E000C87252480068C07A51490978884207DBC0
:1013F00000204E490968C87202204C49096888716A
:1014000009F0E0F9002049490968487106E009F04F
:10141000D9F9002045490968487100BF00BFAFE015
:1014200042480068407903000DF010F80805138B5E
:101430002A8B478B638B09F09BF900203B49096895
:10144000C8733A4800684079401C384909684871B7
:101450007EE037490969354A1268D27A885C09F01A
:10146000FFF9324800684079401C304909684871EA
:101470002E4800684079401C2C490968487167E093
:1014800001F07CFD002811D1252009F0E9F9274859
:1014900000684079401C2549096848712348006864
:1014A0004079401C21490968487105E009F08AF932
:1014B00000201E49096848714AE001F05FFD0028DC
:1014C00010D109F0CDF9194800684079401C17493E
:1014D00009684871154800684079401C134909683B
:1014E000487105E009F06EF900201049096848715B
:1014F0002EE001F043FD002815D10C480068C07AA9
:10150000401C0A490968C87208480068C07A08493E
:101510000978884207DB002004490968C872032063
:1015200002490968887109F04DF905E0D0070020EB
:10153000402B0020CC070020002012490968487188
:1015400006E009F03FF900200E490968487100BF24
:1015500000BF15E000200B49096888710949096836
:101560004871062007490968C87009E009F02AF99E
:10157000002004490968487102490968887100BF60
:1015800000BF10BDD007002010B56A480068407940
:1015900003000CF05BFF090610C627C644C6608E28
:1015A000C60009F0E5F8634800684079401C6149CD
:1015B00009684871BCE0604909695E4A1268D27ADC
:1015C000885C09F04DF95B4800684079401C594936
:1015D00009684871574800684079401C55490968B6
:1015E0004871A5E001F0CAFC002811D14F2009F094
:1015F00037F9504800684079401C4E4909684871E5
:101600004C4800684079401C4A490968487105E027
:1016100009F0D8F8002047490968487188E001F0CE
:10162000ADFC002810D109F01BF942480068407950
:10163000401C4049096848713E4800684079401C98
:101640003C490968487105E009F0BCF800203949B7
:10165000096848716CE001F091FC002822D13548FE
:101660000068C07A401C33490968C8723148006874
:10167000C07A3149097888420FDB00202D4909687A
:10168000C8722C4800684079401C2A490968487192
:10169000002028490968486208E0002025490968B7
:1016A000487103E0002023490968487109F08AF86D
:1016B0003EE020480068407C002816D01E48C068E4
:1016C000002803D01C48C168192088470020194908
:1016D000096848621749096848711649096888719C
:1016E000052014490968C8701AE012480068406A69
:1016F000282807D20F480068406A401C0D49096835
:1017000048620DE000200B490968486209490968F0
:101710004871084909688871052006490968C87038
:1017200006E009F04FF8002002490968487100BF3F
:1017300000BF10BDD0070020402B002010B50024B2
:10174000F7480068807A01287ED1F5480068C079A2
:1017500000287AD0F24800688079002804D0012857
:1017600074D0022873D191E1ED480068007B2428F1
:101770006ED2EB480068C07901287AD1002475E068
:10178000E7480068C07A24214843E64909684018C0
:10179000E3490968097B415CE1480068C07A24227A
:1017A0005043E14A12688018DD4A1268127B805C5F
:1017B000814229D0DA480068C07A24214843DA49B6
:1017C00009684018D6490968097B415CD44800681B
:1017D000C07A24225043D34A12688018D04A126833
:1017E000127B8154CE480068407B242805D3CC4826
:1017F0000068007BCA4909684873C9480068007BD3
:10180000C7490968887308E0C5480068407B2428F8
:1018100003D20120C24909688871C1480068007B71
:10182000401CBF4909680873BD480068007B242834
:1018300008D3BB480068407B242803D20120B84964
:1018400009688871B64805E0D3E1CDE169E0BAE105
:1018500038E00EE00068007B242804D2B04800681D
:101860008079012800D103E0601CC4B2242C87D306
:1018700056E0002413E0AA480068C07A24214843B7
:10188000A94909684018015DA5480068C07A24226A
:101890005043A44A126880180155601CC4B2242C1D
:1018A000E9D300209E490968487323209C490968B0
:1018B000887301209A490968887124209849096829
:1018C00008732DE000209649096808739448006861
:1018D000C07A401C92490968C87291480068C07A71
:1018E00092490978884217DB8D480068007C0128FE
:1018F00004D102208A490968887106E000208849DD
:101900000968887186490968C87100208449096896
:10191000C8728349096808740020814909684871C0
:1019200061E17F480068407903000CF08FFD0805F5
:1019300013A62AA651A68EA6012079490968087423
:1019400008F016FF764800684079401C7449096821
:10195000487199E075490969714A1268D27A885CC0
:1019600008F07EFF6E4800684079401C6C490968A9
:1019700048716B4800684079401C694909684871A2
:1019800082E001F0FBFA00281BD165490968497B18
:10199000491CC8B208F064FF61480068407B604998
:1019A0000968C8735E4800684079401C5C49096852
:1019B00048715B4800684079401C59490968487182
:1019C00005E008F0FFFE00205549096848715BE01A
:1019D00001F0D4FA00282BD151490968C97A242290
:1019E0005143504A126889184D4A1268D27B885C6C
:1019F00008F036FF4A480068C07B401C4849096827
:101A0000C87347480068C07B45490968897B88429C
:101A10001ADD434800684079401C41490968487113
:101A20003F4800684079401C3D49096848710BE017
:101A300008F0C8FE3A480068407B39490968C87315
:101A400000203749096848711EE001F097FA002824
:101A50000CD1334909688871242031490968C87359
:101A60002F49096848732E490968887308F0AAFE4F
:101A700000202B490968487106E008F0A3FE002009
:101A800027490968487100BF00BFACE024480068DE
:101A9000407903000CF0DAFC08050F8E268E4C8E80
:101AA000688E08F065FE1E4800684079401C1C499D
:101AB0000968487185E01D490969194A1268D27A96
:101AC000885C08F0CDFE164800684079401C144937
:101AD00009684871124800684079401C104909683B
:101AE00048716EE001F04AFA002811D1252008F073
:101AF000B7FE0B4800684079401C094909684871E5
:101B0000074800684079401C05490968487105E0AC
:101B100008F058FE002002490968487151E00000B1
:101B2000D0070020CC070020C8070020402B002051
:101B300001F024FA002810D108F092FE64480068F1
:101B40004079401C624909684871614800684079E1
:101B5000401C5F490968487105E008F033FE002029
:101B60005B49096848712CE001F008FA00281AD195
:101B700057480068C07A401C55490968C8725448E3
:101B80000068C07A5349097888420CDB002050492C
:101B90000968C8724E49096888714D4909684871D9
:101BA0004B490968C87108F00DFE002048490968D2
:101BB000487106E008F006FE0020454909684871B2
:101BC00000BF00BF0FE008F0FDFD0020404909689C
:101BD00048713F49096888713D49096808733C4963
:101BE0000968C87200BF71E000203949096888722D
:101BF0006CE037480068807A022867D13448006872
:101C0000007A00285ED0324800684079002804D06D
:101C100001280CD0032846D11BE008F0A9FD2C4870
:101C200000684079401C2A490968487149E0002051
:101C300008F016FE264800684079401C24490968CF
:101C40004871234800684079401C2149096848715F
:101C500037E008F057FD002812D11D480068407891
:101C6000401C1B49096848701948006840780328DF
:101C700012D301F023FA00201549096848700BE0DF
:101C80000020134909680872AA2011490968887060
:101C900000200F490968487008F094FD00200C49A5
:101CA000096848710DE008F08DFD002008490968B9
:101CB0004871074909684870AA2005490968887071
:101CC00000BF03E0002002490968887210BD0000CF
:101CD000D0070020402B0020F8B504460D46002612
:101CE0000C2060431D49085C002801D00120F8BD8C
:101CF0000C2060431949401885600C20604340184F
:101D00008068002801D10120F1E701210C20604307
:101D1000124A115400222046E317DB0E1B185B11F8
:101D20005B01E31A9B000E4FDB19E717FF0E3F190B
:101D30007F11DA550CF0BCFB00222046E317DB0EC6
:101D40001B185B115B01E31A9F00064BFB18E7179A
:101D5000FF0E3F197F11DA553046C8E70003002017
:101D6000006000400061004000BFFEE709480088B5
:101D7000401C08490880084600880749884208DD59
:101D800006480078002804D008460249088001204F
:101D900088707047E4000020DC050000EF000020A0
:101DA00010B515488078012824D1144800780128FE
:101DB0000CD113480078012808D1002011498870FF
:101DC000084602F0F7FC00200D4908700B48007827
:101DD00002280CD10C480078012808D100200949BC
:101DE0008870084602F0E6FC0020074908700020D1
:101DF0000249087010BD0000E4000020EF00002040
:101E0000F1000020FB000020F200002070470000DD
:101E100010B500F03DFE012803D1002001490880E3
:101E2000887010BDE4000020F0B505460E46174648
:101E300000243A463146284600F038FE00BF42E012
:101E400000202101394A126850522101374A126894
:101E50008918488000212001344A12688018818046
:101E60002001324A12688018C18020012F4A12686E
:101E70008018017220012D4A1268801841722001D9
:101E80002A4A1268801881722001284A1268801834
:101E9000C17200202101254A1268891808730021A7
:101EA0002001224A126880184173002021011F4A34
:101EB000126889188873002120011C4A1268801852
:101EC000C173601CC4B21A484078A042B8DC6420D8
:101ED0001849096808807D20C000164909684880B3
:101EE00015481449096888807D2000011149096856
:101EF000C88010490968088110480E49096848815E
:101F00000F480C490968888140000A490968C8815E
:101F10003220084909680882FF20F5300549096820
:101F20004882044909688882F0BD000090070020BB
:101F3000840700208C0700204C04000010270000BC
:101F40003075000038B5002404E00020134908551E
:101F5000601C84B2282CF8D30121684641700170BE
:101F60006A460F490D48FFF75FFF7D21C900322007
:101F700000F08CF90B490C4800F0A6F909486430D0
:101F800000F038F90748C83000F044F9074800F07D
:101F900057F9074800F06AF938BD0000DC2300203B
:101FA00058F5010028230000B80B0000542400005D
:101FB0001027000010B521480078002803D1012027
:101FC0001E49087038E01D480078012810D11C48CF
:101FD0000078012808D100201A498870084602F0CC
:101FE000E9FB00201649087002201449087023E01C
:101FF00012480078022810D113480078012808D12F
:10200000002010498870084602F0D4FB00200E49D9
:1020100008700320094908700EE00848007803287A
:1020200003D104200549087006E00448007804281C
:1020300002D100200149087010BD0000EF0000200F
:10204000F1000020FB000020F2000020F8B5002481
:10205000002500263648007800281ED13548007833
:10206000002803D101203349087016E03148007878
:10207000012803D102202F4908700EE02D48007876
:10208000022803D103202B49087006E02948007874
:10209000032802D10020274908702548007801282C
:1020A0000ED1012417250026234801233246294654
:1020B0000090204601F0E2FD01202049087036E042
:1020C0001B48007802280FD101243B2500261A481E
:1020D000401C0123324629460090204601F0CEFDE7
:1020E00001201749087022E01148007803280DD11B
:1020F000FEF7DAF9002803D101201249087102E045
:102100000020104908710CF073F910E008480078BD
:1021100004280CD1FEF7DAF9002803D1012009497F
:10212000487102E00020074948710CF061F9F8BDE0
:10213000EF000020F0000020FB000020F100002054
:10214000F2000020E800002010B5044623000CF047
:102150007DF90942060E1617181940414500FAF795
:102160004BFB2049884201D3FFF770FF37E0FAF7B5
:1021700043FB1C49884201D3FFF71CFF2FE02EE0F0
:102180002DE02CE0FAF738FB1649884220D301F005
:102190003FFD1548007803280ED114480078002828
:1021A0000AD1FEF78DF9002803D10120104988716A
:1021B00002E000200E4988710B480078012805D103
:1021C0000A480078002801D1FAF7A8FC09F0D8FFE6
:1021D00005E004E003E0FFF7C9FD00E000BF00BF39
:1021E00010BD0000B80B0000F0000020EF00002040
:1021F000E800002001460020054A126852898A4200
:1022000001DC012002E0024A1268118170470000DF
:102210008C07002001460020084A126812898A4271
:1022200001DB012009E0054A126892898A4201DC3B
:10223000012002E0014A1268518170478C0700209A
:1022400001460020084A126852898A4201DB0120B7
:1022500009E0054A1268D2898A4201DC012002E0C5
:10226000014A1268918170478C07002001460020C6
:10227000054A126892898A4201DB012002E0024A83
:102280001268D181704700008C07002002460020B0
:102290000C4B1B681B8A934201DD012010E08A422F
:1022A00001DB01200CE0074B1B689B888B4201DCA3
:1022B000012005E0034B1B681A80024B1B68598004
:1022C000704700008C070020024600200C4B1B6862
:1022D0001B8A934201DD012010E08A4201DB0120CC
:1022E0000CE0074B1B685B88934201DB012005E093
:1022F000034B1B689A80024B1B68D9807047000013
:102300008C07002070B5044600250C206043FE4970
:10231000096840184068002807D00C216143FA4A38
:10232000126889184868804705460C206043F649C2
:102330000968085C002873D10C206043F2490968E1
:1023400040188068002874D02001F04909684018BE
:10235000C07A02280AD1032D08D10C206043EA4A32
:102360001268801881680120884762E02001E749EF
:1023700009684018C07A02280AD1042D08D10C201F
:102380006043E14A1268801881680220884750E063
:102390002001DE4909684018C07A02280AD1052DBB
:1023A00008D10C206043D84A126880188168032045
:1023B00088473EE02001D54909684018C07A0228C4
:1023C0000AD1062D08D10C206043CF4A126880182C
:1023D0008168042088472CE02001CC490968401816
:1023E000C07A02280AD1072D08D10C206043C64AC2
:1023F000126880188168052088471AE02001C349C7
:1024000009684018C07A02280BD1082D09D10C2088
:102410006043BD4A1268801881680620884708E03A
:102420000DE00C206043B84A1268801881680020D3
:1024300088472001B54909684018C5720CE30C2093
:102440006043B1490968085C012873D10C206043DE
:10245000AD49096840188068002874D02001AB4954
:1024600009684018C07A03280AD1022D08D10C202F
:102470006043A54A1268801881680120884762E09D
:102480002001A24909684018C07A04280AD1022D07
:1024900008D10C2060439C4A126880188168022091
:1024A000884750E02001994909684018C07A0528FA
:1024B0000AD1022D08D10C206043934A126880187B
:1024C0008168032088473EE0200190490968401850
:1024D000C07A06280AD1022D08D10C2060438A4A0E
:1024E000126880188168042088472CE02001874901
:1024F00009684018C07A07280AD1022D08D10C209B
:102500006043814A126880188168052088471AE074
:1025100020017E4909684018C07A08280BD1022D95
:1025200009D10C206043784A12688018816806201F
:10253000884708E00DE00C206043734A1268801859
:102540008168002088472001704909684018C572D9
:1025500082E20C2060436C490968085C0228F7D1CC
:10256000002D7DD1200169490968085A6849096828
:10257000098A884275DA200164490968085A0A30D4
:1025800081B22001614A1268115220015F49096835
:10259000085A5F490968098A884231DB20015B4992
:1025A0000968401840885A4909680988884227DB29
:1025B00020015649096840184088554909684988EA
:1025C00088421DDC00202101504A12688918488089
:1025D00020014E4909684018807A0028B8D10C20A3
:1025E000604349490968401880680028B0D00C2031
:1025F0006043454A126880188168012088472BE2B1
:10260000200142490968085A41490968098A8842F3
:102610009EDB20013D490968401840883C49096813
:102620008988884294DB200138490968401840882D
:1026300037490968C98888428ADC00202101334A69
:102640001268891848802001304909684018807A4A
:102650000028D4D10C2060432B490968401801E0C0
:1026600063E00BE080680028C9D00C206043264A54
:1026700012688018816802208847EDE1002021015E
:10268000224A1268891848802101204A1268891854
:10269000C872002120011D4A12688018C1802001E3
:1026A0001A4A1268801841722001184A126880186C
:1026B0008172184801782001144A1268801801724A
:1026C00000202101114A12688918888021010F4ACF
:1026D00012688918087321010C4A12688918487316
:1026E00021010A4A12688918887300212001074ACB
:1026F00012688018C1730C206043034909684018B0
:1027000080680028B9D007E08807002090070020E3
:102710008C070020840700200C206043CF4A1268F9
:10272000801881680020884796E1012DA5D12001FD
:10273000CB4909684018C07AA84225D00021200161
:10274000C74A12688018418000202101C44A1268DB
:102750008918C8802001C24909684018C572C1485B
:1027600000782101BE4A12688918487200202101B0
:10277000BB4A126889188880BA4801782001B84A93
:1027800012688018017267E12001B5490968401894
:10279000007AB4490978884220D0B24800782101F3
:1027A000AF4A1268891808722001AD4909684018BB
:1027B000407AAC490978884209D02001A8490968C3
:1027C000401880882101A64A12688918C880002113
:1027D0002001A34A12688018818012E02001A049DC
:1027E000096840188088A04988420AD220019C4983
:1027F0000968401880880A302101994A12688918AE
:102800008880200196490968401840889649884286
:102810000AD2200192490968401840880A302101F3
:102820008F4A12688918488020018D49096840182C
:10283000407A8C490978884205D001202101884AD4
:1028400012688918887220018549096840184088F3
:10285000864909680988884204DB00212001804AF2
:102860001268115220017E4909684018807A0028B8
:102870007ED10C206043794909684018806800289F
:1028800077D020017649096840184088774909685F
:102890000989884214DB2001714909684018007BCE
:1028A00000280DD10C2060436C4A126880188168A2
:1028B0000320884701202101694A1268891808739A
:1028C00020016749096840184088684909684989B2
:1028D000884214DB2001624909684018407B0028C7
:1028E0000DD10C2060435D4A126880188168042075
:1028F0008847012021015A4A12688918487320012B
:1029000057490968401840885849096889898842A8
:1029100014DB2001524909684018807B00280DD142
:102920000C2060434D4A1268801881680520884752
:10293000012021014A4A12688918887320014849F8
:1029400009684018408849490968C989884210DBEC
:102950002001434909684018C07B00287CD10C2025
:1029600060433E4A1268801881680620884701E06B
:1029700007E03BE001202101394A12688918C87339
:102980006AE02001364909684018407A01282ED1B2
:102990003448007802282AD12001314909684018BA
:1029A000C08832490968498A884255DB20012C4990
:1029B0000968401880882D490968898A88424BDB5C
:1029C0000C2060432549096840188068002843D0DE
:1029D0000C206043214A12688018816807208847CC
:1029E000002021011E4A12688918487234E0200133
:1029F0001B4909684018407A02282DD119480078EF
:102A0000012829D12001164909684018C0881749B2
:102A10000968898A88421FDB20011149096840182A
:102A2000808812490968498A884215DB0C20604376
:102A30000A4909684018806800280DD00C206043BE
:102A4000064A126880188168082088470020210102
:102A5000034A12688918487270BD00008807002078
:102A60009007002084070020F0FF00008C07002062
:102A700010B5002400BF04E02046FFF743FC601CB3
:102A8000C4B202484078A042F6DC10BD84070020A2
:102A900010B50024044802F0BBF8002800D000E084
:102AA0000124204610BD00000304000010B5074BB0
:102AB00014781C7054785C70054B1960054B1860D5
:102AC00003461833044C236010BD00008407002027
:102AD000880700208C0700209007002010B50446CE
:102AE000012C09D1BA220C21002000F0DFF80121CD
:102AF000022004F0A5F808E000220C21104600F0A6
:102B0000D5F80021022004F09BF810BD10B5002478
:102B100004210848F8F7D6FA552801D1012407E026
:102B2000042000F0E7FF002801D0002400E0012489
:102B3000204610BD2808002010B50446012C09D1FC
:102B4000BA221C21002000F0B1F80121062004F077
:102B500077F808E000221C21104600F0A7F80021B9
:102B6000062004F06DF810BD10B50024062000F01A
:102B7000C1FF002801D0012400E00024204610BD40
:102B800010B50446012C09D1BA221721002000F00B
:102B90008DF80121042004F053F808E000221721E9
:102BA000104600F083F80021042004F049F810BD1D
:102BB00000200449097A002901D0012000E000200A
:102BC00070470000D00C002010B50446022C1CD128
:102BD00000220D21104600F069F8FDF7B5FC002831
:102BE00009D0BA220B21002000F060F801210D204D
:102BF00004F026F847E000220B21104600F056F8BA
:102C000000210D2004F01CF83DE0032C1CD1002213
:102C10000B21104600F04AF8FDF796FC002809D079
:102C2000BA220D21002000F041F801210D2004F00E
:102C300007F828E000220D21104600F037F80021A7
:102C40000D2003F0FDFF1EE0012C0ED1BA220D2154
:102C5000002000F02BF800220B21104600F026F88F
:102C600001210D2003F0ECFF0DE000220D211046A4
:102C700000F01CF800220B21104600F017F800218C
:102C80000D2003F0DDFF10BD10B50024FCF7B6FEEB
:102C9000022801D1022406E0FCF7B0FE012801D190
:102CA000032400E00124204610BD000010B5064BAF
:102CB0001B78834207DD242905D224234343034C98
:102CC00024681B195A5410BD402B0020C80700204F
:102CD00010B574480068407903000BF0B7FB0B0790
:102CE00011D325D35A6D77D38DA8D30007F040FDBB
:102CF0006C4800684079401C6A4909684871CFE017
:102D000069494969087807F0ABFD66480068407971
:102D1000401C644909684871624800684079401C59
:102D2000604909684871BBE000F028F9002811D11A
:102D30007F2007F095FD5B4800684079401C5949A9
:102D400009684871574800684079401C554909682E
:102D500048711DE0534800684078401C514909689B
:102D6000487050480068407803280BD300204D4934
:102D700009684870AA204B490968887003204949AE
:102D80000968C87007F01EFD0020464909684871AF
:102D900086E000F0F3F8002807D142480068407947
:102DA000401C40490968487103E000203D4909681A
:102DB000487107F007FD73E007F0DAFC3948006856
:102DC0004079401C37490968487169E036494969CA
:102DD0000978491CC8B207F043FD324800684079C1
:102DE000401C3049096848712E4800684079401CF1
:102DF0002C490968487153E000F0C0F800280FD151
:102E000007F088FC274909688870012007F0FCFC5E
:102E1000244800684079401C22490968487105E04F
:102E200007F0D0FC00201F490968487138E01D48B0
:102E30000068807818280CD102201A4909680870A7
:102E40000020184909684870042016490968C870AC
:102E500011E0144800684078401C12490968487025
:102E6000104800684078032805D300F027F90020B7
:102E70000C490968487007F0A5FC00200949096859
:102E800048710DE007F09EFC002006490968487172
:102E9000044909684870AA2002490968887000BF7F
:102EA00000BF10BDD0070020402B002010B53148D6
:102EB00000684079002804D001280CD0032848D1AC
:102EC0001DE007F055FC2B4800684079401C29495B
:102ED000096848714BE028490969087807F0C0FC87
:102EE000244800684079401C2249096848712148FB
:102EF00000684079401C1F490968487137E000F0BC
:102F00003DF800280CD101201A49096808700020FA
:102F1000184909684870042016490968C87011E00A
:102F2000144800684078401C1249096848701148EC
:102F300000684078032805D300F0C0F800200D4950
:102F40000968487007F03EFC00200A49096848718A
:102F50000DE007F037FC0020064909684871054973
:102F600009684870AA2003490968887000BF00BF3B
:102F700010BD0000D0070020402B002010B507F046
:102F8000C1FB04461F4800680078002838D01D485F
:102F90000068C078042833D3002C09D100211948D7
:102FA0000068C07A8200174800681430815027E01A
:102FB00014480068C07A81001248006814304058F4
:102FC0001149884211D20F480068C07A81000D482B
:102FD000006814304058401C0A490968C97A8A00C0
:102FE00008490968143188500AE000F067F80021A8
:102FF00004480068C07A820002480068143081509A
:10300000204610BDD0070020B80B000000B587B0E7
:103010000120694608710848029008480390084852
:103020000490084805900848069001A9074800F058
:103030000FF807B000BD000075330100FD4D010021
:10304000D9E50100B9F50100B8F501003C240020E4
:10305000F8B506460F46002400253946304600F0F4
:10306000EFF900BF14E000250EE0002124206043AA
:103070000B4A12688018415524206043094A12689F
:1030800080184155681CC5B2242DEED3601CC4B213
:1030900005480078A042E6DC00F010F8F8BD00001A
:1030A000C8070020CC070020402B00200120024947
:1030B0000968087170470000D007002010B500F0C3
:1030C00073F9002003490968087002490968C8704B
:1030D00010BD0000D007002007480068C07806280F
:1030E00008D105480068C079002803D101200249B1
:1030F0000968C87170470000D007002010B5554816
:103100000068C07803000BF0A1F908671D1A1714B6
:10311000110E056650484068002803D04E484168AB
:103120000020884793E000F0E5F890E000F0C6F852
:103130008DE000F0D1F88AE0FFF7B8FE87E0FFF7F6
:10314000C7FD84E044484068002803D042484168F5
:10315000012088473F480068407C00281AD03E483C
:10316000C068002803D03C48C168C82088470020B8
:10317000384909684862374800680078002804D058
:10318000042034490968C87024E0022031490968E4
:10319000C8701FE02F480068406A401C2D4909682C
:1031A00048622C480068406A7D21C900884211D3DA
:1031B00000202849096848622648006800780028ED
:1031C00004D0042023490968C87003E00220214983
:1031D0000968C8703BE000BF1F484068002803D062
:1031E0001D484168002088471A480068407C002834
:1031F00013D01948C068002803D01748C168C820F8
:103200008847002013490968486212480068C0785E
:10321000401C10490968C87018E00E480068406AF0
:10322000401C0C49096848620A480068406A7D21D0
:10323000C90088420AD30020064909684862054847
:103240000068C078401C03490968C87000BF00BF0F
:1032500010BD0000D0070020402B002010B51548FD
:103260000068C078072824D00120124909684874F2
:1032700008E011488068002802D00F49886880471C
:10328000FFF73CFF0B480068C0780628F1D10948D9
:103290000068007A0028ECD106480068C079002850
:1032A000E7D104480068807A0028E2D10149096822
:1032B000487410BDD0070020402B002010B50548F1
:1032C00000680078012802D1FDF732FF01E0F6F72F
:1032D0000FFA10BDD007002010B50548006800782F
:1032E000012802D1FEF750F901E0F6F7DFFD10BD2D
:1032F000D007002010B51D480068807A002829D129
:103300001A480068007A002803D00220174909688B
:10331000887216480068C079002803D0012013493C
:1033200009688872114800680079012812D10020CC
:103330000E49096808710D490968887207200B4910
:103340000968C8700A484068002803D008484168E6
:1033500000208847054800680078012802D1FEF760
:10336000EDF901E0F6F77CFE10BD0000D00700206B
:10337000402B002010B504462146084801F064FCAB
:1033800007480078002805D1002C03D032210548D9
:10339000FCF798FE0248047010BD00000103000015
:1033A0000401002050C3000000202449096848702F
:1033B000AA202249096888700020204909684862CB
:1033C0001E49096808711D49096848711B49096847
:1033D00088711A490968C87118490968087217493B
:1033E0000968887215490968C87214490968087320
:1033F00024201249096848731049096888730F49E5
:103400000968C87300200D49096808740B490968E8
:1034100048740A490968887408490968C8740749E2
:103420000968486100210548006881610348006817
:10343000C16102480068016270470000D0070020A7
:1034400010B50A780D4B1860034628330C4C2360E6
:1034500024235343044628341B190A4C23600A4C86
:103460004B6863608B68A360CB68E3604B69636102
:103470000B6923610B78237010BD0000D00700207A
:10348000C8070020CC070020402B00200748006818
:10349000C078062808D105480068007A002803D1C2
:1034A000012002490968087270470000D007002017
:1034B00010B50446012C09D1BA2220210020FFF7C3
:1034C000F5FB0121084603F0BBFB08E000222021A8
:1034D0001046FFF7EBFB0021012003F0B1FB10BD0C
:1034E00010B50024032000F005FB002801D00124C2
:1034F00000E00024204610BD10B50446032C0ED178
:10350000BA2215210020FFF7D1FB0022142110461A
:10351000FFF7CCFB01210E2003F092FB39E0022CD7
:103520001CD1FDF711F8002809D0BA22142100207F
:10353000FFF7BCFB01210E2003F082FB08E0002214
:1035400014211046FFF7B2FB00210E2003F078FB98
:10355000002215211046FFF7A9FB1AE0012C0ED11D
:10356000BA2214210020FFF7A1FB01210E2003F055
:1035700067FB002215211046FFF798FB09E00022A7
:1035800015211046FFF792FB002214211046FFF789
:103590008DFB10BD10B50024F9F72EF909498842BA
:1035A0000DD3FDF735F8002807D1FCF743FF0128BC
:1035B00001DD032404E0022402E0022400E00124EF
:1035C000204610BDB80B000010B50446012C09D1EF
:1035D000BA221D210020FFF769FB0121002003F022
:1035E0002FFB08E000221D211046FFF75FFB0021A2
:1035F000084603F025FB10BD10B50024022000F0A2
:1036000079FA002810D00124104800780A2805DA39
:103610000E480078401C0D49087015E00A200B493F
:103620000870002048700FE00024084840780A28FD
:1036300005DA06484078401C0449487004E00A2036
:103640000249487000200870204610BD200100206B
:1036500010B50446012C09D1BA221E210020FFF723
:1036600025FB0121092003F0EBFA08E000221E21CE
:103670001046FFF71BFB0021092003F0E1FA10BD03
:1036800070B5002400250026FCF7E2FD0546FCF796
:10369000EBFD064602210848F7F714FD552800D136
:1036A00008E0012E01D1002404E0012D01D1012404
:1036B00000E00024204670BD2808002010B5044614
:1036C000012C09D1BA221F210020FFF7EFFA0121B6
:1036D000082003F0B5FA08E000221F211046FFF78A
:1036E000E5FA0021082003F0ABFA10BD70B5002503
:1036F0000024FCF7E5FD044603210C48F7F7E2FC43
:10370000552803D101200A4908800AE0762C03DA03
:1037100001200749088004E0782C02DB00200449DE
:10372000088003480588284670BD0000280800204E
:103730002201002010B50446012C09D1BA22212112
:103740000020FFF7B3FA0121072003F079FA08E01F
:10375000002221211046FFF7A9FA0021072003F0DB
:103760006FFA10BD10B50024FCF776FE002801D1D9
:10377000012400E00024204610BD10B50446012CB1
:1037800009D1BA2216210020FFF790FA0121032067
:1037900003F056FA08E0002216211046FFF786FAD9
:1037A0000021032003F04CFA10BD10B500240520C1
:1037B00000F0A0F9002801D0012400E000242046F8
:1037C00010BD10B50446012C09D1BA2219210020E0
:1037D000FFF76CFA0121052003F032FA3CE0022CDD
:1037E00017D1FCF7B1FE002809D0BA221921002018
:1037F000FFF75CFA0121052003F022FA2CE00022F9
:1038000019211046FFF752FA0021052003F018FA9B
:1038100022E0032C17D1FCF79DFE002809D0BA2224
:1038200019210020FFF742FA0121052003F008FAD0
:1038300012E0002219211046FFF738FA0021052076
:1038400003F0FEF908E0002219211046FFF72EFAD6
:103850000021052003F0F4F910BD000010B500248C
:10386000FCF72EFE01282FD104211948F7F72AFC76
:10387000552801D1012428E0FCF702FD01280BD0D6
:10388000FCF7FEFC022807D0FCF7FAFC032803D063
:10389000FCF7F6FC052801D1012416E0FCF7F0FC4A
:1038A000042801D1022410E0FCF7EAFC062801D12B
:1038B00003240AE0FCF7E4FC002803D0FCF7E0FC5A
:1038C000072802D1002400E00024204610BD00009B
:1038D0002808002010B50446012C0ED1BA221B2165
:1038E0000020FFF7E3F900221A211046FFF7DEF966
:1038F00001210A2003F0A4F91EE0022C0ED1BA2205
:103900001A210020FFF7D2F900221B211046FFF7F1
:10391000CDF901210A2003F093F90DE000221A21CC
:103920001046FFF7C3F900221B211046FFF7BEF92E
:1039300000210A2003F084F910BD10B50024FCF723
:10394000D3FE012801D1012400E00224204610BD4D
:1039500010B5F8F76BFF0446204610BD10B5034BB9
:1039600007220349034800F013F910BD5139010043
:1039700064F501000424002070B506465C488068A8
:10398000002804D05A4988688047054600E0002591
:103990000024A6E0564841680C206043081840887F
:1039A000A84207D0524841680C206043081840885C
:1039B00002287DD14E4841680C2060430818806879
:1039C00000280CD04A494A680C2161435118886884
:1039D000804747490968E2008918487009E044486F
:1039E00041680C206043095C41480068E20080188F
:1039F00041703F480068E100401840783C49096840
:103A0000E200895C88420FD039480068E100401824
:103A1000417837480068E200815400203449096841
:103A2000E200891848605AE031480068E100401817
:103A300041782F4842680C2060431018407881423A
:103A40001FD12B480068E1004018416828484268AF
:103A50000C2060431018808881420BD824480068ED
:103A6000E10040184068801921490968E20089187E
:103A7000486034E001201E490968E2008918488046
:103A80002DE01B480068E100401841681848426872
:103A90000C2060431018C08881420DD8144800687B
:103AA000E10040184068811911480068E20000E018
:103AB00009E08018416012E000200D490968E20029
:103AC000891848800BE0002009490968E20089183C
:103AD0004880002106480068E20080184160601CB0
:103AE00084B203488089A04200DD53E770BD000026
:103AF000F82A00200146064A92898A4205DD044AD6
:103B00001268CB00D218508800E0002070470000F7
:103B1000F82A0020002000BF14E00D494A680C215B
:103B200041435118498801290AD10021084A1268E5
:103B3000C300D2185180064A1268C300D2185160DF
:103B4000411C88B2024989898142E6DC7047000045
:103B5000F82A0020002000BF13E00C494A680C211D
:103B6000414351184988002909D1084A1268C30005
:103B7000D2185180054A1268C300D2185160411C06
:103B800088B2024989898142E7DC7047F82A00201F
:103B9000F0B504460020164DAB6069602C60AA8128
:103BA00000BF1FE0124D6E680C254543755D104E39
:103BB0003668C700F61975700D4D6E680C254543C3
:103BC000755D0B4E3668C700F5550025084E366802
:103BD000C700F6197580064E3668C700F61975607D
:103BE000451CA8B2024DAD898542DBDCF0BD00006A
:103BF000F82A002070B505460E46002E05D0314645
:103C00002846F4F79DFA044600E02C46204670BD95
:103C100010B5FCF721FC00280DD1074800780128D9
:103C200009D005480078032805D00448007800280A
:103C300001D1F9F7D7FA10BDF0000020EF00002005
:103C40000120054988710020044908700449087062
:103C50000449087070470000E8000020EF000020D1
:103C6000F1000020F2000020002003490871487193
:103C70000120887170470000E800002070B5049CA6
:103C80002578914216DD01280AD18D4206DAFF26F9
:103C9000F61AAE420ED3EE18F5B20BE0154609E067
:103CA000022807D1954204DD9D4203DBEE1AF5B2EE
:103CB00000E00D46257070BD0D4A41685160816974
:103CC0009161C168D160416A5162016A1162016803
:103CD00011604169516181689160C169D161016977
:103CE0001161816A91620021024A117070470000DF
:103CF000142B0020C407002010B5FFF70BFFF8F7C6
:103D000015FC00210148F7F7DDFA10BD340800204A
:103D100010B5F8F70BFCFFF71DFF08F073FC08F077
:103D20000FFDFBF717FDFAF749FAFFF789FFF8F7E0
:103D3000FDFFF7F7CDF855210148F7F7C3FA10BD9D
:103D4000340800201CB500202F49087006F0C0FC84
:103D50000020FCF75BFD0AF0A1FEF7F7B1FD55214D
:103D60002A48F7F7AFFAF8F719FEF6F7CBFCF6F7A3
:103D700049FFE12040020AF0D3FA00F05DFAF7F7BC
:103D8000A7F806F089FEF8F7D1FBFAF715F8F9F76E
:103D900059F8F8F7D7FFFFF7E1FDFEF7D3F8FFF783
:103DA00035F9FFF75BFAF9F71FFFFBF7FFFCFAF7AE
:103DB00005FA174AFF219131012008F089FD002200
:103DC0001146012008F0C8FC08F002FC08F0B8FC1D
:103DD000FFF74AFFF9F7C2FC00200E4988714871CD
:103DE0000871012088704870142008700722684606
:103DF000F4F73DFA0199009800F076FF02210120C6
:103E000000F052FE1CBD0000030100203408002019
:103E10000090D003140100207047000010B5044644
:103E2000552C03D105494869804702E003490868D9
:103E3000804700200249087010BD0000142B0020AC
:103E4000C407002010B54648007803000AF0FEFAC7
:103E50000A06111B26303B46505173814148406889
:103E6000002802D03F494868804701203C4908703B
:103E700000BF3C488068002804D03A4988688047E1
:103E80003749087069E03748C068002802D03549D2
:103E9000C868804703203249087000BF3148006974
:103EA000002804D02F49086980472D49087054E044
:103EB0002C484069002802D02A49486980470020E0
:103EC0002749087049E027488069002802D0254921
:103ED0008869804706202249087000BF2148C069D0
:103EE000002804D01F49C86980471D49087034E084
:103EF00000BF1B48007807280AD11A48006A00282A
:103F000002D01849086A804709201549087011E055
:103F10001348007808280AD11248406A002802D0C5
:103F20001049486A804709200D49087002E00020C6
:103F30000B49087000BF0A480078002808D00948DB
:103F4000806A002804D00749886A804704490870BD
:103F500003E000200249087000BF00BF10BD000050
:103F6000C4070020142B00207047000010B500206B
:103F70000AF050FE07F056FC07F0AAFC07F0C0FC60
:103F800000F086FCF6F7CEFE0220FCF73FFC002096
:103F900007490870FFF762F9FFF788F8FFF7AEF8F6
:103FA000F6F720FD102009F0A9F800F071FD10BD12
:103FB0009C01002010B5012407F016F8012801D15A
:103FC000052407E0F8F712FC0349884201D20124D6
:103FD00000E00224204610BD204E000010B506244B
:103FE00007F002F8002800D1002407F003F80128A8
:103FF00003D006F0FFFF072800D90924204610BD92
:1040000010B5F6F78FFE00221146012008F0D6FC0D
:1040100000213A48F7F756F9002400BF00F0EEFE01
:1040200032217D200001FCF74DF800203449087052
:104030000AE00022324801781046FEF737FE304889
:104040000078401C2E4908702D4800782428F0DBA9
:1040500000202C49087009E000212A48007808F067
:10406000BFF828480078401C264908702548007889
:104070000D28F1DBFFF742F8F6F78AFB06F006FFA2
:1040800021480078401C204908700846007805281F
:1040900012D300200870FFF71FF81C4800780A2888
:1040A00005D3002019490870FFF7F0F904E017481C
:1040B0000078401C1549087006F09CFF0128ADD916
:1040C00006F098FF0728A9D200200E49087008E0E2
:1040D0000C48007808F09EF80A480078401C09490E
:1040E0000870084800780D28F2DBF6F78BFD5521A3
:1040F0000248F7F7E7F8204610BD0000340800201A
:104100001D0100201B0100201C0100201E010020B9
:1041100010B5032408E000F071FE012000F078FDE6
:10412000002801D0042400E0F5E700BF204610BDC0
:1041300010B500202449086006F0CAFA0120FCF7F7
:1041400065FBF7F7BDFB55212048F7F7BBF80AF0F0
:10415000A5FCF6F7D7FAF9F7F7FDF6F753FD06F0E9
:10416000A5FEF9F729FEFAF711F8F8F76BFEFFF74D
:10417000F5FBFDF7E7FEFFF7EDFCFFF761FDFEF74E
:1041800045FFFFF76BF800F057F8E12040020AF016
:10419000C7F8F6F79DFEFBF709FBFAF70FF80C4A94
:1041A000FF219131012008F093FB002211460120EC
:1041B00008F0D2FA08F00CFA08F0C2FA0221012045
:1041C00000F072FC10BD00005000002034080020F8
:1041D0000090D00370B506460D4614460E480660A2
:1041E0000E4805600E49206808600E496068086046
:1041F0000D49A06808600D49206908600C49E06815
:1042000008600C496069086005480068002802D011
:1042100003480068804770BDC4000020CC00002027
:10422000AC000020B0000020B4000020B800002046
:10423000BC000020C000002000B587B00C480190F1
:104240000C4802900C4803900020049005900B4805
:10425000069000200A49086048600A4908604860E2
:1042600001AA0121C9020848FFF7B4FF07B000BD49
:104270008D420100D54501005D450100E544010086
:10428000E4140020DC0C0020EC1900200120704711
:10429000F3B5C3B00446449E0020009057E002E00E
:1042A000641C761E00BF022E05D32078EB28F7D1C0
:1042B00060789028F4D1072E00D24AE0A778FD1C40
:1042C000B54200D945E0A81E205C0002691E615C71
:1042D00008434290042D38D9291FA01C0AF0F8FB8E
:1042E0004299884226D11D480068002804D0B91E92
:1042F000E01C1A4A1268904719480068002824D028
:10430000E178684601712079811168464171207910
:104310008106890E68468171381FC1B26846C17135
:10432000C279611D02A8F3F7A2FF01A80C49096830
:1043300088470AE00020009002E00098401C0090AE
:104340000098A842F9D3002000906419761B072E2C
:10435000A5D200BF4498801B45B0F0BDB800002036
:10436000C0000020F7B5C0B0154600260027E81DA4
:10437000FF210131884202DD002043B0F0BDEB2176
:104380006846017090214170281DC1B26846817055
:104390000021C1704098C1B2684601710524002611
:1043A00005E04198805D69460855641C761CAE4264
:1043B000F7DBA11E00A802300AF08AFB87B2381290
:1043C00069460855641C0F55641C0648006800289F
:1043D00005D021466846034A12689047CDE7002081
:1043E000CBE70000B000002070B5002400250026B7
:1043F0001B4840681A490968884200D170BD1848B6
:10440000406817490968884205D915484068144929
:104410000968451A07E01248006811494968401ABE
:10442000012189020D1AFF2D01D9FF2600E02E4639
:1044300000240DE00A4801680830405C094908552D
:1044400007480088401C8005800D05490860641CF1
:10445000B442EFD3B1B2034809F0BEFF00BFCDE7CD
:10446000E4140020EC18002070B500251A480068FC
:10447000002830D0194A1288FF230133991A184AAC
:104480001268164B1B88D018134A126890470546CD
:10449000002D20D011480088401910490880084696
:1044A00001880F480068FFF7F3FE0446002C0DDD7D
:1044B0000A480088844209DA08480088021B084834
:1044C0000068011906480068F3F7D1FE0348008828
:1044D000001B0249088070BDB4000020C800002005
:1044E000C400002010B50446A07810280CD1207913
:1044F000194908700846007801282BD1002211467E
:104500002020FFF72FFF25E0A078122803D1207983
:10451000114908721EE0A07801281BD120793328A8
:1045200003D101200C49487005E02079352802D1DB
:10453000002009494870607907498870607A000650
:10454000217A09040843E17909020843A179084363
:104550000149486010BD0000D00C002070B5034632
:104560000022002400251A484068194E3668B042DF
:1045700001D1002070BD16484068154E3668B04223
:1045800005D913484068124E3668841B07E010486E
:1045900000680F4E7668801B0126F602341AA1428D
:1045A00001D9254600E00D4600220CE008480668C7
:1045B0000830805D985406480088401C4005400D36
:1045C000034E3060521CAA42F0D32846D2E70000C6
:1045D000DC0C002070B5034600220024154840681A
:1045E000144D2D68A84208D312484068114D2D681B
:1045F000401B0125AD022C1A04E00E4800680D4D49
:104600006D68441BA14201D9012070BD00220CE05D
:104610009D5C084846680830855508388088401CED
:104620008005800D034D6860521C8A42F0D3002043
:10463000EBE70000E414002010B50248FFF73CFB54
:1046400010BD000040F601000021014A11757047BD
:1046500040600040014600BFF020084000110A23DE
:10466000584302460807000F8018C0B27047014641
:10467000002204E0501CC2B208460A38C1B20A291E
:10468000F8DA1007000E08437047000010B5044622
:1046900001218020F6F7A0FE607A012805D142486A
:1046A000C078102108434049C870607AA22805D11B
:1046B0003E48007F802108433C490877607A3B49A7
:1046C000087700203A4948770846407F2178084318
:1046D00037494877E07B002805D00846407F2021F5
:1046E0000843334948773248407FC008C000A17A68
:1046F00008432F4948770846807FF72108402C4916
:104700008877E078FFF7B3FF29498874A078FFF72E
:10471000AEFF2749C8746078FFF7A9FF24490875E0
:104720002078002805D10846007D217908432049DA
:104730000875E079FFF79BFF1D4988756079FFF7E1
:1047400096FF1B494875A079FFF791FF1849C87576
:10475000207AFFF78CFF164908760846807F4006CE
:10476000400E8877E07A002806D00846807F4021F6
:1047700008430F49887703E00D48807F0C4988770C
:10478000A07BFFF774FF0A498876607BFFF76FFF15
:104790000749C876207B08770846807F1021884328
:1047A0000349887710BD00002004024060040440E3
:1047B000404F044010B504461B48807F0121084348
:1047C000194988772078FFF752FF174908756078F4
:1047D000FFF74DFF1449C874A078FFF748FF12494E
:1047E000887420780C2806DD0846407F082108439D
:1047F0000D49487709E00C48407F0B494877084647
:10480000007DE1780843084908750748807F400823
:1048100040000549887700BF0348807F0221084097
:104820000028F9D110BD0000404F044010B5002011
:1048300014490876162009F02FFE0021124801764F
:104840001248407F80210843104948770846807FFE
:10485000012108430D49887700BF0C48807F022161
:1048600008400028F9D00948807F400840000749E7
:10487000887700BF0548807F022108400028F9D1D1
:1048800010BD00004060004040610040404F0440C7
:1048900010B500200749087000212020F6F79CFD84
:1048A000012105480175002004490875152009F00B
:1048B000DBFD10BD005004404061004040600040FE
:1048C00070B504460D46002C14D0002D12D0042DD6
:1048D00010D800F013F800280CD1002608E0064993
:1048E000885D22460121F4F741FDA41C701CC6B26C
:1048F000AE42F4DB70BD00008401002000200549B9
:10490000897DC907C90F002901D0012000E00020DE
:10491000704700000050044030B585B005460C4695
:10492000002003900490009001900290072C0BDC73
:104930000120A04081B2684681810121C17303A991
:104940000220FBF76DF83EE0082C01D0092C0BD1BA
:104950000120A04081B2684681810121C17303A971
:104960000120FBF75DF82EE00A2C03D00B2C01D0C0
:104970000D2C0BD10120A04081B26846818101211C
:10498000C17303A90020FBF74BF81CE00C2C01D0ED
:104990000F2C0BD10120A04081B2684681810121FA
:1049A000C17303A90E20FBF73BF80CE00E2C0AD1D3
:1049B0000120A04081B2684681810121C17303A911
:1049C0000C20FBF72DF8002168460170C170417082
:1049D0000121817000210171C1720D218172FF21BD
:1049E000017200214172F4F721FD03491520FDF702
:1049F00073F905B030BD00004946010010B5002034
:104A000010490875152009F02FFD00210E48017589
:104A10001520002809DB00BF00BFC206D20E01210D
:104A200091400A4A116000BF00BF00BF084880796A
:104A30008011032805D006480078802108430449E6
:104A4000087010BD406000404061004000E100E09F
:104A50000050044010B5F4F7E3FD10BD10B501237C
:104A60001A4600211846F6F773FC0122114610463B
:104A7000F6F7E4FCF6F7D0FC03480AF001F8024828
:104A80000249086010BD00000090D00348070020D4
:104A900000BF04480069042108430249086130BF8F
:104AA00000BF704700ED00E0F3B585B0054600207B
:104AB00003900490EEB22804070E0F2F54DA082E4C
:104AC00052DA002009E00C214143284A515AA942F8
:104AD00001D1044603E0411CC8B21728F3D300BF3C
:104AE0000120B04086B20C20604320494018C378B2
:104AF0000C20604340188278F8B231460190FBF7F1
:104B000033F868468681012181730021C173022137
:104B10004174F8B203A9FAF783FF0C216143134AE9
:104B20008918C888FBF798FF0C2060430F4940188C
:104B3000C1886846018169460698887202A8FBF719
:104B4000A5FE0C226243094BD21891680C226243E5
:104B5000D21804201056FDF7BFF80C216143034A18
:104B60008918C888FBF7FCFE07B0F0BDD4F7010038
:104B7000FEB505460C460020C0430290EFB2280463
:104B8000060E0F2E42DA082F40DA0120B84069469F
:104B9000088080202040002816D101208870A007BE
:104BA000800F022801D1487109E0A007800F012879
:104BB00002D16946487102E0002069464871F0B2AE
:104BC0006946FAF72DFF1FE00020694688700E2025
:104BD0002040002800D000BF10202040002802D133
:104BE0006946087102E0012069460871E007C00FBC
:104BF000002802D16946887102E001206946887167
:104C0000F0B26946FAF70CFF002002900298FEBD50
:104C100030B50146CAB20C04230E00200F2B0FDA68
:104C2000082A0DDA01249440A2B2064C03252D0275
:104C30006419E45C1440002C01D0012000E0002045
:104C400030BD000000000440F8B504460F460020C7
:104C5000C0430090E6B22004050E0F2D11DA082E95
:104C60000FDA0120B04086B2002F04D1E8B23146FD
:104C7000FAF7D2FF03E0E8B23146FAF7DDFF002091
:104C800000900098F8BD00001649897F0122114369
:104C9000144A917700BF1349897F022211400029ED
:104CA000F9D01049897C81700E49C97C41700D4949
:104CB000097D01700B498A7D8271497D0171094925
:104CC000CA7D42710A7EC271897F49084900054A3E
:104CD000917700BF0349897F022211400029F9D151
:104CE00070470000404F044003B585B0002001909C
:104CF000029003900490002168464173817E01A8D0
:104D0000C1706846417E01A881706846017E41718C
:104D1000002101A80171082168460171817D01A867
:104D2000C1716846C17D4172417D01A881716846AB
:104D3000017D01A80172002168468173C17301A839
:104D400081730C2141734121684601740021C174B3
:104D500001A8FFF79BFC1A20044988820449162009
:104D6000FCF7BAFF00F006F807B000BD204F044082
:104D7000CDEB010010B5FFF759FD10BD70B504462D
:104D80000D46601E0D49884200D90124002C00D137
:104D9000012440200A490870084600786043094908
:104DA00048610321081F09F08FFB00200549886135
:104DB000072008610448056070BD0000FFFFFF0088
:104DC0007401002000E000E0700100200020C043DA
:104DD000002809DBC206D20E01219140054A11606C
:104DE000BFF34F8FBFF36F8F00BF002002490861F0
:104DF0008861704780E100E000E000E010B509F054
:104E000009FB10BD1A20084908722B2048723C206B
:104E100088724D20C8727F20044909680860AC2060
:104E200003494870704700000004024078010020E8
:104E30000010024000B518480078012812D1174828
:104E40000078642809DB02201549487108710020A8
:104E5000124908701049087004E010480078401C9E
:104E60000E4908700F480078012814D10E480078C8
:104E7000012804D100200C4908700C4908700B4827
:104E80000078322802DBF7F7D1FD04E0074800780C
:104E9000401C0649087000BD1907002018070020B3
:104EA0000807002012070020140700201307002025
:104EB000F8B504460D4600270020009003200003AB
:104EC000204000130090102C04D0122C02D0114866
:104ED000844217D122202840222806D127073F0FDD
:104EE00039460098F5F7FAFB0646122028401228AA
:104EF0000ED12007000F471C39460098F5F7EEFB4E
:104F0000064605E02107090F0098F5F7E7FB06467E
:104F10003046F8BD10100000F8B504460D460026D6
:104F200000270120000320400713102C04D0122C6E
:104F300002D00F48844215D122202840222805D1D2
:104F40002607360F31463846FAF768FA122028400D
:104F500012280CD12007000F461C31463846FAF7BC
:104F60005DFA04E02107090F3846FAF757FAF8BD51
:104F700010100000FFB58BB01C4600200790069073
:104F800005903848049010210B980840002801D063
:104F9000022707E040210B980840002801D0012794
:104FA00000E00027002C04D0149804700120089021
:104FB00001E010200890002548E0002C08D025468C
:104FC0006000294A115A0C98F3F7BAF8079006E0E6
:104FD0006800254A115A0C98F3F7B2F807903E463C
:104FE00030E0711C0798F3F7ABF8400806900D9875
:104FF000F3F7FCF903900D9A0699881AF3F7F6F97E
:1050000018490190F3F777F902900399F3F7B0F993
:1050100005900598F3F7F1F94900490803910290CA
:105020000498F3F7EAF94900490801910090039BBD
:10503000029AF3F7F7F903D20A95099605980490B6
:10504000701CC6B27F2ECCDD681CC5B208988542A4
:10505000B3DB14990A980870149909984870049859
:105060000FB0F0BD0000C842E8F801000246412A36
:105070002ED010DC212A2AD006DC102A45D0122A94
:105080004BD0202A59D11CE0222A26D0232A2AD00C
:10509000402A52D116E081235B01D01A9A4228D0CF
:1050A00008DC422A1AD0432A1ED0254810180028AE
:1050B00043D13AE0012822D020281BD021283CD11E
:1050C0001EE000BF1F4803890B43038136E000BF89
:1050D0001C4843890B43438130E000BF1948838952
:1050E0000B4383812AE000BF1648C3890B43C38169
:1050F00024E000BF144883880B4383801EE000BF78
:105100001148C3880B43C38018E00E4843890B4302
:10511000438103890B43038110E00A48C3890B4391
:10512000C38183890B43838108E00748C3880B430D
:10513000C38083880B43838000E000BF00BF7047BB
:10514000F0EFFFFF0011044000140440F0B50546E5
:105150000E46412D30D010DC212D2CD006DC102D38
:1051600051D0122D56D0202D62D11CE0222D2AD0F4
:10517000232D30D0402D5BD116E081214901681AE2
:105180008D4230D008DC422D1ED0432D24D02A4839
:10519000281800284CD144E001282CD0202823D006
:1051A000212845D128E000BF244F3888314600F03F
:1051B00049F804463DE000BF204F7888314600F0B2
:1051C00041F8044635E000BF1C4FB888314600F076
:1051D00039F804462DE000BF184FF888314600F03A
:1051E00031F8044625E000BF154F3888314600F0FD
:1051F00029F804461DE000BF114F7888314600F0C1
:1052000021F8044615E00D4F7888314600F01AF871
:1052100004460EE0094FF888314600F013F80446C2
:1052200007E0074F7888314600F00CF8044600E0AC
:1052300000BF00BF2046F0BDF0EFFFFF00110440AB
:10524000001404400246002013460B40002B01D0FE
:10525000012000E000207047FFB581B00E461746E0
:10526000012F07D1F748407D00090001C01DF54915
:10527000487505E0F348407D00090001F149487593
:10528000049801287ED10A210198F2F759FF0546BA
:10529000ED48445DE007C00F002807D0E948007CD6
:1052A00000090001C01DE749087405E0E548007CDD
:1052B00000090001E349087402202040002807D0BB
:1052C000E048C07BF02188437030DE49C87305E0B8
:1052D000DC48C07BF0218843DA49C87304202040B1
:1052E000002807D0D748807C00090001C01DD5499F
:1052F000887405E0D348807C00090001D149887496
:1053000008202040002807D0CE48407CF021884368
:105310007030CC49487405E0CA48407CF02188438D
:10532000C849487410202040002807D0C548407C58
:1053300000090001C01DC349487405E0C148407C14
:1053400000090001BF49487420202040002807D0F0
:10535000BC48007CF02188437030BA49087405E0ED
:10536000B848007CF0218843B649087440202040AA
:10537000002808D0B348807CF02188437030B149C0
:10538000887406E08BE0AF48807CF0218843AD490B
:1053900088740A210198F2F7D3FE0D46AA48445DAD
:1053A000E007C00F002807D0A648807BF021884383
:1053B0007030A449887305E0A248807BF0218843BF
:1053C000A049887302202040002807D09D48807B98
:1053D00000090001C01D9B49887305E09948807B46
:1053E000000900019749887304202040002807D055
:1053F0009448007DF021884370309249087505E09B
:105400009048007DF02188438E490875082020408F
:10541000002807D08B48007D00090001C01D894984
:10542000087505E08748007D000900018549087579
:1054300010202040002807D08248C07CF0218843FB
:1054400070308049C87405E07E48C07CF0218843F4
:105450007C49C87420202040002807D07948C07BB0
:1054600000090001C01D7749C87305E07548C07B7D
:10547000000900017349C87340202040002807D06C
:105480007048C07C00090001C01D6E49C87454E01A
:105490006C48C07C000900016A49C8744DE0694845
:1054A000007C00090001674908740846C07BF021B0
:1054B00088436449C8730846807C000900018874E9
:1054C0000846407CF02188435E4948740846407C89
:1054D0000009000148740846007CF02188435949BE
:1054E00008740846807CF021884356498874084631
:1054F000807BF0218843534988730846807B0009EC
:10550000000188730846007DF02188434D490875E5
:105510000846007D0009000108750846C07CF0219E
:1055200088434849C8740846C07B00090001C87315
:105530000846C07C00090001C8740A9801287DD182
:105540000A213046F2F7FCFD05463F48445DE0077E
:10555000C00F002807D03B48407B00090001C01D58
:105560003849487305E03748407B00090001354958
:10557000487302202040002807D03248007BF021E9
:10558000884370302F49087305E02E48007BF021D6
:1055900088432C49087304202040002807D029485C
:1055A000807DF021884370302649887505E02548C4
:1055B000807DF021884323498875082020400028F9
:1055C00007D02048807D00090001C01D1D49887555
:1055D00005E01C48807D000900011A4988751020EB
:1055E0002040002807D01748407DF02188437030C4
:1055F0001449487505E01348407DF021884311495E
:10560000487520202040002807D00E48407BF0211C
:10561000884370300B49487305E00A48407BF0210D
:105620008843084948734020204000280ED0054890
:10563000C07D00090001C01D024900E092E0C8756C
:105640000AE00000EC21002038F301006D48C07D25
:10565000000900016B49C8750A213046F2F770FD58
:105660000D466948445DE007C00F002807D0654833
:10567000C07AF021884370306249C87205E0614801
:10568000C07AF02188435F49C87202202040002878
:1056900007D05C48C07A00090001C01D5949C87292
:1056A00005E05848C07A000900015649C872042034
:1056B0002040002807D05348407E00090001C01D4B
:1056C0005049487605E04F48407E000900014D49A9
:1056D000487608202040002807D04A48007EF02164
:1056E000884370304749087605E04648007EF0213F
:1056F00088434449087610202040002807D04148BC
:10570000007E00090001C01D3E49087605E03D48C5
:10571000007E000900013B49087620202040002837
:1057200007D03848007B00090001C01D35490873C7
:1057300005E03448007B000900013249087340202D
:105740002040002807D02F48C07DF02188437030CA
:105750002C49C87554E02B48C07DF0218843294965
:10576000C8754DE02748407B000900012549487372
:105770000846007BF0218843224908730846807D53
:10578000F02188431F4988750846807D0009000183
:1057900088750846407DF02188431A4948750846B7
:1057A000407BF0218843174948730846C07D0009B3
:1057B0000001C8750846C07AF02188431149C872B3
:1057C0000846C07A00090001C8720846407E0009F8
:1057D000000148760846007EF02188430949087692
:1057E0000846007E0009000108760846007B000993
:1057F000000108730846C07DF02188430149C8753F
:1058000005B0F0BDEC21002038F30100FFB581B0F8
:105810000E461746019801287ED10498002828D109
:10582000FB480078012824D0F6F7E6FFF9498842C2
:105830001FD3FAF789FE00280DD0F748807DF021AC
:1058400088437030F44988750846C07C000900011F
:10585000C01DC8741AE0F048807DF02188431030E4
:10586000ED4988750846C07C00090001401CC874D9
:105870000CE0E948807DF02188437030E649887566
:105880000846C07C00090001C01DC874E248C07C05
:10589000F02188437030E049C8740846007EF0214A
:1058A00088437030DC4908760846807D0009000195
:1058B000401C88750846407DF02188431030D64949
:1058C00048750846407D00090001401C487508469F
:1058D000007DF02188431030CF4908750846007DCF
:1058E00000090001401C0875330008F0AFFD062ECA
:1058F000261E140C042FC848007D00090001C01D9D
:10590000C549087500BFC448007DF0218843703048
:10591000C149087500BF00E0AFE1BF48407D000904
:105920000001C01DBC49487500BFBB48407DF02147
:1059300088437030B849487500BFB748807D00097A
:105940000001C01DB449887500BF00E000BF00BF62
:10595000049800285ED1AE48007801285AD0F6F7A6
:105960004BFFAC49884255D3AB48C07FF0218843F8
:10597000A949C8770846807F000900018877084652
:10598000407FF0218843A44948770846007FF021F2
:105990008843A14908770846C07DF02188439E4985
:1059A000C8750846C07F00090001C8770846807F97
:1059B000F0218843984988770846407F0009000114
:1059C000C01D48770846807EF0218843924988763A
:1059D0000846807E0009000188760846407E00095E
:1059E000000148760846007E000900010876084656
:1059F000007F0009000108770846C07EF021884337
:105A00008549C8760846407EF02188437030824937
:105A10004876B8E164213846F2F792FB0546012D3D
:105A200007D17D48C07FF021884370307A49C8771C
:105A300005E07948C07FF02188437749C8770A217B
:105A40003846F2F77DFB0A210090F2F779FB0D460C
:105A5000642F02D37148445D01E07148445DE00762
:105A6000C00F002807D06C48807F00090001C01DCE
:105A70006949887705E06848807F00090001664928
:105A8000887702202040002807D06348407FF0211B
:105A9000884370306049487705E05F48407FF021D7
:105AA00088435D49487704202040002807D05A48A1
:105AB000007FF021884370305749087705E0564849
:105AC000007FF021884354490877082020400028AF
:105AD00007D05148C07DF021884370304E49C875C9
:105AE00005E04D48C07DF02188434B49C875102022
:105AF0002040002807D04848C07F00090001C01D91
:105B00004549C87705E04448C07F00090001424983
:105B1000C87720202040002807D03F48807FF02110
:105B2000884370303C49887705E03B48807FF0210E
:105B300088433949887740202040002807D03648DC
:105B4000407F00090001C01D3349487705E0324815
:105B5000407F00090001304948770A213846F2F7B2
:105B6000EFFA0D462D48445DE007C00F002807D02E
:105B70002948807EF021884370302749887605E0E7
:105B80002548807EF02188432349887602202040E2
:105B9000002807D02048807E00090001C01D1E4952
:105BA000887605E01C48807E000900011A49887645
:105BB00004202040002807D01748407E000900013B
:105BC000C01D1549487605E01348407E00090001D4
:105BD0001149487608202040002807D00E48007E52
:105BE00000090001C01D0C49087605E00A48007E46
:105BF000000900010849087610202040002811D033
:105C00000548007F00090001C01D034908770FE027
:105C100003010020B80B0000C022002038F301006F
:105C20004BF301005948007F0009000157490877EC
:105C300020202040002807D05448C07EF02188430F
:105C400070305249C87605E05048C07EF021884344
:105C50004E49C87640202040002807D04B48407E5F
:105C6000F02188437030494948768CE04748407EAF
:105C7000F02188434549487685E04448807D000905
:105C80000001424988750846407DF02188433F491C
:105C900048750846407D0009000148750846007DAA
:105CA000F0218843394908750846007D0009000144
:105CB00008750846C07C00090001C8740846807D4C
:105CC000F0218843314988750846C07CF02188431B
:105CD0002E49C8740846007EF02188432B49087677
:105CE0000846C07FF02188432849C8770846807F4E
:105CF0000009000188770846407FF0218843234946
:105D000048770846007FF0218843204908770846F5
:105D1000C07DF02188431D49C8750846C07F000931
:105D20000001C8770846807FF021884317498877AB
:105D30000846407F0009000148770846807EF02130
:105D40008843124988760846807E000900018876DB
:105D50000846407E0009000148760846007E00099A
:105D6000000108760846007F000900010877084610
:105D7000C07EF02188430549C8760846407EF02160
:105D800088430249487605B0F0BD0000C0220020DB
:105D900010B50146002200200A0EFE4B985CC30796
:105DA000DB0F002B07D0FC4BDB7FF024A3437033C9
:105DB000F94CE37705E0F84BDB7FF024A343F64C86
:105DC000E37702230340002B07D0F34BDB7F1B0953
:105DD0001B01DB1DF04CE37705E0EF4BDB7F1B097C
:105DE0001B01ED4CE37704230340002B07D0EA4B63
:105DF0009B7F1B091B01DB1DE74CA37705E0E64BEE
:105E00009B7F1B091B01E44CA37708230340002B55
:105E100009D0E14B20335B781B091B01DB1DDE4CF5
:105E20002034637007E0DC4B20335B781B091B01D7
:105E3000D94C2034637010230340002B09D0D64B7B
:105E400020331B78F024A3437033D34C20342370C9
:105E500007E0D14B20331B78F024A343CE4C2034F1
:105E6000237020230340002B09D0CB4B20331B7819
:105E70001B091B01DB1DC84C2034237007E0C64BF7
:105E800020331B781B091B01C34C20342370402393
:105E90000340002B07D0C04B9B7FF024A3437033FB
:105EA000BD4CA37705E0BC4B9B7FF024A343BA4CC9
:105EB000A377FF231B040B401A0CB64B985CC30757
:105EC000DB0F002B07D0B44B1B7F1B091B01DB1D15
:105ED000B14C237705E0B04B1B7F1B091B01AE4C77
:105EE000237702230340002B07D0AB4BDB7EF0244B
:105EF000A3437033A84CE37605E0A74BDB7EF02488
:105F0000A343A54CE37604230340002B07D0A24B08
:105F10009B7EF024A34370339F4CA37605E09E4BF9
:105F20009B7EF024A3439C4CA37608230340002BC4
:105F300007D0994B5B7FF024A3437033964C637773
:105F400005E0954B5B7FF024A343934C63771023CC
:105F50000340002B07D0904B5B7F1B091B01DB1D0F
:105F60008D4C637705E08C4B5B7F1B091B018A4CD2
:105F7000637720230340002B07D0874B1B7FF0243F
:105F8000A3437033844C237705E0834B1B7FF024BD
:105F9000A343814C237740230340002B07D07E4B43
:105FA000DB7E1B091B01DB1D7B4CE37605E07A4B96
:105FB000DB7E1B091B01784CE376FF231B020B40A1
:105FC0001A0A744B985CC307DB0F002B07D0724B87
:105FD0001B7EF024A34370336F4C237605E06E4B99
:105FE0001B7EF024A3436C4C237602230340002B3A
:105FF00007D0694B1B7E1B091B01DB1D664C2376FA
:1060000005E0654B1B7E1B091B01634C23760423B3
:106010000340002B07D0604BDB7D1B091B01DB1D00
:106020005D4CE37505E05C4BDB7D1B091B015A4CA5
:10603000E37508230340002B07D0574B9B7E1B09B9
:106040001B01DB1D544CA37605E0534B9B7E1B09C3
:106050001B01514CA37610230340002B07D04E4B5D
:106060005B7EF024A34370334B4C637605E04A4BD0
:106070005B7EF024A343484C637620230340002B2F
:1060800007D0454B5B7E1B091B01DB1D424C637631
:1060900005E0414B5B7E1B091B013F4C63764023AF
:1060A0000340002B07D03C4BDB7DF024A34370332F
:1060B000394CE37505E0384BDB7DF024A343364CC7
:1060C000E375CAB2334B985CC307DB0F002B07D0D4
:1060D000314B1B7DF024A34370332F4C237505E017
:1060E0002D4B1B7DF024A3432B4C2375022303402F
:1060F000002B07D0284B1B7D1B091B01DB1D264CE9
:10610000237505E0244B1B7D1B091B01224C2375C5
:1061100004230340002B07D01F4BDB7C1B091B0112
:10612000DB1D1D4CE37405E01B4BDB7C1B091B01D5
:10613000194CE37408230340002B07D0164B9B7CBB
:10614000F024A3437033144CA37405E0124B9B7CE2
:10615000F024A343104CA37410230340002B07D05A
:106160000D4B5B7DF024A34370330B4C637505E04E
:10617000094B5B7DF024A343074C63752023034048
:10618000002B0BD0044B5B7D1B091B01DB1D024C5C
:10619000637509E038F30100A02200200C4B5B7D01
:1061A0001B091B010A4C637540230340002B07D0D9
:1061B000074BDB7CF024A3437033054CE37405E00C
:1061C000034BDB7CF024A343014CE37410BD0000BF
:1061D000A022002000B501287ED1FE4AD278F0230B
:1061E0009A437032FB4BDA701A4612791209120187
:1061F000D21D1A711A461279F0239A437032F54B68
:106200001A711A46527912091201D21D5A711A4690
:106210005279F0239A437032EE4B5A711A46D27972
:1062200012091201D21DDA711A46D279F0239A436B
:106230007032E84BDA711A46527A12091201D21DF5
:106240005A721A46527AF0239A437032E14B5A72CC
:106250001A46927AF0239A437032DE4B9A721A46AB
:106260009278F0239A437032DA4B9A701A46D27AB7
:1062700012091201D21DDA721A465278120912015D
:10628000D21D5A701A46D27AF0239A437032D14BFB
:10629000DA721A46203AD27FF0239A437032CD4BFD
:1062A000203BDA77CB4A127B12091201D21D203330
:1062B0001A731A46203A927F12091201D21D203B0E
:1062C0009A77C44A127BF0239A437032C14B1A73F7
:1062D0001A46203A127F00E0F2E1F0239A4370322E
:1062E000BC4B203B1A77BB4A527B12091201D21DCC
:1062F00020335A731A46203AD27E12091201D21D57
:10630000203BDA76B44AD278F0239A437032B24B0B
:10631000DA701A46127B12091201D21D1A731A463C
:10632000127912091201D21D1A711A46927AF023BB
:106330009A437032A84B9A721A461279F0239A4304
:106340007032A54B1A711A46527912091201D21DE8
:106350005A711A46927912091201D21D9A711A467F
:10636000127A12091201D21D1A721A46127AF023F9
:106370009A437032984B1A721A46527A12091201D5
:10638000D21D5A72934A927912091201521C914BF2
:106390009A711A469279F0239A4310328D4B9A7172
:1063A0001A46127A12091201521C1A721A46127AED
:1063B000F0239A431032874B1A721A46927A1209C6
:1063C0001201521C9A721A46D27812091201521CFA
:1063D000DA701A46927812091201521C9A701A4603
:1063E0005278F0239A4310327A4B5A701A46127838
:1063F000F0239A431032774B1A701A46127812091A
:106400001201521C1A701A46203AD27F1209120148
:10641000521C203BDA771A46927FF0239A431032BF
:106420006C4B203B9A771A46527FF0239A431032E6
:10643000684B203B5A771A46527F12091201521CB0
:106440005A771A46127F12091201521C1A771A46FD
:10645000D27EF0239A4310325E4B203BDA761A4606
:10646000927EF0239A4310325A4B203B9A765A4A36
:10647000127BF0239A431032574B1A731A46D27A82
:10648000F0239A431032544BDA721A46D27A120928
:106490001201521CDA721A46927A12091201521C27
:1064A0009A721A46527AF0239A4310324A4B5A7221
:1064B0001A465279F0239A431032474B5A711A46C2
:1064C000D279F0239A431032434BDA710B0007F074
:1064D000BDFF19F3E9DFD5CBC1B7ADA3998F87789D
:1064E0006E645A50463E362E261E160EF5003A4A67
:1064F000D279F0239A437032374BDA7100BF364AB3
:106500005279F0239A437032334B5A7100BF324AAA
:10651000527AF0239A4370322F4B5A7200BF2E4AA0
:10652000927A12091201D21D2B4B9A7200BF2A4A8D
:10653000D27A12091201D21D274BDA7200BF264A05
:10654000D27AF0239A437032234BDA7200BF224A88
:10655000127BF0239A4370321F4B1A7300BF1D4AFF
:10656000203A927EF0239A4370321A4B203B9A765F
:1065700000BF184A203AD27EF0239A437032154B5E
:10658000203BDA7600BF134A203A127F120912012B
:10659000D21D104B203B1A7700BF0E4A203A527F83
:1065A00012091201D21D0B4B203B5A7700BF094A3A
:1065B000203A527FF0239A437032064B203B5A77A1
:1065C00000BF044A203A927FF0239A437032014B75
:1065D000203B03E00C220020E02200209A7700BF3D
:1065E000DC4AD27F12091201D21DDA4BDA7700BFE2
:1065F000D84A2032127812091201D21DD54B20330D
:106600001A7000BFD34A20321278F0239A437032B6
:10661000D04B20331A7000BFCE4A20325278F0237C
:106620009A437032CB4B20335A7000BFC94A203294
:10663000927812091201D21DC64B20339A7000BF06
:10664000C44A2032D27812091201D21DC14B203324
:10665000DA7000BFBF4A2032927A12091201D21DAD
:10666000BC4B20339A7200BFBA4A2032127AF02310
:106670009A437032B74B20331A7200BFB54A2032AA
:10668000127A12091201D21DB24B20331A7200BFC6
:10669000B04A20329279F0239A437032AD4B2033C6
:1066A0009A7100BFAB4A2032927912091201D21DB1
:1066B000A84B20339A7100BF01E0FFE700BF47E11C
:1066C000A44A2032D278F0239A43A24B2033DA70C6
:1066D0001A461279120912011A711A461279F02318
:1066E0009A439C4B20331A711A46527912091201AF
:1066F0005A711A465279F0239A43964B20335A71B5
:106700001A46D27912091201DA711A46D279F023A7
:106710009A43904B2033DA711A46527A12091201C9
:106720005A721A46527AF0239A438A4B20335A728D
:106730001A46927AF0239A43864B20339A721A466D
:106740009278F0239A43834B20339A701A46D27A78
:1067500012091201DA721A465278120912015A709D
:106760001A46D27AF0239A437A4B2033DA72794A66
:10677000D27FF0239A43774BDA771A462032127B86
:106780001209120120331A73724A927F1209120100
:10679000203B9A771A462032127BF0239A436D4BA6
:1067A00020331A736B4A127FF0239A43694B1A778E
:1067B0001A462032527B1209120120335A73654A5D
:1067C000D27E12091201203BDA76634AD278F02396
:1067D0009A43614BDA701A46127B120912011A733E
:1067E0001A461279120912011A711A46927AF02386
:1067F0009A43594B9A721A461279F0239A43564B90
:106800001A711A465279120912015A711A4692796E
:10681000120912019A711A46127A120912011A7299
:106820001A46127AF0239A434B4B1A721A46527A3E
:10683000120912015A72474A203292791209120142
:10684000444B20339A711A469279F0239A43414B74
:1068500020339A711A46127A120912011A721A46D4
:10686000127AF0239A433B4B20331A721A46927ADB
:10687000120912019A721A46D27812091201DA70BC
:106880001A469278120912019A701A465278F02329
:106890009A43304B20335A701A461278F0239A43A9
:1068A0002C4B20331A701A461278120912011A70F2
:1068B000284AD27F12091201203BDA771A46927FCA
:1068C000F0239A43234B9A771A46527FF0239A4338
:1068D000204B5A771A46527F120912015A771A46EC
:1068E000127F120912011A771A46D27EF0239A43B8
:1068F000184BDA761A46927EF0239A43154B9A7615
:10690000154A127BF0239A43134B1A731A46D27A14
:10691000F0239A43104BDA721A46D27A1209120106
:10692000DA721A46927A120912019A721A46527A49
:10693000F0239A43084B5A721A465279F0239A432D
:10694000054B5A711A46D279F0239A43024BDA71F9
:1069500000BD0000EC210020E022002070B50546BB
:106960000C46012D7ED1B348407D00090001C01DB9
:10697000B04948750846007DF02188431030AD4984
:1069800008750846007D00090001401C087508468E
:10699000C07CF02188431030A649C8740846807C2A
:1069A000F02188431030A34988740846807C000990
:1069B0000001401C8874F9F72BFE022803D0F9F778
:1069C00027FE01286ED19C48007801286AD0F5F78F
:1069D00013FF9A49884265D3F9F7B6FD00282FD0F6
:1069E0009448007DF021884370309249087508462C
:1069F000007D00090001C01D08750846C07CF0211B
:106A0000884370308B49C8740846807CF0218843E5
:106A10007030884988740846807C00090001C01DD8
:106A200088740846407DF02188437030814948755C
:106A30000846407CF021884370307E494874F8E075
:106A40007C48007DF021884310307A49087508465B
:106A5000007D00090001401C08750846C07CF0213B
:106A6000884300E0B8E010307249C8740846807C62
:106A7000F021884310306F4988740846807C0009F3
:106A80000001401C88740846407DF0218843103086
:106A9000684948750846407CF021884310306549B4
:106AA0004874C6E0F9F7C6FC002826D1F5F7A4FE25
:106AB0006249884221D3F9F747FD00280ED05D488E
:106AC000407DF021884370305A4948750846407C23
:106AD000F02188437030574948741CE05548407D88
:106AE000F02188431030534948750846407CF02116
:106AF000884310304F4948740DE04E48407DF021E6
:106B0000884370304B4948750846407CF0218843E3
:106B1000703048494874F9F78DFC01282AD146485D
:106B20000078012826D0F5F767FE4449884221D332
:106B30004048407DF021884370303E494875084602
:106B4000407CF021884370303A494874F9F7FCFCE6
:106B5000002807D03748007DF02188437030354940
:106B6000087566E03348007DF021884310303149D4
:106B700008755EE0230007F069FC062C241C140C49
:106B8000042D2C48807C00090001C01D294988740F
:106B900000BF2848807CF0218843703025498874E4
:106BA00000BF2448C07CF021884370302149C8745C
:106BB00000BF2048007D00090001C01D1D49087567
:106BC00000BF1C48007DF0218843703019490875CA
:106BD00000BF00E000BF2CE01648407DF021884354
:106BE000144948750846007DF0218843114908750D
:106BF0000846007D0009000108750846C07CF021A8
:106C000088430C49C8740846807CF02188430949B0
:106C100088740846807C0009000188740846407D1D
:106C20000009000148750846407CF021884301496D
:106C3000487470BD0C22002003010020B80B000036
:106C400030B50246002901D1002000E007201300E2
:106C500007F0FCFB0F09141F2B3743505D67727C54
:106C600088929FA9B500574B5B7EF024A343040193
:106C7000F0252C402343534C6376A1E0524B9B7983
:106C8000F024A3430401F0252C4023434E4CA37170
:106C900096E04D4B2033DB791B091B010407240FC1
:106CA0002343494C2034E3718AE0464B2033DB7C9C
:106CB0001B091B010407240F2343424C2034E374B7
:106CC0007EE0404B40331B781B091B010407240F57
:106CD00023433C4C4034237072E03A4B2033DB7F3B
:106CE000F024A3430401F0252C402343354C2034E9
:106CF000E37765E0334B20335B7BF024A34304014F
:106D0000F0252C4023432F4C2034637358E02E4B46
:106D10009B791B091B010407240F23432A4CA371F1
:106D20004EE0294B9B7CF024A3430401F0252C402A
:106D30002343254CA37443E0234BDB7E1B091B013B
:106D40000407240F2343204CE37639E01D4B203306
:106D5000DB7F1B091B010407240F2343194C20343C
:106D6000E3772DE0174B9B7E1B091B010407240FC3
:106D70002343144CA37623E0134B20339B79F02458
:106D8000A3430401F0252C4023430F4C2034A3716E
:106D900016E00D4BDB7D1B091B010407240F234369
:106DA000094CE3750CE0074B20335B7C1B091B018E
:106DB0000407240F2343034C2034637400E000BF16
:106DC00000BF30BDEC210020C0220020F7B582B00A
:106DD0000746154600260024FE480078012804D006
:106DE000F5F70AFDFC49884279D2FC48407CF02145
:106DF00088437030F94948740846807C00090001D6
:106E0000C01D88740846007D00090001C01D08757A
:106E10000846007DF02188437030F0490875084627
:106E2000807CF02188437030EC4988740846C07C2F
:106E300000090001C01DC8740846C07CF0218843C9
:106E40007030E649C8740846407C00090001C01D46
:106E500048740846407D00090001C01D4875084679
:106E6000407DF02188437030DC4948750846007C3D
:106E7000F02188437030D94908740846007C000925
:106E80000001C01D08740846C07BF02188437030A3
:106E9000D249C873BA220A210020FBF707FFBA22A1
:106EA00013210020FBF702FFBA2211210020FBF77B
:106EB000FDFEBA2212210020FBF7F8FEBA220E21B5
:106EC0000020FBF7F3FEBA220F210020FBF7EEFEB5
:106ED000BA2210210020FBF7E9FEFDE3FFE703984B
:106EE000801E0F2878D243007B449B885B009F4420
:106EF0000E007400D9003F01AC011002730074024F
:106F0000730073007300DA023D037300A303B348F8
:106F1000407CF0218843B14948740846807C0009D0
:106F2000000188740846007D00090001C01D087535
:106F30000846007DF02188437030A849087508464E
:106F4000807CF0218843A54988740846C07C0009EC
:106F50000001C01DC8740846C07CF02188439F49C9
:106F6000C8740846407C0009000148740846407D0A
:106F70000009000148750846407DF0218843974983
:106F800048750846007CF0218843944908740846F7
:106F9000007C0009000108740846C07BF02188438A
:106FA0008E49C873BA220A210020FBF77FFEBA225D
:106FB00013210020FBF77AFE00220E211046FBF77A
:106FC00075FE00220F211046FBF770FE00221021F3
:106FD0001046FBF76BFEF6E393E38048407CF0211C
:106FE00088437E4948740846807C00090001887403
:106FF0000846007D00090001C01D08750846007D97
:10700000F02188437030754908750846807CF0216E
:107010008843724988740846C07C00090001C8741E
:107020000846C07CF02188436C49C8740846407CFF
:107030000009000148740846407D00090001C01D98
:1070400048750846407DF0218843644948750846E4
:10705000007CF0218843614908740846007C0009DF
:10706000000108740846C07BF02188435B49C8735F
:10707000BA220A210020FBF719FEBA2213210020B0
:10708000FBF714FE00220E211046FBF70FFE002234
:107090000F211046FBF70AFE002210211046FBF7D5
:1070A00005FE90E34D48407CF02188434B494874ED
:1070B0000846807C00090001C01D88740846007DD8
:1070C00000090001C01D08750846007DF0218843B5
:1070D0007030424908750846807CF0218843703042
:1070E0003E4988740846C07C00090001C8740846FF
:1070F000C07CF02188433949C8740846407C0009A7
:10710000000148740846407D0009000148750846A2
:10711000407DF0218843314948750846007CF021C4
:1071200088432E4908740846007C00090001087451
:107130000846C07BF02188432849C873BA220A2137
:107140000020FBF7B3FDBA2213210020FBF7AEFDB0
:1071500000220E211046FBF7A9FD00220F21104648
:10716000FBF7A4FD002210211046FBF79FFD2AE348
:107170001A48407CF0218843184948740846807CAE
:1071800000090001C01D88740846007D0009000147
:10719000C01D08750846007DF021884370300F49F6
:1071A00008750846807CF02188430C49887408469D
:1071B000C07C00090001C8740846C07CF0218843E7
:1071C0000649C8740846407C00090001C01D487487
:1071D000084605E003010020B80B00002C22002027
:1071E000407D0009000148750846407DF021884334
:1071F000FE4948750846007CF0218843FB49087425
:107200000846007C0009000108740846C07BF02194
:107210008843F649C873BA220A210020FBF746FDCD
:10722000BA2213210020FBF741FD00220E21104657
:10723000FBF73CFD00220F211046FBF737FD002233
:1072400010211046FBF732FDBDE2E848407CF021FA
:107250008843E64948740846807C00090001887428
:107260000846007D0009000108750846007DF021F0
:1072700088437030DD4908750846807CF0218843DA
:10728000DA4988740846C07C00090001C8740846C1
:10729000C07CF02188437030D449C8740846407CD3
:1072A0000009000148740846407D00090001487546
:1072B0000846407DF0218843CC4948750846007C4B
:1072C000F0218843C94908740846007C0009000180
:1072D00008740846C07BF0218843C449C873BA22A9
:1072E0000A210020FBF7E2FCBA2213210020FBF761
:1072F000DDFC00220E211046FBF7D8FC00220F21F6
:107300001046FBF7D3FC002210211046FBF7CEFC01
:1073100059E2B648407CF0218843B4494874084695
:10732000807C0009000188740846007D0009000186
:1073300008750846007DF02188437030AB49087518
:107340000846807CF0218843A84988740846C07CA0
:1073500000090001C8740846C07CF0218843A34995
:10736000C8740846407C0009000148740846407D06
:107370000009000148750846407DF02188437030BF
:107380009A4948750846007CF0218843974908745B
:107390000846007C0009000108740846C07BF02103
:1073A00088439249C873BA220A210020FBF77EFC69
:1073B000BA2213210020FBF779FC00220E2110468F
:1073C000FBF774FC00220F211046FBF76FFC002234
:1073D00010211046FBF76AFCF5E18448407CF0215F
:1073E00088437030814948740846807C0009000158
:1073F000C01D88740846007D00090001C01D087585
:107400000846007DF02188437030784908750846A9
:10741000807CF0218843754988740846C07C000947
:107420000001C8740846C07CF02188436F49C874C5
:107430000846407C0009000148740846407D000968
:10744000000148750846407DF0218843674948752A
:107450000846007CF0218843644908740846007C93
:107460000009000108740846C07BF02188435F4989
:10747000C873BA220A210020FBF718FCBA22132194
:107480000020FBF713FC00220E211046FBF70EFC38
:1074900000220F211046FBF709FC002210211046A4
:1074A000FBF704FC8FE15148407CF02188434F49B1
:1074B00048740846807C0009000188740846007DF5
:1074C0000009000108750846007DF02188434749FE
:1074D00008750846807CF021884344498874084632
:1074E000C07C00090001C8740846C07CF0218843B4
:1074F0003E49C8740846407C0009000148740846AB
:10750000407D0009000148750846407DF021884310
:10751000364948750846007CF02188433349087491
:107520000846007C0009000108740846C07BF02171
:10753000884370302D49C87300220A211046FBF79A
:10754000B5FB002213211046FBF7B0FBBA220E2137
:107550000020FBF7ABFB00220F211046FBF7A6FB38
:10756000002210211046FBF7A1FB2CE11F48407CB4
:10757000F02188431D4948740846807C00090001B9
:1075800088740846007D0009000108750846007DE2
:10759000F0218843154908750846807CF02188430E
:1075A000124988740846C07C00090001C874084666
:1075B000C07CF02188430D49C8740846407C00090E
:1075C000000148740846407D0009000148750846DE
:1075D000407DF0218843054948750846007CF0212C
:1075E0008843024908740846007C01E02C220020F0
:1075F00000090001C01D08740846C07BF0218843C3
:10760000F949C87300220A211046FBF74FFB0022FC
:1076100013211046FBF74AFB00220E211046FBF710
:1076200045FBBA220F210020FBF740FB002210216E
:107630001046FBF73BFBC6E0EB48407CF02188435B
:10764000E94948740846807C0009000188740846AE
:10765000007D0009000108750846007DF02188437F
:10766000E14908750846807CF0218843DE4988742A
:107670000846C07C00090001C8740846C07CF0219F
:107680008843D949C8740846407C00090001487401
:107690000846407D0009000148750846407DF021FC
:1076A0008843D14948750846007CF02188437030F2
:1076B000CD4908740846007C00090001087408469A
:1076C000C07BF0218843C849C87300220A211046B4
:1076D000FBF7ECFA002200E076E013211046FBF7FE
:1076E000E5FA00220E211046FBF7E0FA00220F21F6
:1076F0001046FBF7DBFABA2210210020FBF7D6FA7E
:1077000061E0B948407CF0218843B7494874084695
:10771000807C0009000188740846007D0009000192
:1077200008750846007DF0218843AF490875084672
:10773000807CF0218843AC4988740846C07C0009ED
:107740000001C8740846C07CF0218843A649C8746B
:107750000846407C0009000148740846407D000945
:10776000000148750846407DF02188439E494875D0
:107770000846007CF02188439B4908740846007C39
:107780000009000108740846C07BF021884396492F
:10779000C87300220A211046FBF788FA0022132141
:1077A0001046FBF783FA00220E211046FBF77EFA03
:1077B00000220F211046FBF779FA00221021104613
:1077C000FBF774FA00BF00BF002F76D0BA22112158
:1077D0000020FBF76BFABA2212210020FBF766FAB1
:1077E00082480078012804D0F5F706F880498842DD
:1077F00016D28048807BF021884370307D498873A1
:10780000084640300078F021884370307949403193
:1078100008700846007800090001C01D08702DE0BE
:107820007D20C000854214D27248807BF0218843BD
:1078300070498873084640300078F02188437030E2
:107840006C49403108700846007800090001087052
:1078500014E06848807BF021884370306549887364
:10786000084640300078F021884362494031087072
:107870000846007800090001C01D08707D20C00086
:10788000854205D201462846F0F75AFC064604E038
:1078900059492846F0F754FC06465848845DE007ED
:1078A000C00F00280AD053484030C07800090001BA
:1078B000C01D50494031C87008E0A6E24D48403034
:1078C000C078000900014B494031C87002202040B7
:1078D000002807D04748C07900090001C01D45496C
:1078E000C87105E04348C079000900014149C871E9
:1078F00004202040002807D03E488079000900017C
:10790000C01D3C49887105E03A48807900090001B2
:107910003849887108202040002807D03548407930
:10792000F021884370303349487105E0314840798F
:10793000F02188432F49487110202040002807D0AB
:107940002C48407900090001C01D2A49487105E012
:10795000284840790009000126494871202020402C
:10796000002807D023480079F0218843703021494E
:10797000087105E01F480079F02188431D4908710E
:1079800040202040002807D01A488079F021884301
:1079900070301849887105E016488079F0218843D5
:1079A000144988717D20C000854207D26421284691
:1079B000F0F7C6FB06461148845D27E0642128469F
:1079C000F0F7BEFB7D21C9000090F0F7B9FB0191F3
:1079D00064210198F0F7B4FB06460948854213D3A9
:1079E0000848845D12E000002C22002003010020E2
:1079F000B80B0000A0220020A08601004BF301007C
:107A00001027000038F30100F948845DE007C00F3B
:107A1000002807D0F7488078F02188437030F54976
:107A2000887005E0F3488078F0218843F149887038
:107A300002202040002809D0EE484038807A000912
:107A40000001C01DEB494039887207E0E948403821
:107A5000807A00090001E7494039887204202040FB
:107A6000002809D0E3484038407A00090001C01DD1
:107A7000E0494039487207E0DE484038407A000962
:107A80000001DC494039487208202040002809D014
:107A9000D8484038007AF02188437030D5494039C1
:107AA000087207E0D3484038007AF0218843D14972
:107AB0004039087210202040002809D0CD484038B5
:107AC000007A00090001C01DCA494039087207E068
:107AD000C8484038007A00090001C6494039087298
:107AE00020202040002809D0C2484038C079F02129
:107AF00088437030BF494039C87107E0BD484038FD
:107B0000C079F0218843BB494039C87140202040EA
:107B1000002809D0B7484038407AF02188437030B7
:107B2000B4494039487207E0B2484038407AF02101
:107B30008843B049403948727D20C000854210D248
:107B40000A212846F0F7FCFA0A210190F0F7F8FA2A
:107B50000E460A2D02D3A848845D11E0A448845D36
:107B60000EE064212846F0F7EBFA0A210090F0F7C6
:107B7000E7FA0A210190F0F7E3FA0E469E498C5D80
:107B8000E007C00F002807D09A488078000900015C
:107B9000C01D9849887005E096488078000900016A
:107BA0009449887002202040002809D0914840382C
:107BB000807B00090001C01D8E494039887307E0B1
:107BC0008C484038807B000900018A49403988731D
:107BD00004202040002809D086484038407B000916
:107BE0000001C01D83494039487307E0814840388F
:107BF000407B000900017F4940394873082020403C
:107C0000002809D07B484038007BF0218843703041
:107C100078494039087307E076484038007BF02106
:107C2000884374494039087310202040002809D047
:107C300070484038C07A00090001C01D6D494039C4
:107C4000C87207E06B484038C07A000900016949F2
:107C50004039C87220202040002809D065484038AB
:107C6000807AF0218843703062494039887207E099
:107C700060484038807AF02188435E4940398872F4
:107C800040202040002809D05A484038407BF0214D
:107C90008843703057494039487307E055484038A9
:107CA000407BF02188435349403948737D20C00010
:107CB000854207D20A212846F0F742FA0E464E487E
:107CC000845D0AE064212846F0F73AFA0A2101901F
:107CD000F0F736FA0E4648498C5DE007C00F0028E1
:107CE00007D044484078F0218843703041494870BB
:107CF00005E040484078F02188433E494870022022
:107D00002040002807D03B48407800090001C01DF2
:107D10003849487005E03748407800090001354986
:107D2000487004202040002809D032484038007CA8
:107D3000F021884370302F494039087407E02D48FE
:107D40004038007CF02188432A49403908740820D3
:107D50002040002809D027484038007C0009000155
:107D6000C01D24494039087407E022484038007C8F
:107D7000000900011F4940390874102020400028E4
:107D800009D01C484038C07BF02188437030194925
:107D90004039C87307E017484038C07BF02188435A
:107DA00014494039C87320202040002809D01148C8
:107DB0004038C07B00090001C01D0E494039C8731E
:107DC00007E00C484038C07B0009000109494039F0
:107DD000C87340202040002810D006484038407C1E
:107DE00000090001C01D034940394874E8E0000063
:107DF0004BF30100E022002038F301007148407C81
:107E0000000900016F494874DAE000220A21104697
:107E1000FAF74CFF002213211046FAF747FF002221
:107E200011211046FAF742FF002212211046FAF7FC
:107E30003DFF00220E211046FAF738FF00220F21E5
:107E40001046FAF733FF002210211046FAF72EFFF2
:107E50005C484030C078000900015A494031C87080
:107E60005848C079000900014039C8710846807936
:107E700000090001887108464079F0218843514982
:107E800048710846407900090001487108460079A8
:107E9000F02188434B49087108468079F0218843D6
:107EA00048498871084640308078F0218843454928
:107EB000403188704348807A000900014039887257
:107EC0000846407A0009000148720846007AF0210D
:107ED00088433C4908720846007A0009000108728C
:107EE0000846C079F02188433649C8710846407A6F
:107EF000F0218843334948720846403080780009B1
:107F00000001403188702F48807B00090001403912
:107F100088730846407B0009000148730846007BCF
:107F2000F0218843274908730846C07A00090001F8
:107F3000C8720846807AF021884322498872084630
:107F4000407BF02188431F49487308464030407801
:107F5000F02188431B4940314870084640780009A9
:107F6000000148701748007CF021884315490874C7
:107F70000846007C0009000108740846C07BF02117
:107F800088431049C8730846C07B00090001C873C4
:107F90000846407C0009000148740846807BF021B7
:107FA000884308498873084640300078F0218843A8
:107FB0000449403108700846007800090001087043
:107FC00005B0F0BDA0220020F7B582B007460E46EE
:107FD0000121FF200830FCF737FE0121FC48FCF7A7
:107FE00033FEFC48007801287ED0F4F705FCFA49FE
:107FF000884279D3F8F72AFA032843D1F8F720FA10
:10800000002803D0F8F71CFA01283BD1002F1CD11F
:10801000F8F79AFA00280CD0F048407CF021884309
:10802000EE4948740846807C00090001C01D887430
:10803000EEE0EA48407CF0218843E849487408466D
:10804000807C000900018874E2E0F8F77DFA0028DE
:108050000CD0E248407CF02188437030DF494874FE
:108060000846807C000900018874D1E0DB48407C30
:10807000F0218843D94948740846807C00090001F2
:108080008874C5E0F8F7DCF9002803D0F8F7D8F9D0
:10809000012865D1002F0CD1D048407CF0218843C5
:1080A000CE4948740846807C00090001C01D8874D0
:1080B0000BE0CA48407CF02188437030C7494874BF
:1080C0000846807C000900018874F8F7B9F9002897
:1080D00021D1C2482030C078F02188437030BF4998
:1080E0002031C870BD4800E064E0807D00090001D7
:1080F000203988750846807DF0218843B749887506
:10810000BA2223210020FAF7D1FD002222211046B5
:10811000FAF7CCFD7CE0F8F793F9012878D1AF4865
:108120002030C078F0218843AC492031C870AB487A
:10813000807D00090001C01D203988750846807DBA
:10814000F02188437030A54988750022232110460C
:10815000FAF7ACFDBA2222210020FAF7A7FD57E07A
:108160009E48407CF02188439C4948740846807CA6
:1081700000090001887408462030C078F021884347
:1081800096492031C8709548807D0009000120394A
:1081900088750846807DF0218843904988750022C3
:1081A00023211046FAF782FD002222211046FAF719
:1081B0007DFD2DE08948407CF0218843703087495F
:1081C00048740846807C00090001C01D8874084678
:1081D0002030C078F0218843703080492031C87049
:1081E0007E48807D00090001C01D20398875084641
:1081F000807DF0218843703078498875BA22232128
:108200000020FAF753FDBA2222210020FAF74EFD92
:10821000F8F716F9002808D06E480078012804D035
:10822000F4F7EAFA6C49884276D26D48864209D959
:108230006A4820304079F021884370306749203106
:10824000487107E0654820304079F0218843634950
:108250002031487163493046EFF772FF0A210190DF
:10826000EFF76EFF0D465E48401C864202D35E4823
:10827000445D01E05D48445DE007C00F002809D07F
:1082800056482030C07800090001C01D53492031F4
:10829000C87007E051482030C078000900014F49FC
:1082A0002031C87002202040002809D04B482030DF
:1082B0008078F0218843703048492031887007E089
:1082C000464820308078F021884344492031887026
:1082D00004202040002809D0404820304078F02178
:1082E000884370303D492031487007E03B482030DA
:1082F0004078F021884339492031487008202040D7
:1083000000280AD035482030407900090001C01DFE
:1083100032492031487108E0A1E2304820304079EC
:10832000000900012D49203148711020204000280B
:1083300009D02A4820300079F0218843703027493D
:108340002031087107E0254820300079F02188436A
:1083500022492031087120202040002809D01F48E0
:108360002030007900090001C01D1C49203108712E
:1083700007E01A4820300079000900011749203130
:10838000087140202040002809D01448203080780F
:1083900000090001C01D11492031887007E00F4815
:1083A00020308078000900010C49203188707D213F
:1083B000C9003046EFF7C4FE0A210190EFF7C0FE76
:1083C0000D460848864213D30748445D12E000007A
:1083D0000505000003010020B80B0000A0220020CA
:1083E0009F8601001027000038F301004BF30100C5
:1083F000F948445DE007C00F002807D0F748C07F68
:10840000F02188437030F549C87705E0F348C07F14
:10841000F0218843F149C87702202040002807D086
:10842000EE48C07F00090001C01DEC49C87705E097
:10843000EA48C07F00090001E849C87704202040CD
:10844000002807D0E548807F00090001C01DE349EE
:10845000887705E0E148807F00090001DF498877DF
:1084600008202040002809D0DC482030407800094E
:108470000001C01DD9492031487007E0D74820309D
:10848000407800090001D549203148701020204073
:10849000002809D0D14820300078F021884370307E
:1084A000CE492031087007E0CC4820300078F02118
:1084B0008843CA492031087020202040002809D074
:1084C000C6482030007800090001C01DC349203192
:1084D000087007E0C1482030007800090001BF495A
:1084E0002031087040202040002807D0BB48807F02
:1084F000F02188437030B949887705E0B748807F1C
:10850000F0218843B549887764213046EFF718FE9B
:108510000A210190EFF714FE0D467D20C00086422F
:1085200002D3AF48445D01E0AB48445DE007C00FB3
:10853000002807D0A948007F00090001C01DA749F5
:10854000087705E0A548007F00090001A3490877E6
:1085500002202040002807D0A048C07EF021884398
:1085600070309E49C87605E09C48C07EF021884363
:108570009A49C87604202040002807D09748807E7A
:10858000F021884370309549887605E09348807ED5
:10859000F02188439149887608202040002807D0A0
:1085A0008E48407FF021884370308C49487705E041
:1085B0008A48407FF021884388494877102020402E
:1085C000002807D08548407F00090001C01D83496D
:1085D000487705E08148407F000900017F494877DE
:1085E00020202040002807D07C48007FF0218843CD
:1085F00070307A49087705E07848007FF021884399
:108600007649087740202040002807D07348C07E74
:1086100000090001C01D7149C87605E06F48C07EA1
:10862000000900016D49C8760A213046EFF788FD40
:108630000A210190EFF784FD0D46642E02D36848AD
:10864000445D01E06448445DE007C00F002807D0A6
:108650006248007EF021884370306049087605E06A
:108660005E48007EF02188435C4908760220204065
:10867000002807D05948007E00090001C01D574955
:10868000087605E05548007E000900015349087648
:1086900004202040002807D05048C07D0009000178
:1086A000C01D4E49C87505E04C48C07D0009000159
:1086B0004A49C87508202040002807D04748807ED6
:1086C00000090001C01D4549887605E04348807EC9
:1086D000000900014149887610202040002807D079
:1086E0003E48407EF021884370303C49487605E0A2
:1086F0003A48407EF021884338494876202020407F
:10870000002807D03548407E00090001C01D3349CC
:10871000487605E03148407E000900012F4948763F
:1087200040202040002807D02C48C07DF0218843FD
:1087300070302A49C87505E02848C07DF02188437B
:108740002649C8750A213046EFF7FAFC0D46244841
:10875000445DE007C00F002807D02048007DF021CD
:10876000884370301D49087505E01C48007DF021E4
:1087700088431A49087502202040002807D017486E
:10878000007D00090001C01D1449087505E013486B
:10879000007D0009000111490875042020400028CF
:1087A00007D00E48C07C00090001C01D0B49C874E9
:1087B00005E00A48C07C000900010849C874082087
:1087C000204000280ED00548807CF021884370307E
:1087D000024988740CE000004BF30100A022002045
:1087E00038F30100FA48807CF0218843F849887406
:1087F00010202040002807D0F548407DF021884314
:108800007030F349487505E0F148407DF021884318
:10881000EF49487520202040002807D0EC48407DD3
:1088200000090001C01DEA49487505E0E848407D9F
:1088300000090001E649487540202040002807D083
:10884000E348C07CF02188437030E149C8746DE290
:10885000DF48C07CF0218843DD49C874F7E7F7F7AB
:10886000EFFD01287CD1DA4820304079F02188439F
:10887000D749203148710846C07800090001C87006
:1088800008468078F0218843D14920318870084615
:108890004078F0218843CE4920314870084640791D
:1088A00000090001487108460079F0218843C84951
:1088B0002031087108460079000900010871084656
:1088C00080780009000188707D21C9000498EFF7C5
:1088D00037FC0546BF48445DE007C00F002807D0BD
:1088E000BB48C07FF02188437030B949C87705E0A4
:1088F000B748C07FF0218843B549C877022020409F
:10890000002807D0B248C07F00090001C01DB0494F
:10891000C87705E0AE48C07F00090001AC49C877C0
:1089200004202040002807D0A948807F00090001CA
:10893000C01DA749887705E0A548807F0009000190
:10894000A34988770820204000280AD0A04820307A
:10895000407800090001C01D9D492031487008E0A1
:10896000ECE19B4820304078000900019849203113
:10897000487010202040002809D095482030007809
:10898000F0218843703092492031087007E0904808
:1089900020300078F02188438D4920310870202054
:1089A0002040002809D08A482030007800090001C2
:1089B000C01D87492031087007E0854820300078C5
:1089C0000009000182492031087040202040002821
:1089D00007D07F48807FF021884370307C498877BA
:1089E00005E07B48807FF0218843794988776421BE
:1089F0000498EFF7A5FB0A210190EFF7A1FB0D46C4
:108A00007D21C9000498884202D37348445D01E087
:108A10007048445DE007C00F002807D06C48007F15
:108A200000090001C01D6A49087705E06848007F19
:108A3000000900016649087702202040002807D07D
:108A40006348C07EF021884370306149C87605E0F4
:108A50005F48C07EF02188435D49C87604202040ED
:108A6000002807D05A48807EF0218843703058494A
:108A7000887605E05648807EF02188435449887600
:108A800008202040002807D05148407FF02188432B
:108A900070304F49487705E04D48407FF0218843CA
:108AA0004B49487710202040002807D04848407F95
:108AB00000090001C01D4649487705E04448407F51
:108AC000000900014249487720202040002807D0B3
:108AD0003F48007FF021884370303D49087705E02A
:108AE0003B48007FF02188433949087740202040E7
:108AF000002807D03648C07E00090001C01D344957
:108B0000C87605E03248C07E000900013049C876C9
:108B10000A210498EFF714FB0A210190EFF710FBEC
:108B20000D462D48445DE007C00F002807D02848B7
:108B3000007EF021884370302549087605E02448FE
:108B4000007EF02188432249087602202040002838
:108B500007D01F48007E00090001C01D1C4908768F
:108B600005E01B48007E0009000119490876042031
:108B70002040002807D01648C07D00090001C01D14
:108B80001349C87505E01248C07D0009000110496D
:108B9000C87508202040002807D00D48807E0009B5
:108BA0000001C01D0A49887605E00948807E000959
:108BB0000001074988761020204000280ED0044884
:108BC000407EF02188437030014948760CE0000077
:108BD000A02200204BF3010038F30100FE48407E44
:108BE000F0218843FC49487620202040002807D007
:108BF000F948407E00090001C01DF749487605E0AC
:108C0000F548407E00090001F349487640202040A5
:108C1000002807D0F048C07DF02188437030EE492D
:108C2000C87505E0EC48C07DF0218843EA49C87565
:108C30000A210498EFF784FA0D46E848445DE007FE
:108C4000C00F002807D0E448007DF0218843703031
:108C5000E149087505E0E048007DF0218843DE49E0
:108C6000087502202040002807D0DB48007D00095D
:108C70000001C01DD849087505E0D748007D0009EE
:108C80000001D549087504202040002807D0D248AB
:108C9000C07C00090001C01DCF49C87405E0CE4862
:108CA000C07C00090001CC49C8740820204000287D
:108CB00007D0C948807CF02188437030C649887449
:108CC00005E0C548807CF0218843C34988741020A2
:108CD0002040002807D0C048407DF02188437030F4
:108CE000BD49487505E0BC48407DF0218843BA493C
:108CF000487520202040002807D0B748407D000953
:108D00000001C01DB449487505E0B348407D000925
:108D10000001B149487540202040002807D0AE48E6
:108D2000C07CF02188437030AB49C8744CE2AA483B
:108D3000C07CF0218843A849C87445E2F7F780FB5E
:108D400002287DD1A44820304079F0218843A249EF
:108D5000203148710021A248F2F7B4F9552830D1EA
:108D6000A048FDF715F89C482030C07800090001A4
:108D700099492031C87008468078F0218843964987
:108D80002031887008464078F0218843924920318C
:108D9000487008464079000900014871084600798A
:108DA000F02188438C492031087108460079000978
:108DB000000108710846807800090001C01D887014
:108DC00002E289480078401C8749087082482030B8
:108DD000C07800090001C01D7F492031C8700846D5
:108DE0008078F021884370307B49203188700846B4
:108DF0004078F0218843784920314870084640790E
:108E000000090001487108460079F021884370305C
:108E10007149203108710846007900090001C01D20
:108E200008710846807800090001C01D88706F48ED
:108E3000007800280FD16E48006800280BD100E0B0
:108E400070E0FCF7A5FF00206749087069490860D9
:108E500069490860B8E164480078642828DA6748FE
:108E6000007862490978884204DB60480078401E37
:108E7000624908705D4802785D495E480068F6F70F
:108E800011FA00280FD15D48007880005849085831
:108E9000002808D0594800788000085855490860D3
:108EA000002051490870534800685349086034E075
:108EB0004D480078642830DB50480078401C4F490A
:108EC00008700846007849490978884202DB00208A
:108ED0004A49087049480078800045490858454982
:108EE000086000204049087042480068424909680B
:108EF000884212D13D480078401E40490978884296
:108F00000BDD3E480078401C3C490870084600785C
:108F10008000374908583749086036480068FCF730
:108F200037FF51E1F7F78CFA032893D12A48203014
:108F30004079F02188432849203148710846C0789B
:108F400000090001C01DC87008468078F0218843E0
:108F500021492031887008464078F02188437030DC
:108F60001D49203148700846407900090001C01DA4
:108F7000487108460079F02188431749203108716B
:108F80000846007900090001C01D08710846807874
:108F900000090001C01D88700F48C07FF021884380
:108FA0000D49C8770846C07F00090001C877084608
:108FB000807F00090001887708462030407800094A
:108FC00000012031487008460078F02188430249AA
:108FD00020310870084613E0A022002038F3010079
:108FE000280800200B0B0B0B7000002082000020D3
:108FF000B00B0020680000206C00002064000020FE
:10900000007800090001087008462038807FF021B0
:1090100088436E4988770846007F00090001C01D1B
:1090200008770846C07EF021884370306749C876CB
:109030000846807EF021884370306449887608466F
:10904000407FF02188437030604948770846407F70
:1090500000090001C01D48770846007FF0218843C1
:1090600070305A4908770846C07E00090001C8766A
:10907000F7F726FA002855D15448007EF02188439E
:109080007030524908760846007E000900010876D3
:109090000846C07D00090001C8750846807E0009A9
:1090A000000188760846407EF021884370304749A9
:1090B00048760846407E00090001C01D48760846F3
:1090C000C07DF021884370304049C8750846007D56
:1090D000F021884370303D4908750846007D00093D
:1090E000000108750846C07C00090001C8740846E4
:1090F000807CF0218843354988740846407DF02102
:1091000088437030314948750846407D00090001A8
:10911000C01D48750846C07CF021884370302B493B
:10912000C87451E02948007EF021884370302749F7
:1091300008760846007E00090001C01D0876084632
:10914000C07D00090001C01DC8750846807E000969
:10915000000188760846407EF021884370301B4924
:1091600048760846407E00090001C01D4876084642
:10917000C07DF02188431549C8750846007DF0215F
:109180008843124908750846007D000900010875EA
:109190000846C07C00090001C8740846807CF021A4
:1091A00088430A4988740846407DF021884307496E
:1091B00048750846407D0009000148750846C07C96
:1091C000F02188430149C87405B0F0BDA0220020F9
:1091D000FFB581B006461D46002000900027002EF6
:1091E00076D0FA488079F02188437030F749887149
:1091F00008462038007FF02188437030F349203939
:109200000877F3480078012873D0F3F7F5FAF149AD
:1092100088426ED3F7F71AF904286CD1002D34D1A7
:10922000EA482038807EF02188437030E7492039B1
:109230008876E6480079F02188437030E349087168
:10924000F7F782F9002810D0E0482038807D000927
:109250000001DE49203988750846807DF021884369
:109260007030DA4920398875A5E0D8482038807DEB
:1092700000090001D549203988750846807DF02114
:109280008843D2492039887595E0D0482038807EBF
:10929000F0218843CD4920398876CC480079F021E7
:1092A0008843CA490871F7F74FF9002811D0C74819
:1092B0002038807D00090001C01DC449203988750F
:1092C0000846807DF0218843C0492039887572E0C6
:1092D0007CE3BE482038807D00090001BB4920396D
:1092E00088750846807DF0218843B8492039887503
:1092F00061E040E0FFE7002D1FD1B4482038807DB9
:1093000000090001B149203988750846807DF021A7
:1093100088437030AD49203988750846807EF02139
:1093200088437030A94920398876A8480079F0210F
:1093300088437030A54908713DE0A4482038807DFD
:1093400000090001C01DA149203988750846807DAB
:10935000F02188439D49203988750846807EF02198
:1093600088439A492039887698480079F0218843C3
:10937000964908711FE095482038807D000900015A
:10938000C01D9249203988750846807DF0218843A8
:1093900070308E49203988750846807EF0218843D8
:1093A00070308A492039887688480079F0218843CE
:1093B0007030864908710A9801287DD10A210298E7
:1093C000EEF7BEFE0090844900980C5CE007C00FE9
:1093D000002807D07D48C07900090001C01D7B49E5
:1093E000C87105E07948C079000900017749C87162
:1093F00002202040002807D074488079000900012D
:10940000C01D7249887105E070488079000900012B
:109410006E49887104202040002807D06B484079AD
:1094200000090001C01D6949487105E0674840799D
:10943000000900016549487108202040002807D034
:109440006248007AF021884370306049087205E074
:109450005E48007AF02188435C4908721020204061
:10946000002807D05948007A00090001C01D57495B
:10947000087205E05548007A000900015349087256
:1094800020202040002807D05048C079F021884390
:1094900070304E49C87105E04C48C079F0218843CE
:1094A0004A49C87140202040002809D047484079E7
:1094B000F0218843703000E097E04449487105E0AE
:1094C00042484079F0218843404948710A21029876
:1094D000EEF736FE0091404900980C5CE007C00FA3
:1094E000002807D03948C07800090001C01D37495D
:1094F000C87005E03548C078000900013349C870DC
:1095000002202040002807D030488078F02188438E
:1095100070302E49887005E02C488078F02188430F
:109520002A49887004202040002807D02748407826
:10953000F021884370302549487005E02348407881
:10954000F02188432149487008202040002807D096
:109550001E48407800090001C01D1C49487005E004
:109560001A4840780009000118494870102020402E
:10957000002807D01548007900090001C01D1349D3
:10958000087105E011480079000900010F490871D0
:1095900020202040002807D00C48C078F0218843C4
:1095A00070300A49C87005E00848C078F021884347
:1095B0000649C8704020204000280FD0034880781A
:1095C00000090001C01D014988705CE02C220020C8
:1095D00003010020B80B000038F30100F94880783F
:1095E00000090001F74988704DE0F6484079F02104
:1095F00088437030F34948710846807800090001BB
:10960000C01D88700846C07900090001C87108466D
:10961000807900090001887108464079000900013D
:1096200048710846007AF0218843E64908720846E6
:10963000007A0009000108720846C079F0218843C9
:10964000E049C8710846C07800090001C8700846A2
:109650008078F0218843DB49887008464078F02103
:109660008843D8494870084640780009000148708E
:10967000084600790009000108710846C078F02109
:109680008843D049C8700B9801287DD10A210398DE
:10969000EEF756FD0746CC48C45DE007C00F002832
:1096A00009D0C8482038407F00090001C01DC549C5
:1096B0002039487707E0C3482038407F000900017F
:1096C000C0492039487702202040002809D0BD48F1
:1096D0002038007F00090001C01DBA4920390877F1
:1096E00007E0B8482038007F00090001B54920395B
:1096F000087704202040002809D0B2482038C07ED6
:1097000000090001C01DAF492039C87607E0AD4807
:109710002038C07E00090001AA492039C8760820F7
:109720002040002809D0A7482038807FF0218843B6
:109730007030A4492039887707E0A2482038807F1C
:10974000F02188439F492039887710202040002845
:1097500009D09C482038807F00090001C01D99492C
:109760002039887707E097482038807F000900017A
:109770009449203988772020204000280BD0914838
:109780002038407FF02100E0C5E0884370308D49EB
:109790002039487707E08B482038407FF021884304
:1097A00088492039487740202040002809D0854842
:1097B0002038C07EF0218843703082492039C87635
:1097C00007E080482038C07EF02188437D49203959
:1097D000C8760A210398EEF7B3FC0F467A48C45DB9
:1097E000E007C00F002809D076482038407E0009E5
:1097F0000001C01D73492039487607E071482038C0
:10980000407E000900016F4920394876022020403F
:10981000002809D06B482038007EF0218843703042
:1098200068492039087607E066482038007EF02134
:10983000884364492039087604202040002809D054
:1098400060482038C07DF021884370305D49203960
:10985000C87507E05B482038C07DF021884359492E
:109860002039C87508202040002809D055482038E4
:10987000C07D00090001C01D52492039C87507E0AC
:1098800050482038C07D000900014E492039C87574
:1098900010202040002809D04A482038807E000946
:1098A0000001C01D47492039887607E04548203827
:1098B000807E00090001434920398876202020401D
:1098C000002809D03F482038407EF021884370307E
:1098D0003C492039487607E03A482038407EF0215C
:1098E000884338492039487640202040002809D054
:1098F00034482038007E00090001C01D314920395C
:10990000087629E12F482038007E000900012D4902
:109910002039087620E12B482038C07EF02188438A
:10992000703028492039C8760846007E00090001B9
:10993000C01D08760846407F0009000148770846A8
:10994000007F0009000108770846C07E0009000179
:10995000C8760846807FF02188431A4920398877E5
:109960000846807F0009000188770846407FF02183
:1099700088431449203948770846407E0009000191
:1099800048760846007EF02188430E492039087643
:109990000846C07DF02188430A492039C875084629
:1099A000C07D00090001C8750846807E00090001DD
:1099B00088760846407EF02188430249203948765F
:1099C000CAE000002C22002038F301006348C07E6A
:1099D000F02188436149C8760846007E00090001ED
:1099E00008760846407F0009000148770846007F56
:1099F0000009000108770846C07E00090001C8760A
:109A00000846807FF0218843544988770846807F44
:109A10000009000188770846407FF02188434F49BC
:109A200048770846407E0009000148760846007ED7
:109A3000F0218843494908760846C07DF0218843D3
:109A40004649C8750846C07D00090001C87508462A
:109A5000807E0009000188760846407EF021884318
:109A60003E494876084620304079F02188433B49FA
:109A70002031487108468078000900018870084646
:109A8000C07900090001C871084680790009000109
:109A90008871084640790009000148710846007A3B
:109AA000F02188432D49203108720846007A0009C8
:109AB000000108720846C079F02188432749203107
:109AC000C8710846C07800090001C870084680784F
:109AD000F021884321492031887008464078F021E0
:109AE00088431E492031487008464078000900012B
:109AF0004870084600790009000108710846C078DE
:109B0000F021884315492031C8701448807D000930
:109B10000001203988750846807DF02188430F496F
:109B200088750846807EF02188430C49887608466F
:109B3000007FF021884309490877084620300079E2
:109B4000F021884305492031087108468079F021C9
:109B5000884302492031887105B0F0BD0C220020F5
:109B6000F7B582B00D4617460026029801287CD131
:109B7000632D0ADD0121FF200630FBF765F8012186
:109B8000FF200730FBF760F816E0092D0ADD012100
